:020000040000FA
:080000000002040000000000F2
:04000C007C1F000055
:100010007C1F0000CA1F00007C1F00007C1F000026
:100020007C1F00007C1F00007C1F00007C1F000064
:100030007C1F00007C1F00007C1F00007C1F000054
:100040007C1F00007C1F00007C1F00007C1F000044
:100050007C1F0000B01F00007C1F00007C1F000000
:100060007C1F00007C1F00007C1F00007C1F000024
:100070007C1F00007C1F00007C1F00007C1F000014
:100080007C1F00007C1F00007C1F00007C1F000004
:100090007C1F00007C1F00007C1F00007C1F0000F4
:1000A000022000007C1F00007C1F00007C1F00005D
:1000B0007C1F00007C1F00007C1F00007C1F0000D4
:1000C0007C1F00007C1F00007C1F00007C1F0000C4
:1000D0007C1F00007C1F00007C1F00007C1F0000B4
:1000E0007C1F00007C1F00007C1F00007C1F0000A4
:1000F0007C1F00007C1F00007C1F00007C1F000094
:100100007C1F00007C1F00007C1F00007C1F000083
:100110007C1F00007C1F00007C1F00007C1F000073
:100120007C1F00007C1F00007C1F00007C1F000063
:100130007C1F00007C1F00007C1F00007C1F000053
:100140007C1F00007C1F00007C1F00007C1F000043
:100150007C1F00007C1F00007C1F00007C1F000033
:100160007C1F00007C1F00007C1F00007C1F000023
:100170007C1F00007C1F00007C1F00007C1F000013
:100180007C1F00007C1F00007C1F00007C1F000003
:100190007C1F00007C1F00007C1F00007C1F0000F3
:1001A0007C1F00007C1F00007C1F00007C1F0000E3
:1001B0007C1F00007C1F00007C1F00007C1F0000D3
:1001C0007C1F00007C1F00007C1F00007C1F0000C3
:1001D0007C1F00007C1F00007C1F00007C1F0000B3
:1001E0007C1F00007C1F00007C1F00007C1F0000A3
:1001F0007C1F00007C1F00007C1F00007C1F000093
:10040000404424004005880000802000E1FF2100D6
:10041000018009000018EB002060EF0004002800B4
:10042000841188000440200094118800A40020005A
:10043000C41188002C23EF002A23EF000FF82100BD
:10044000F0FF210020A0B700000000000028EF000E
:100450005468EF005568EF00E4112200044488005E
:10046000141622001444880024C123002444880068
:10047000140424003444880014C227004444880033
:100480008443250054448800645525006444880052
:100490008401220074448800545525008444880057
:1004A000548527009444880004522500A444880001
:1004B00044552500B444880084072200C4448800C1
:1004C00054652500D444880044852700E44488000E
:1004D00004422500F4448800544525000445880062
:1004E00084C7210014458800242226002445880062
:1004F00024022100344588008453250044458800A7
:1005000054552500544588008481230064458800A3
:100510005445250074458800548521008445880091
:10052000844325009445880054652500A44588002F
:1005300084012000B445880054C42700C4458800C5
:1005400014042000D445880004502400E4458800A9
:10055000D4172400F4458800C028EF0054E4270095
:100560001446880004042000244688008457210093
:10057000344688004451210044468800848727007F
:100580005446880044512100644688004481270075
:1005900074468800C44725008446880064552500B9
:1005A0009446880044442200A446880044852700DD
:1005B000B446880044852400C4468800E49720009F
:1005C000D4468800E4972400E446880094842300FD
:1005D000F4468800545424000447880054842300BF
:1005E000144788008453240024478800445424007E
:1005F00034478800848323004447880054642400DF
:10060000544788004484230064478800C4132400AE
:10061000744788001414220084478800C4C723004C
:100620009447880014242400A447880004C22700AB
:10063000B4478800C4102500C4478800041525006D
:10064000D4478800C4832300E4478800544424002E
:10065000F44788005484230004488800C41324000D
:10066000144888000414240024488800C40320008F
:10067000344888000829EF000A29EF00048224008A
:1006800064488800E493240074488800240620000D
:10069000844888001229EF001429EF001629EF0082
:1006A0001829EF0004002400D448880084E62300C1
:1006B000E448880094202000F44888000442250083
:1006C00004498800645525001449880084072000E7
:1006D0002449880044E42700344988001404200099
:1006E0004449880084432400544988006454240009
:1006F0006449880084C323007449880004242400CA
:100700008449880014C2270094498800C4972000B7
:10071000A449880054502000B449880084C72700A9
:10072000C449880094102100D449880014C22700CD
:10073000E4498800E4572200F4498800546222000A
:10074000044A880080C1B30042E9B70004202000B9
:10075000845E880004102000945E88000408200055
:10076000A45E880004042000B45E88000402200017
:10077000C45E880004012000D45E8800840020004C
:10078000E45E880044002000F45E8800240020001D
:10079000045F880014002000145F8800C42D20002E
:1007A000245F8800E4162000345F8800740B20006A
:1007B000445F880074282000545F8800F4392000CA
:1007C000645F880034312000745F88005435200055
:1007D000845F880064372000945F8800B41B200089
:1007E000A45F880014202000B45F8800C43D20006E
:1007F000C45F8800E41E2000D45F8800740F2000CE
:10080000E45F8800742A2000F45F8800F438200038
:1008100004608800B431200014608800843D20000A
:1008200024608800443D200034608800C4252000F6
:1008300044608800C43C2000546088008425200067
:100840006460880097C0A900040E2000140288008C
:100850002CA3EF002AA3EF00040024003416880024
:1008600004082000641688000450200094168800B4
:1008700044012000F4168800042021002417880079
:10088000CA02A900C602A90040A7A900CA02A9007D
:10089000C602A9000100200001007800861B0200AA
:1008A000000000008100E8003322AF00FEFF3700A7
:1008B000A0118800300220000008E600F6FF370093
:1008C00044200200000000007A2402000000000022
:1008D0008C250200000000003A6DEF003B6DEF0038
:1008E000A62002000000000006E8A8000500200085
:1008F00005007800B81B0200000000000040B300B3
:100900004220AF00050037008502E80036EDB70051
:100910002424020000000000F5FF37003A6DEF00CC
:1009200010C0B3003BEDB700A6200200000000009D
:1009300006E8A9000500200005007800D41B02008D
:10094000000000000040B3004220AF000500370067
:100950008502E80036EDB700242402000000000004
:10096000F5FF370020C0B30030EDB7002E240200A1
:100970000000000030C0B30030EDB7002E240200AC
:10098000000000003A6DEF0040C0B3003BEDB7003F
:10099000A6200200000000000500200005007800ED
:1009A000F01B0200000000000040B3004220AF0036
:1009B000050037008502E80036EDB7002424020068
:1009C00000000000F5FF370050C0B30030EDB70065
:1009D0002E2402000000000030C0B3003AEDB70042
:1009E00050C0B3003BEDB700A6200200000000009D
:1009F00005002000050078000C1C0200000000002B
:100A00000040B3004220AF00050037008502E80037
:100A100036EDB7002424020000000000F5FF370087
:100A2000401F2000641F020000000000F0260200AA
:100A300000000000727C0200000000002768EF0048
:100A400020C0B3005CECB700D078020000000000CA
:100A500000C3B3001CEDB7001D6DEF00B428020009
:100A60000000000050C3B3001CEDB7001D6DEF0087
:100A7000B4280200000000000F4CE20003003A001E
:100A8000A834020000000000C76BEF000628A80091
:100A900010C0B3000CE8B70058E8EF00D222EF0016
:100AA00004802000B4168800000000000000000050
:100AB000F43F200094168800D742A800D342A90032
:100AC0000000000000000000D242A800D442AE00A6
:100AD0001D0037000500200005007800261C0200DC
:100AE000000000000040B3004220AF0006003700C5
:100AF0008502E8003322AF00FEFF370034E2B70082
:100B00003562EF00F4FF37003322AF00FEFF3700FD
:100B100004022000A41188001EEDEF00C41F200075
:100B2000E4688800362B020000000000304A020012
:100B3000000000006452020000000000DC790200A6
:100B4000000000008560A9007A2502000000000076
:100B500097C0A8004220EF0054C8BF005548E300EA
:100B600003003200D27E020000000000FAFF3700CE
:100B70009560A90097C0A900040E20001402880007
:100B80000F4CE20002003A00B05F020000000000DB
:100B90008E8C0200000000000290020000000000A5
:080BA000EBFF37000040FE00EE
:0C2004003220EF00C30A200083015000CE
:1020100005003100E3012100008041001040BA00BA
:102020000160EF0000000600F00121008381410003
:10203000808141001380BA000000060080E00000AB
:10204000F8FC00003E0E00000F070C0007070E0012
:10205000070F0E001E7C0E00F8F01E0080FF1F0010
:10206000FFFF3700000077000000E3000000E10000
:10207000000080000000000000FF0000FFFF1C00C7
:10208000010F3C001F3F7C0078F07000E0E0F000A2
:10209000E0E0E000E070E000783FE0001F07E000D3
:1020A0000000E000000070000000780070783F0041
:1020B0003CFE1F00FFFF0F000000000000000000BA
:1020C0000000000000000000000000000000000010
:1020D00000000000FFFFC000FF00E0000000F8006B
:1020E00000007C0000001E000000FF000000FF0058
:1020F000E0E0FF00E0FF0000FFFF0000E0E0000084
:10210000E00000000000E0000030F000383CF80083
:102110001E0EFE000707DF000707CF000F0EC300EB
:10212000FEFCC100F800C0000000C0000000FF007D
:1021300080C0FF00E0F0FF007038C0003C1EC0000F
:102140000F0FC0000300000000000100007C010030
:10215000FFFF0100E3E10100E0E00100E0E0010039
:10216000E0E00100E0E00100C0000100000001002B
:10217000001CFF001E0EFF000E07FF0007070100F6
:10218000070F01000EFE0100FCF00000000000003F
:10219000000000003220EF00C30A2000830150003D
:1021A00005003100630E2100008041001040BA009C
:1021B0000160EF0000000600700E210083814100E5
:1021C000808141001380BA00000006000083F30004
:1021D000FFFFFF007F877F0087C73F00C7C71E0044
:1021E000C7C70E00C7870E0007030E0000001F00C0
:1021F0001F1F3F001F0F7B000703F9000101F000C4
:102200000101C0000103000007FF0000FEF80F00FD
:10221000001C3F003C7C7F0070E07800E0E0F000B4
:10222000E0E0E000F070E000783EE0001F0FE0002A
:102230000300E0000000F00080E07800F0787F000C
:102240003C1E3F000F070F00030000000000E000ED
:102250000000F80000F8FC00FFFF3E001F1D0E000C
:102260000C0E0F000E0E07000E0E07001E3C07009E
:10227000FCF80700E0000F00071F1E003F7C3E0037
:1022800070F0FC00E0E0F800E0E0E000F07000003A
:102290007C3F0F001F071F0007073F00070778005C
:1022A000070770000707F00007C7E000E7F7E00046
:1022B0007F3FE0001F0FE00003007000000070008F
:1022C0000000F80080F0FF00FCFFFF003F071F0048
:1022D0000100000000000000000080000000C000BD
:1022E00040F0C000FE7FE0001F03E0000000E000BF
:1022F00000007000000078000000380000001E00A0
:10230000F0FC1F00FC1E07000F070300070700007A
:10231000070700008FFE0000FCF80000000000002E
:1023200000C100003220EF00030A200083015000AA
:1023300005003100E31A2100008041001040BA007E
:102340000160EF0000000600F01A210083814100C7
:10235000808141001380BA000000060000003200B6
:102360000000490000007900005F410000003E00CD
:1023700000077E0000071100001411007F141100F7
:102380007F147E00242A7F007F2A490012234900FF
:10239000130849006462360036493E005522410068
:1023A000500041000503410000002200001C7F0096
:1023B0002241410000004100412222001C001C007B
:1023C00014087F003E08490014084900083E4900EF
:1023D0000808410000507F00300009000008090093
:1023E000080809000808010000603E006000410084
:1023F000002049001008490004027A003E517F0085
:10240000494508003E000800427F080040007F0068
:10241000426100005149410046217F004145410091
:102420004B31000018142000127F4000102741009B
:1024300045453F00453901003C4A7F0049490800B5
:1024400030011400710922000503410036497F0064
:10245000494940003606400049494000291E4000D5
:1024600000367F003600020000000C0056360200E5
:1024700000007F0008147F002241040000140800BF
:102480001414100014147F0000413E002214410077
:10249000080241000151410009063E003220EF00D0
:1024A000030A20008301500005003100A32621000B
:1024B000008041001040BA000160EF0000000600FB
:1024C000B026210083814100808141001380BA0041
:1024D000000006007F097C0009091400063E140074
:1024E00041511400215E08007F09080019291400D9
:1024F000464614004949180049317C0001017C001E
:102500007F010800013F040040400400403F0800F4
:102510001F204800402054001F3F54004038540002
:10252000403F20006314040008143F006307440088
:10253000087040000807200061513C0049454000F8
:10254000430040007F41200041007C0002041C0049
:102550000810200020004000414120007F001C00A6
:1025600004023C00010240000440300040404000B2
:1025700040403C00000144000204280000201000FC
:1025800054542800547844007F480C0044445000C0
:10259000383850004444500044203C003844440043
:1025A000444864007F38540054544C00541844008C
:1025B000087E000009010800020C3600525241005A
:1025C000523E00007F0800000404000078007F00F5
:1025D000447D00004000000020400000443D4100D8
:1025E000007F360010280800440000000041100061
:1025F0007F400800007C08000418100004780800E0
:102600007C087800040446007838410044444600C1
:10261000443878003220EF0063312100008041000F
:102620001040BA000160EF00000006004C430000BB
:10263000440000003220EF0063322100008041009E
:102640001040BA000160EF00000006004272000076
:1026500069670000687400006E6500007373000015
:10266000000000003220EF00E33321000080410031
:102670001040BA000160EF00000006004164000055
:102680006A75000073740000000000003220EF0043
:1026900023352100008041001040BA000160EF00A6
:1026A00000000600546500006368000044650000F7
:1026B00073690000676E00002E6200006500000074
:1026C0003220EF00C3362100008041001040BA00E4
:1026D0000160EF0000000600566F0000703D000032
:1026E0002025000075200000000000003220EF00CF
:1026F00023382100008041001040BA000160EF0043
:102700000000060020200000202000002020000003
:1027100020200000202000002020000020200000B9
:10272000000000003220EF00E3392100008041006A
:102730001040BA000160EF00000006002D2D0000DF
:102740002D2D00002D2D00002D2D0000000000007B
:102750003220EF00C301200083015000050031004A
:10276000433C2100008041001040BA000160EF00AE
:1027700000000600503C210083814100808141001F
:102780001380BA0000000600202020002020200036
:1027900020202000202020002020200020202000B9
:1027A00020202000202020002020200020202000A9
:1027B00020202000202020002020200020200000B9
:1027C0003220EF00C33E2100008041001040BA00DB
:1027D0000160EF0000000600202000002020000023
:1027E00020200000202000002020000020200000E9
:1027F00020200000202000002020000020200000D9
:1028000020200000200000003220EF0003412100C2
:10281000008041001040BA000160EF000000060097
:102820004D6F00006E0000003220EF0003422100D7
:10283000008041001040BA000160EF000000060077
:1028400054750000650000003220EF0003432100B2
:10285000008041001040BA000160EF000000060057
:1028600057650000640000003220EF00034421009F
:10287000008041001040BA000160EF000000060037
:1028800054680000750000003220EF00034521006D
:10289000008041001040BA000160EF000000060017
:1028A00046720000690000003220EF00034621005C
:1028B000008041001040BA000160EF0000000600F7
:1028C00053610000740000003220EF000347210034
:1028D000008041001040BA000160EF0000000600D7
:1028E000537500006E0000003220EF000348210005
:1028F000008041001040BA000160EF0000000600B7
:102900004A6100006E0000003220EF000349210000
:10291000008041001040BA000160EF000000060096
:1029200046650000620000003220EF00034A2100EB
:10293000008041001040BA000160EF000000060076
:102940004D610000720000003220EF00034B2100B7
:10295000008041001040BA000160EF000000060056
:1029600041700000720000003220EF00034C210093
:10297000008041001040BA000160EF000000060036
:102980004D610000790000003220EF00034D21006E
:10299000008041001040BA000160EF000000060016
:1029A0004A7500006E0000003220EF00034E210047
:1029B000008041001040BA000160EF0000000600F6
:1029C0004A7500006C0000003220EF00034F210028
:1029D000008041001040BA000160EF0000000600D6
:1029E00041750000670000003220EF000350210015
:1029F000008041001040BA000160EF0000000600B6
:102A000053650000700000003220EF0003512100E8
:102A1000008041001040BA000160EF000000060095
:102A20004F630000740000003220EF0003522100C9
:102A3000008041001040BA000160EF000000060075
:102A40004E6F0000760000003220EF00035321009B
:102A5000008041001040BA000160EF000000060055
:102A600044650000630000003220EF0003542100A1
:102A7000008041001040BA000160EF000000060035
:102A80000A0D0000205400004D43000020540000B7
:102A90003D25000075200000463D00002575000022
:102AA00020440000503D000025750000000000009B
:102AB0003220EF0043562100008041001040BA0050
:102AC0000160EF0000000600204400003D250000EA
:102AD0007520000064690000723D0000257500004B
:102AE00020450000585400003D25000075000000FE
:102AF0003220EF0043582100008041001040BA000E
:102B00000160EF0000000600204500005654000060
:102B10003D2500004C750000204C00004F43000094
:102B20003D2500004C750000000000003220EF0041
:102B3000235A2100008041001040BA000160EF00DC
:102B40000000060020430000433D000025780000FF
:102B5000204C0000544E00003D250000780000008D
:102B60003220EF00C35B2100008041001040BA001A
:102B70000160EF00000006002053000049440000FF
:102B80003D25000078200000000000003220EF000A
:102B9000235D2100008041001040BA000160EF0079
:102BA0000000060065720000723000003120000055
:102BB000000000003220EF00635E21000080410031
:102BC0001040BA000160EF000000060073740000BE
:102BD000696E00003D200000257500002A200000DD
:102BE000000000003220EF00E35F21000080410080
:102BF0001040BA000160EF000000060074610000A0
:102C0000733D000020250000752A00002000000010
:102C10003220EF0043612100008041001040BA00E3
:102C20000160EF0000000600206C000065760000E7
:102C3000656C00003D25000030330000750A00007F
:102C40000D0000003220EF00E3622100008041000F
:102C50001040BA000160EF00000006002D2D0000BA
:102C60002D0000003220EF00E363210000804100CE
:102C70001040BA000160EF0000000600202A0000AA
:102C80002A200000626100006E64000020630000E2
:102C9000686100006E670000652000006672000039
:102CA0006F6D000020250000752000002A2A00001A
:102CB000200000003220EF00636621000080410008
:102CC0001040BA000160EF00000006000A0D00008D
:102CD000204600004D200000253300002E32000069
:102CE000672000004D6800005A0000003220EF000D
:102CF00023682100008041001040BA000160EF000D
:102D000000000600464D0000200000003220EF00C9
:102D100023692100008041001040BA000160EF00EB
:102D200000000600204D0000572000002534000060
:102D30002E320000672000006B6800005A0000007F
:102D40003220EF00C36A2100008041001040BA0029
:102D50000160EF00000006004D5700002000000059
:102D60003220EF00C36B2100008041001040BA0008
:102D70000160EF00000006006B6800005A000000D0
:102D80003220EF00C36C2100008041001040BA00E7
:102D90000160EF0000000600204C000057200000FA
:102DA000253300002E320000672000006B68000011
:102DB0005A0000003220EF00636E210000804100C5
:102DC0001040BA000160EF00000006004C57000000
:102DD000200000003220EF00636F210000804100DE
:102DE0001040BA000160EF00000006002053000010
:102DF0005731000020250000342E0000326700000B
:102E0000204D0000685A0000000000003220EF0052
:102E100023712100008041001040BA000160EF00E2
:102E200000000600535700003120000000000000A1
:102E30003220EF0043722100008041001040BA00B0
:102E40000160EF0000000600205300005732000030
:102E500020250000352E000032670000204D0000C4
:102E6000685A0000000000003220EF0003742100C7
:102E7000008041001040BA000160EF000000060031
:102E80005357000032200000000000003220EF0005
:102E900023752100008041001040BA000160EF005E
:102EA000000006004D6800005A0000003220EF00CC
:102EB00023762100008041001040BA000160EF003D
:102EC00000000600205300005733000020250000BA
:102ED000352E000032670000204D0000685A0000C7
:102EE000000000003220EF00E37721000080410065
:102EF0001040BA000160EF000000060053570000C8
:102F000033200000000000003220EF000379210090
:102F1000008041001040BA000160EF000000060090
:102F2000205300005734000020250000352E0000FB
:102F300032670000204D0000685A000000000000C9
:102F40003220EF00C37A2100008041001040BA0017
:102F50000160EF000000060053570000342000001D
:102F6000000000003220EF00E37B210000804100E0
:102F70001040BA000160EF00000006004946000062
:102F80004341000050200000616C000069670000B0
:102F90006E200000310000003220EF00837D210010
:102FA000008041001040BA000160EF000000060000
:102FB000204900004643000041500000206100000D
:102FC0006C690000676E00002031000020000000E6
:102FD0003220EF00437F2100008041001040BA0002
:102FE0000160EF0000000600204900004643000099
:102FF000415000003D2500003375000020200000F6
:10300000000000003220EF00E3802100008041003A
:103010001040BA000160EF000000060049460000C1
:1030200043410000503D0000000000003220EF004E
:1030300023822100008041001040BA000160EF00AF
:1030400000000600494600004346000020610000E1
:103050006C690000676E0000000000003220EF0085
:10306000A3832100008041001040BA000160EF00FE
:1030700000000600204900004643000046200000F2
:10308000616C0000696700006E2000000000000015
:103090003220EF0043852100008041001040BA003B
:1030A0000160EF0000000600506C00006561000048
:1030B0007365000020770000616900007400000063
:1030C0003220EF00C3862100008041001040BA008A
:1030D0000160EF0000000600206400006966000047
:1030E0006625000064200000000000003220EF0090
:1030F00023882100008041001040BA000160EF00E9
:103100000000060020630000665F0000763D0000BE
:1031100025750000200000003220EF008389210087
:10312000008041001040BA000160EF00000006007E
:103130002049000046430000463D000025330000C2
:103140007520000020200000000000003220EF0069
:10315000238B2100008041001040BA000160EF0085
:103160000000060049460000434600003D00000004
:103170003220EF00438C2100008041001040BA0053
:103180000160EF00000006004946000043460000D1
:10319000206100006C690000676E00003F200000A5
:1031A000000000003220EF00E38D2100008041008C
:1031B0001040BA000160EF0000000600454E00001C
:1031C00054450000523A0000206100006363000093
:1031D00065700000740000003220EF00838F210032
:1031E000008041001040BA000160EF0000000600BE
:1031F0003C2000003E200000746F000020630000AF
:10320000616E0000636500006C200000000000009B
:103210003220EF0043912100008041001040BA00AD
:103220000160EF00000006000A0D0000202A0000E7
:103230002A4900004643000046200000616C00005F
:10324000696700006E3F00002A2A0000200000008D
:103250003220EF0043932100008041001040BA006B
:103260000160EF0000000600204500004E54000001
:1032700045520000207400006F20000061630000D0
:103280006365000070740000000000003220EF0051
:1032900023952100008041001040BA000160EF003A
:1032A00000000600203C0000203E000020740000CA
:1032B0006F200000636100006E630000656C000019
:1032C000200A00000D0000003220EF0003972100CB
:1032D000008041001040BA000160EF0000000600CD
:1032E0002A200000494600004346000020610000FB
:1032F0006C690000676E0000202A000000000000DA
:103300003220EF00C3982100008041001040BA0035
:103310000160EF0000000600506C000065610000D5
:103320007365000020740000756E000065200000C9
:10333000746F0000000000003220EF00839A21002B
:10334000008041001040BA000160EF00000006005C
:10335000612000006B6E00006F7700006E2000009F
:10336000667200006571000020200000000000006F
:103370003220EF00439C2100008041001040BA0041
:103380000160EF00000006006E6500006172000041
:1033900020390000382E0000302000004D68000069
:1033A0005A200000000000003220EF00039E2100A0
:1033B000008041001040BA000160EF0000000600EC
:1033C0002B20000070720000657300007320000065
:1033D000454E000054450000522E00000000000041
:1033E0003220EF00C39F2100008041001040BA004E
:1033F0000160EF00000006000A0D00002A2A00000C
:103400002A200000494600004346000020610000D9
:103410006C690000676E0000202000002A2A00006E
:103420002A200000000000003220EF0003A221004B
:10343000008041001040BA000160EF00000006006B
:10344000506C00006561000073650000207400008E
:10345000756E000065200000746F000020610000A0
:10346000200000003220EF00E3A321000080410093
:103470001040BA000160EF00000006006B6E000013
:103480006F7700006E20000073740000617400000C
:10349000696F00006E2000006E6500006172000020
:1034A00020390000382E0000302000004D68000058
:1034B0005A200000000000003220EF0083A6210007
:1034C000008041001040BA000160EF0000000600DB
:1034D000616E0000642000007072000065730000DF
:1034E00073200000454E000054450000522E00009D
:1034F0000A0D0000200000003220EF0083A8210008
:10350000008041001040BA000160EF00000006009A
:10351000747500006E6500002B4500004E540000DD
:1035200045520000000000003220EF0003AA2100F5
:10353000008041001040BA000160EF00000006006A
:10354000496E000069740000207000007265000080
:1035500073650000747300003F0000003220EF002C
:10356000A3AB2100008041001040BA000160EF00D1
:10357000000006003C2000003E200000746F0000A8
:1035800020630000616E0000636500006C000000B5
:103590003220EF0043AD2100008041001040BA000E
:1035A0000160EF0000000600202A00002A49000008
:1035B0006E690000742000007072000065730000E6
:1035C00065740000733F00002A2A000020000000FC
:1035D0003220EF0043AF2100008041001040BA00CC
:1035E0000160EF000000060020500000757300002D
:1035F00068200000454E00005445000052200000A5
:10360000746F0000206100006363000065700000BB
:1036100074200000000000003220EF0083B1210080
:10362000008041001040BA000160EF000000060079
:10363000205000007265000073730000203C000001
:10364000203E0000207400006F2000006361000035
:103650006E630000656C0000200000003220EF0067
:10366000A3B32100008041001040BA000160EF00C8
:1036700000000600696E0000697400002070000000
:1036800072650000736500007473000000000000A4
:103690003220EF0043B52100008041001040BA0005
:1036A0000160EF0000000600446500006661000054
:1036B000756C000074200000696E000074650000E5
:1036C0007272000075700000740D00000A000000A6
:1036D0003220EF0043B72100008041001040BA00C3
:1036E0000160EF00000006005374000061630000F9
:1036F0006B200000696E00007465000072720000AB
:1037000075700000740D00000A0000003220EF0008
:1037100023B92100008041001040BA000160EF0091
:10372000000006000A0D000020690000303400008F
:10373000312000002D200000547500006E6500004F
:10374000722000004D6F0000647500006C65000081
:10375000204900006E740000657200006661000080
:1037600063650000202000000A0D0000000000003A
:103770003220EF0043BC2100008041001040BA001D
:103780000160EF000000060020540000756E00008C
:1037900065720000204D00006F640000756C000031
:1037A00065200000000000003220EF0003BE210071
:1037B000008041001040BA000160EF0000000600E8
:1037C0006930000034310000206900006E74000090
:1037D0006572000066610000636500000000000083
:1037E0003220EF00C3BF2100008041001040BA002A
:1037F0000160EF0000000600206F00006D6E000009
:10380000696200006F610000726400002E620000B7
:1038100065200000000000003220EF0083C121007D
:10382000008041001040BA000160EF000000060077
:10383000746500006368000064650000736900003F
:10384000676E00002E620000650000003220EF006D
:1038500023C32100008041001040BA000160EF0046
:1038600000000600202A00002A6900006E6900009E
:103870003D3000002A2A0000200000003220EF0026
:10388000A3C42100008041001040BA000160EF0095
:1038900000000600202A00002A6500006E74000067
:1038A000657200002A2A0000200000003220EF008C
:1038B00023C62100008041001040BA000160EF00E3
:1038C00000000600202A00002A6C00006566000047
:1038D000742A00002A200000000000003220EF00BF
:1038E000A3C72100008041001040BA000160EF0032
:1038F00000000600202A00002A720000696700000C
:10390000687400002A2A0000200000003220EF0026
:1039100023C92100008041001040BA000160EF007F
:1039200000000600202A00002A750000702A00000E
:103930002A200000000000003220EF0083CA21008E
:10394000008041001040BA000160EF000000060056
:10395000207600006F6C0000756D0000653D000072
:1039600025750000200000003220EF0003CC21006C
:10397000008041001040BA000160EF000000060026
:10398000202A00002A6400006F7700006E2A0000E1
:103990002A200000000000003220EF0083CD21002B
:1039A000008041001040BA000160EF0000000600F6
:1039B00020500000533D000025730000000000006F
:1039C0003220EF00C3CE2100008041001040BA0039
:1039D0000160EF000000060020500000493D00009B
:1039E000254C0000780000003220EF0003D02100B9
:1039F000008041001040BA000160EF0000000600A6
:103A00002020000020200000000000003220EF00F5
:103A100023D12100008041001040BA000160EF0076
:103A200000000600746D0000630000003220EF000B
:103A300023D22100008041001040BA000160EF0055
:103A40000000060054410000200000003220EF007A
:103A500023D32100008041001040BA000160EF0034
:103A60000000060054500000200000003220EF004B
:103A700023D42100008041001040BA000160EF0013
:103A80000000060020200000200000003220EF008F
:103A900023D52100008041001040BA000160EF00F2
:103AA00000000600544D0000430000003220EF00EB
:103AB00023D62100008041001040BA000160EF00D1
:103AC00000000600544100002072000000000000C9
:103AD0003220EF0043D72100008041001040BA009F
:103AE0000160EF000000060020430000545F00006A
:103AF0004D4A0000443D0000256C000075000000A8
:103B00003220EF00C3D82100008041001040BA00ED
:103B10000160EF000000060020430000543D00005B
:103B200025300000317500003A0000003220EF001F
:103B300023DA2100008041001040BA000160EF004C
:103B40000000060020520000546100003D250000E6
:103B5000730A00000D0000003220EF0083DB21001B
:103B6000008041001040BA000160EF000000060034
:103B700020520000546200003D250000730A00003E
:103B80000D0000003220EF00E3DC21000080410046
:103B90001040BA000160EF0000000600202A00007B
:103BA0002A200000676F0000746F00002070000082
:103BB0007265000073650000742000002575000028
:103BC000202A00002A200000000000003220EF0020
:103BD00023DF2100008041001040BA000160EF00A7
:103BE00000000600207700005F5000004C4C0000F1
:103BF0003D2500006C750000200000003220EF0021
:103C0000A3E02100008041001040BA000160EF00F5
:103C100000000600202A00002A2000007361000036
:103C2000766500002070000072650000736500007A
:103C30007420000025750000202A00002A200000C2
:103C4000000000003220EF00E3E22100008041008C
:103C50001040BA000160EF00000006002063000081
:103C60005F66000072650000713D000025300000B5
:103C7000332E000032660000200000003220EF00EA
:103C8000A3E42100008041001040BA000160EF0071
:103C900000000600206300005F5000004C4C000054
:103CA0003D2500006C750000200000003220EF0070
:103CB00023E62100008041001040BA000160EF00BF
:103CC0000000060066720000640000003220EF0071
:103CD00023E72100008041001040BA000160EF009E
:103CE0000000060066720000750000003220EF0040
:103CF00023E82100008041001040BA000160EF007D
:103D00000000060067660000720000003220EF002D
:103D100023E92100008041001040BA000160EF005B
:103D20000000060073660000720000003220EF0001
:103D300023EA2100008041001040BA000160EF003A
:103D400000000600616C0000610000003220EF00FE
:103D500023EB2100008041001040BA000160EF0019
:103D600000000600616C0000620000003220EF00DD
:103D700023EC2100008041001040BA000160EF00F8
:103D800000000600696E0000690000003220EF00AC
:103D900023ED2100008041001040BA000160EF00D7
:103DA00000000600202A00002A660000726400005D
:103DB0003D3000002A2A0000200000003220EF00E1
:103DC000A3EE2100008041001040BA000160EF0026
:103DD00000000600202A00002A660000727500001C
:103DE0003D3000002A2A0000200000003220EF00B1
:103DF00023F02100008041001040BA000160EF0074
:103E000000000600202A00002A67000066720000F9
:103E10003D3000002A2A0000200000003220EF0080
:103E2000A3F12100008041001040BA000160EF00C2
:103E300000000600202A00002A73000066720000BD
:103E40003D3000002A2A0000200000003220EF0050
:103E500023F32100008041001040BA000160EF0010
:103E600000000600202A00002A6100006C610000AA
:103E70003D3000002A2A0000200000003220EF0020
:103E8000A3F42100008041001040BA000160EF005F
:103E900000000600202A00002A6100006C62000079
:103EA0003D3000002A2A0000200000003220EF00F0
:103EB00023F62100008041001040BA000160EF00AD
:103EC00000000600000000000000E0004220AF00FB
:103ED00008003700190E0900000000000500090065
:103EE00000000000FF3F0900000000000000E900A2
:103EF000F5FF3700000006003600F800801F78004C
:103F0000200020000C000900B01F780001002000F4
:103F100001007800481B0200000000008100E8005A
:103F20003322AF00FEFF3700A011880020012000DF
:103F30000008E600F6FF3700803E2000641F020004
:103F4000000000000000FE00A00120000C0009009D
:103F50004F1078004F0078003600F900004006004E
:103F60003600F800801F7800200020000C000900B7
:103F7000B01F7800000000008560A900A0012000AB
:103F80000C0009004F1078004F0078003600F9004F
:103F9000004006003600F800801F78002000200056
:103FA0000C000900B01F780001002000010078001B
:103FB000681B0200000000008100E8003322AF000F
:103FC000FEFF3700A0118800000120000008E60075
:103FD000F6FF3700803E2000641F02000000000052
:103FE0000000FE00000000008060A900A001200089
:103FF0000C0009004F1078004F0078003600F900DF
:10400000004006003600F800801F780020002000E5
:104010000C000900B01F7800A44280000960EF0086
:1040200043832000830242003202AE00FEFF3700CD
:10403000B0118000804A780054C8BF0056E8B7002D
:10404000A4428000614242000440780000E0B700D2
:104050007F40600054E8B70054C8BF005548E300F3
:1040600002003A0056C8BF0054E8B70087C0A90054
:10407000A00120000C0009004F1078004F007800CC
:104080003600F900004006000000000000000600B5
:10409000851F780080C0B3005DE9B7005D49E2008C
:1040A00018003200E842A900E442A900C600090055
:1040B000000000003FCDBF000048B2000004E00057
:1040C00003003A00E862A900E462A9000200370098
:1040D000E862A800E462A900C60009000000000030
:1040E000E842A800E442A900C60009000000000060
:1040F0003F6DD400C6000900000000005D69ED00BE
:10410000E6FF3700CF02780000000600D1A2A90028
:10411000C600090000000000CA22A900C622A900AA
:10412000C6000900000000003ECDBF003FEDB70013
:104130004820020000000000C60009000000000046
:10414000CA22A800C622A90000000600851F780028
:104150003BCDBF0067406000804278000544B3005B
:10416000054078003EEDB700862002000000000008
:104170003ACDBF00F047B200804278000548B30056
:10418000054078003EEDB7008620020000000000E8
:10419000CF02780000000600D1A2A800C6000900E6
:1041A00000000000CA22A900C622A900C60009001A
:1041B000000000003ACDBF003FEDB70048200200EC
:1041C00000000000C600090000000000CA22A8008C
:1041D000C622A90000000600244A80004822DE0012
:1041E00074CCB20003003A0000C8B30045E9B70040
:1041F00009013700244A80004822DE00C4CFB20003
:1042000003003A0010C8B30045E9B70002013700C7
:10421000244A80004822DE0094CEB20003003A0017
:1042200020C8B30045E9B700FB003700244A8000EE
:104230004822DE0024CEB20003003A0030C8B300AA
:1042400045E9B700F4003700244A80004822DE0028
:1042500044CEB20003003A0040C8B30045E9B700BD
:10426000ED003700244A80004822DE0004CEB20070
:1042700003003A0050C8B30045E9B700E600370034
:10428000244A80004822DE0054CEB20003003A00E7
:1042900060C8B30045E9B700DF003700244A80005A
:1042A0004822DE0074CEB20003003A0070C8B300AA
:1042B00045E9B700D8003700244A80004822DE00D4
:1042C000A4CEB20003003A0080C8B30045E9B700AD
:1042D000D1003700244A80004822DE00B4CEB2006C
:1042E00003003A0090C8B30045E9B700CA003700A0
:1042F000244A80004822DE0084CEB20003003A0047
:10430000A0C8B30045E9B700C3003700244A8000C5
:104310004822DE00F4CEB20003003A00B0C8B30079
:1043200045E9B700BC003700244A80004822DE007F
:10433000E4CEB20003003A00C0C8B30045E9B700BC
:10434000B5003700244A80004822DE00C4CEB20007
:1043500003003A00D0C8B30045E9B700AE0037000B
:10436000244A80004822DE0044CCB20003003A0018
:10437000E0C8B30045E9B700A7003700244A800031
:104380004822DE0054CCB20003003A00F0C8B3006B
:1043900045E9B700A0003700244A80004822DE002B
:1043A00094CCB20003003A0000C9B30045E9B7005D
:1043B00099003700244A80004822DE0064CEB20013
:1043C00003003A0010C9B30045E9B7009200370076
:1043D000244A80004822DE0064CCB20003003A0088
:1043E00020C9B30045E9B7008B003700244A80009C
:1043F0004822DE0044CFB20003003A0030C9B300C7
:1044000045E9B70084003700244A80004822DE00D6
:1044100064CFB20003003A0040C9B30045E9B700D9
:104420007D003700244A80004822DE0024CFB200FD
:1044300003003A0050C9B30045E9B70076003700E1
:10444000244A80004822DE00B4CFB20003003A00C4
:1044500060C9B30045E9B7006F003700244A800007
:104460004822DE0094CFB20003003A0070C9B300C6
:1044700045E9B70068003700244A80004822DE0082
:10448000F4CFB20003003A0080C9B30045E9B70099
:1044900061003700244A80004822DE0064CDB2006B
:1044A00003003A0090C9B30045E9B7005A0037004D
:1044B000244A80004822DE00C4CDB20003003A0046
:1044C000A0C9B30045E9B70053003700244A800073
:1044D0004822DE0084CFB20003003A00B0C9B30026
:1044E00045E9B7004C003700244A80004822DE002E
:1044F00034CAB20003003A00C0C9B30045E9B700AE
:1045000045003700244A80004822DE0084CDB200F6
:1045100003003A00D0C9B30045E9B7003E003700B8
:10452000244A80004822DE0074CDB20003003A0025
:10453000E0C9B30045E9B70037003700244A8000DE
:104540004822DE0034C8B20003003A00F0C9B300CC
:1045500045E9B70030003700244A80004822DE00D9
:1045600014CEB20003003A0000CAB30045E9B70018
:1045700029003700244A80004822DE00D4CEB20051
:1045800003003A0010CAB30045E9B7002200370023
:10459000244A80004822DE0034CFB20003003A00F3
:1045A00020CAB30045E9B7001B003700244A800049
:1045B0004822DE00A4CFB20003003A0030CAB300A4
:1045C00045E9B70014003700244A80004822DE0085
:1045D00014CFB20003003A0040CAB30045E9B70067
:1045E0000D003700244A80004822DE0014CDB200BE
:1045F00003003A0050CAB30045E9B700060037008F
:10460000244A80004822DE00F4CDB20002003A00C5
:1046100060CAB30045E9B70000000600851F7800B6
:10462000D1A2A800CA22A900C622A90080C0B30056
:104630005DE9B7005D49E20012003200E842A900DE
:10464000E442A900260009000000000037CDBF00A9
:10465000614060000004E00003003A00E862A90045
:10466000E462A90002003700E862A800E462A90041
:10467000E842A800E442A900376DD5005D69ED006D
:10468000ECFF3700CA22A800C622A900CF0278009A
:1046900000000600851F7800861F7800244A8000ED
:1046A0004822DE0003022000041CE1000200360064
:1046B0006200370007003700244A80004822DE00ED
:1046C000F3072000041CE10002003100EC2002008E
:1046D00000000000244A80004822DE00030220007F
:1046E000041CE1000100360054003700244A800019
:1046F0004822DE00630A2000041CE10001003100B2
:104700004E0037004369EF00144A80004822DE0063
:104710006524E10040003100244A80004822DE0088
:1047200003052000041CE1000C00360045C9BF0051
:104730000042B100004278000960EF006520B80037
:104740005CE9B7005CC9BF004349B40092110200A4
:104750000000000044E9B70023003700244A80002D
:104760004822DE0003082000041CE1000C00360093
:1047700045C9BF000045B100004278000960EF0064
:104780006520B8005CE9B7005CC9BF004349B400CC
:104790004E1202000000000044E9B700120037008A
:1047A000244A80004822DE00730A2000041CE10035
:1047B0000D00360045C9BF000048B1000042780036
:1047C0000960EF006520B8005CE9B7005CC9BF0074
:1047D0004349B4000080FB0004882000040040002E
:1047E0001040780044E9B70006E8AE000400370046
:1047F000244A8000F4CFB2000440780044E9B700B6
:1048000044C9BF003AEDB700CC2002000000000010
:104810004369EC00BCFF370006E8AF000400370036
:10482000376DEF000E230200000000000300370088
:1048300037EDEF000E230200000000004F03780068
:10484000CF0278000000060036CDBF0045E9B70072
:104850004A2302000000000000000600851F7800C7
:104860003A6DEF0030CDBF003BEDB700A62002004F
:10487000000000000500200005007800761302000B
:10488000000000000040B3004220AF0005003700E8
:104890008502E80036EDB700242402000000000085
:1048A000F5FF3700CF027800000006003A6DEF00F8
:1048B0003B6DEF00A620020000000000841F2000D6
:1048C000344A88004609E200050032003A6DEF00E4
:1048D000CC200200000000004629ED00F9FF37005F
:1048E00050C0B30030EDB7002E24020000000000DD
:1048F00000000600D1A2A800CA22A800C622A90072
:10490000D1C2A900A0002000641F02000000000026
:10491000D1C2A80010C2B3003EEDB700862002004D
:10492000000000007FC8BF003EEDB70086200200F7
:104930000000000030C1B3003EEDB7008620020049
:104940000000000000C2B3003EEDB7008620020068
:104950000000000090C0B3003EEDB70086200200CA
:1049600000000000562402000000000080C0B300D8
:104970003EEDB7008620020000000000C0C0B3007A
:104980003EEDB70086200200000000000000060097
:10499000851F7800C500200003000900B51F7800BE
:1049A000800378008404780004F0A1000400E00093
:1049B00006003A0009F0A7000200370005002000B9
:1049C0000F003700050020000D003700E6425200BE
:1049D0000A0039000003200009F0A60000022000B0
:1049E0003322AF00FEFF3700A01188008502E900E6
:1049F000FBFF3B00550020000100370084027800D7
:104A00006400200005E0A00009F0A70005F0A00068
:104A100008712200110009008883D8004225020095
:104A20000000000081037800883E2000110009008A
:104A30008883D8004225020000000000810378002E
:104A400048062000110009008883D8004225020092
:104A50000000000081037800A80020001100090078
:104A60008883D800422502000000000000032000D7
:104A700000C040003322AF00FEFF3700A0118800C5
:104A800017003700060320000000E0000E003A0087
:104A900005E0A6000D0037000402E9000524E1004E
:104AA000020032004200AF00000006000000E000FB
:104AB00005003A0005E0A6000400370005F0A60056
:104AC000060220000100370005E0A100004043007D
:104AD0003322AF00FEFF3700A0118800000006005F
:104AE0002501200003000900CF127800CF027800D2
:104AF00000000600D742A900D342A9000000000030
:104B000000000000047020009416880000000000DF
:104B10000000000000000600851F7800D222EF0090
:104B200004802000B416880000000000000000008F
:104B3000F43F200094168800D742A800D342A90071
:104B40000000000000000000E0C1B3003AEDB70033
:104B500010C0B3003BEDB700A6200200000000002B
:104B600005002000050078000A1302000000000084
:104B70000040B3004220AF00050037008502E80086
:104B800036EDB7002424020000000000F5FF3700D6
:104B9000C0C0B3003AEDB70020C0B3003BEDB70092
:104BA000A62002000000000005002000050078009B
:104BB0001A130200000000000040B3004220AF00C2
:104BC000050037008502E80036EDB7002424020016
:104BD00000000000F5FF370080C1B3003AEDB700D8
:104BE00030C0B3003BEDB700A6200200000000007B
:104BF00005002000050078003213020000000000CC
:104C00000040B3004220AF00050037008502E800F5
:104C100036EDB7002424020000000000F5FF370045
:104C200030C0B3003AEDB70050C0B3003BEDB70061
:104C3000A62002000000000005002000050078000A
:104C400046130200000000000040B3004220AF0005
:104C5000050037008502E80036EDB7002424020085
:104C600000000000F5FF3700D202A800D402AE0019
:104C700029003700F44380004822DE00F4CFB20060
:104C800025003200F44380004822DE0061424200E9
:104C9000044078007FE8B700800C2000641F020009
:104CA0000000000010C2B3003EEDB70086200200F5
:104CB000000000007FC8BF003EEDB7008620020064
:104CC00000000000010020000100780060130200D5
:104CD000000000008100E8003322AF00FEFF370033
:104CE000A0118800400020000008E600F6FF370011
:104CF0007FC8BF000160EF0004002000C82402004C
:104D0000000000003322AF00FEFF37000402200045
:104D1000A4118800D4FF3700D222A800D422AE000C
:104D200029003700F44380004822DE0003082000F9
:104D3000041CE10024003100F44380004822DE001E
:104D4000614052007FE8B700800C2000641F020021
:104D50000000000010C2B3003EEDB7008620020044
:104D6000000000007FC8BF003EEDB70086200200B3
:104D70000000000001002000010078006013020024
:104D8000000000008100E8003322AF00FEFF370082
:104D9000A0118800400020000008E600F6FF370060
:104DA0007FC8BF000160EF0004002000C82402009B
:104DB000000000003322AF00FEFF37000402200095
:104DC000A4118800D4FF37007A25020000000000FB
:104DD0007A24020000000000CF02780000000600E4
:104DE000306DEF002E2402000000000010C0B30060
:104DF00030EDB7002E2402000000000020C0B300F8
:104E000030EDB7002E2402000000000030C0B300D7
:104E100030EDB7002E2402000000000040C0B300B7
:104E200030EDB7002E2402000000000050C0B30097
:104E300030EDB7002E240200000000000000060044
:104E4000820020000200090000000000E8C2A90062
:104E5000E8C2A900030009000000000081C0D200E0
:104E6000E902A9004200AF00E902A8004200AE003A
:104E7000E902A900E8C2A800E6C2AE00FEFF3700C2
:104E80000201E900EFFF3A00020009000000000003
:104E9000E8C2A900E8C2A90000000000E902A800D9
:104EA00003000900000000000300090000000000EA
:104EB000E8C2A800E6C2AE00FEFF3700030009000A
:104EC0000000000000002000E702AF000000A0008A
:104ED000E8C2A900E8C2A900E902A900E902A90004
:104EE0000000060083002000E902A800030009007A
:104EF00000000000E8C2A800E6C2AE00FEFF3700D6
:104F0000E702AF004200A800E702AE004200A9009D
:104F10000281D2000200090000000000E8C2A900DE
:104F2000E8C2A9008301E900EFFF3A00E902A80006
:104F300003000900000000000100E0004220AE0074
:104F4000E902A90000000000E8C2A800E6C2AE0025
:104F5000FEFF37000200090000000000E8C2A900BF
:104F6000E8C2A9000300090000000000E902A9004E
:104F7000E902A9000200780000000600851F780001
:104F8000861F7800E902A90000000000E8C2A8001E
:104F9000E6C2AE00FEFF370002000900000000007C
:104FA0000100090000000000E902A8000200090059
:104FB00000000000E902A800020009000000000053
:104FC000E8C2A8000300090000000000E902A900EF
:104FD000E902A9000200090000000000E8C2A900DF
:104FE000E8C2A90005638000C72ADE006280620073
:104FF00000437800864AB3008640780020270200EC
:105000000000000001638000202702000000000073
:10501000E902A8000200090000000000E8C2A800A0
:105020000300090000000000E6C2AE00FEFF3700EA
:10503000E902A900E902A90002000900000000003D
:10504000E8C2A900E8C2A90005638000C72ADE0003
:105050006280620000437800964AB3008640780080
:10506000202702000000000001002000811F7800BE
:10507000CF00780072270200000000005FECB7004C
:10508000E902A90000000000E8C2A800E6C2AE00E4
:10509000FEFF3700020009000000000001000900C7
:1050A00000000000E902A800020009000000000062
:1050B0005FCCBF0000E0B7004F037800CF0278005C
:1050C0000000060082002000280009000000000007
:1050D000E2C2A900DEC2A900290009000000000008
:1050E00081C0D200D722A9004200AF00D322A8007D
:1050F0004200AE00D322A900DEC2A800E0C2AE008A
:10510000FEFF37000201E900EFFF3A002800090026
:1051100000000000E2C2A900DEC2A90000000000F9
:10512000D322A8002900090000000000290009007E
:1051300000000000DEC2A800E0C2AE00FEFF3700A3
:10514000290009000000000000002000D522AF0067
:105150000000A000E2C2A900DEC2A900D722A90077
:10516000D322A90000000600851F7800D322A800E2
:105170002800090000000000DEC2A8002900090084
:1051800000000000D722A900D322A90028000900AE
:1051900000000000E2C2A900DEC2A90021CCB300D9
:1051A00062280200000000006104E10003003A00F0
:1051B00010C0B30000E0B7001E003700E1688000B7
:1051C00062280200000000006104E10003003A00D0
:1051D00020C0B30000E0B700160037001DCDBF00AF
:1051E0008000780062280200000000006104E100F5
:1051F00003003A0030C0B30000E0B7000D003700F4
:10520000D322A90000000000DEC2A800E0C2AE0068
:10521000FEFF37002800090000000000010009001F
:1052200000000000D322A8002800090000000000B0
:105230000060EF00CF02780000000600830020002D
:10524000D322A8002900090000000000DEC2A80047
:10525000E0C2AE00FEFF3700D522AF004200A8003A
:10526000D522AE004200A9000281D2002800090028
:1052700000000000DEC2A900E2C2A9008301E9002B
:10528000EFFF3A00D322A800290009000000000027
:10529000D722A9000100E0004220AE00D322A900DD
:1052A00000000000DEC2A800E0C2AE00FEFF370032
:1052B0002800090000000000E2C2A900DEC2A90027
:1052C0002900090000000000D722A900D322A9006C
:1052D0000200780000000600851F7800136CEF00C4
:1052E000206CEF00216CEF00226CEF00236CEF00CC
:1052F000246CEF00256CEF00D322A80028000900E1
:1053000000000000DEC2A800290009000000000023
:10531000D722A900D322A90028000900000000001C
:10532000E2C2A900DEC2A90031CCB30062280200AB
:10533000000000006104E10010003A0005002000B8
:1053400005007800C6150200000000000040B30010
:105350004220AF00060037008502E8003322AF008C
:10536000FEFF370034E2B7003562EF00F4FF37008C
:1053700010C0B30000E0B700BA00370011002000F1
:10538000811F7800CF0078001E2902000000000075
:1053900013ECB70011002000811F7800CF007800C7
:1053A0001E2902000000000020ECB70011002000C0
:1053B000811F7800CF0078001E2902000000000045
:1053C00021ECB70011002000811F7800CF00780089
:1053D0001E2902000000000022ECB700110020008E
:1053E000811F7800CF0078001E2902000000000015
:1053F00023ECB70011002000811F7800CF00780057
:105400001E2902000000000024ECB700010020006B
:10541000811F7800CF0078001E29020000000000E4
:1054200025ECB700D322A90000000000DEC2A800CE
:10543000E0C2AE00FEFF37002800090000000000B7
:105440000100090000000000D322A8002800090084
:10545000000000000608A900224CAF000608A800C2
:1054600022CCBF006340600028ECB7008549A9004A
:1054700024ECAF008549A8008042EB000608AF008D
:105480008502E8000100200001007800DA15020022
:10549000000000008100E8003322AF00FEFF37006B
:1054A000A0118800500020000008E600F6FF370039
:1054B000054078000160EF0004002000C8240200CD
:1054C000000000003322AF00FEFF3700A4022000DE
:1054D000A41188003322AF00FEFF37000402200031
:1054E000A41188000100200001007800F2150200DC
:1054F000000000008100E8003322AF00FEFF37000B
:10550000A0118800400020000008E600F6FF3700E8
:1055100028CCBF000160EF0004002000C824020076
:10552000000000003322AF00FEFF3700A40220007D
:10553000A41188003322AF00FEFF370004022000D0
:10554000A411880013CCBF000160EF00040020000C
:10555000C8240200000000003322AF00FEFF370025
:1055600004022000A411880020CCBF000160EF00DD
:1055700004002000C8240200000000003322AF0015
:10558000FEFF370004022000A411880021CCBF00D8
:105590000160EF0004002000C824020000000000A9
:1055A0003322AF00FEFF370004022000A411880060
:1055B00022CCBF000160EF0004002000C8240200DC
:1055C000000000003322AF00FEFF3700040220007D
:1055D000A411880023CCBF000160EF00040020006C
:1055E000C8240200000000003322AF00FEFF370095
:1055F00004022000A411880024CCBF000160EF0049
:1056000004002000C8240200000000003322AF0084
:10561000FEFF370004022000A411880025CCBF0043
:105620000160EF0004002000C82402000000000018
:105630003322AF00FEFF370004022000A4118800CF
:105640003322AF00FEFF3700A4002000A411880021
:105650003322AF00FEFF3700D4002000A4118800E1
:105660000060EF00CF02780000000600851F780080
:10567000861F7800E902A80002000900000000006F
:10568000E8C2A8000300090000000000E902A90028
:10569000E902A9000200090000000000E8C2A90018
:1056A000E8C2A900E5688000C72ADE0062806200C7
:1056B00000437800864AB300864078002027020025
:1056C000000000001F0DA9000000AF001F0DA80082
:1056D000E168800020270200000000001F0DA900E3
:1056E0000000AF001F0DA800F16880002027020015
:1056F000000000001F0DA9000000AF001F0DA80052
:10570000E902A90000000000E8C2A800E6C2AE005D
:10571000FEFF370002000900000000000100090040
:1057200000000000E902A8000200090000000000DB
:105730004F037800CF02780000000600861F780033
:10574000871F7800881F7800891F78000002EB000F
:105750008002EB000003EB008003EB000304690010
:1057600011003200080220004200A9000080D2008F
:105770008180D2000482D2008582D2000328E10019
:1057800001003A0002A0E1000300390002025200C9
:1057900083825A004200A8000683D2008783D20089
:1057A0000804E900F0FF3A0087007800060078005E
:1057B000CF0478004F047800CF0378004F037800BF
:1057C00000000600851F7800C500200003000900C6
:1057D000B51F780000037800810378000406780084
:1057E00004F0A1000400E00006003A0009F0A70060
:1057F00002003700050020001300370005002000DC
:1058000011003700EB4252000E0039000003200067
:1058100009F0A6000002200036EDB70024240200A3
:105820000000000041E0AF00FBFF3700801088005F
:105830001162EF008502E900F7FF3B0055002000F0
:105840000100370084027800E800200009002000F1
:105850001000FA000C377C000884E900FDFF3B00D3
:10586000A400200005E0A0000CF0A70005F0A000B7
:10587000040F78001507980006007800870078006C
:1058800002A02C00A3B92300087122000DF0A10092
:105890000DF0A2009E2B0200000000000DF0A700FA
:1058A0000700370040079800510798000001780072
:1058B000810178002E009000BE009000F4FF3700B8
:1058C000420798005307980024079800350798006E
:1058D0001E0278009E029000060320000000E000F7
:1058E00012003A0005E0A600120037000402E900A9
:1058F000040F78000400E0000E0032000524E100EF
:10590000020032004200AF000E0037000603200004
:105910000000E00005003A0005E0A60005003700A1
:1059200005F0A600060220000200370005E0A100F5
:10593000150798000040430036EDB700242402000C
:10594000000000004E009000DE009000A200200049
:105950008001EB006100E10001003200CCFF370064
:105960000080FA002501200003000900CF12780012
:10597000CF02780000000600851F7800861F78009F
:105980005624020000000000A0C0B3003AEDB700AA
:1059900050C0B3003BEDB700A6200200000000009D
:1059A0000500200005007800B2170200000000008A
:1059B0000040B3004220AF00050037008502E80038
:1059C00036EDB7002424020000000000F5FF370088
:1059D0000500200005007800CC1702000000000040
:1059E0000040B3004220AF00060037008502E80007
:1059F0003322AF00FEFF370034E2B7003562EF001C
:105A0000F4FF3700803E2000641F02000000000009
:105A1000F0C0B30052ECB700524CE200110032006B
:105A2000956280000548B30080C2B3001CEDB7004A
:105A3000054078001DEDB700B4280200000000000A
:105A40006C290200000000008549AF000300370008
:105A500052CCBF0029ECB70002003700526CED00B9
:105A6000EDFF370029CCBF00EF42600080C2B300D9
:105A70001CEDB700054078001DEDB700B42802000A
:105A80000000000029CCBF001EEDB700E41F20007D
:105A9000E4688800362B02000000000001002000AE
:105AA00001007800E8170200000000008100E80013
:105AB0003322AF00FEFF3700A011880060002000F5
:105AC0000008E600F6FF370029CCBF000160EF00B8
:105AD00034002000C8240200000000003322AF0080
:105AE000FEFF370004022000A41188003322AF001B
:105AF000FEFF370004022000A411880050C0B3004C
:105B000030EDB7002E24020000000000A0C0B3005A
:105B10003AEDB70050C0B3003BEDB700A62002003D
:105B200000000000050020000500780002180200B7
:105B3000000000000040B3004220AF000500370025
:105B40008502E80036EDB7002424020000000000C2
:105B5000F5FF370029CCBF00800278000B60EF0012
:105B60000600200005007800860078003400200040
:105B7000E22B020000000000007D2000641F0200F4
:105B80000000000050C0B30030EDB7002E2402002A
:105B9000000000004F037800CF02780000000600EC
:105BA000851F7800C500200004000900B51F78009B
:105BB00000027800810278008303780002037800F5
:105BC0004200A9004220A9008180D2000180FD008E
:105BD000F10FB2000100E000480032004200A900CD
:105BE0004220A9008381D2000380FD00F30FB200A0
:105BF0000300E000410032000080FB0001C04100D2
:105C000004003100F007B1003C0032003B003900D5
:105C1000020037001048B0003800310007856A00E4
:105C20004200A9004220A900F50FB2000570A000B3
:105C30004220EF00F70FB2000770A0000621B80065
:105C4000062CB80083014C0089007800043CB800A1
:105C500083014C0081804C00072CB80081004C006F
:105C60000000E8000100E0004220AF000100370022
:105C7000030037000300E0004220AF0005003700BA
:105C800001F0A700030037008381D2008180D20099
:105C90000000E900010178004200A9000370A6009D
:105CA0000900370007F02F00878161000310B00062
:105CB000600149000200E00003003A000300E00038
:105CC00001003A000000E8000080FD004200A90049
:105CD0004220A9008080D3000AF0A70001F0A000B4
:105CE00002F0A1000280FD00814069000380FD00F8
:105CF0000341780002007800030037000000200014
:105D000001002000000037004501200004000900C8
:105D1000CF127800CF02780000000600851F7800BF
:105D2000861F7800871F78000382680004F0A600B1
:105D3000060037004200A9004220A90001F0A60099
:105D4000260037004200A800240037000102780036
:105D50008002780003037800820378008180D200FB
:105D60000180FD008381D2000380FD0081C05100CD
:105D70000500320004F0A6001800370010002000D3
:105D800042C0B60015003700844078008641780094
:105D90000170A1000370A10081C051000500320014
:105DA00004F0A6000D0037001000200042E0B6000D
:105DB0000A003700858053000500320004F0A60079
:105DC000060037001000200042E0B6000300370054
:105DD0004200A9000100370000003700CF0378001F
:105DE0004F037800CF02780000000600851F78007E
:105DF000C500200003000900B51F78008004EB00F7
:105E0000080028004300AF0083016C000105780002
:105E10008A8569000103780083037800030678000F
:105E20004220A9004200A9000683D2000680FD009E
:105E3000F60FB2000600E000960032004220A900F2
:105E40004200A9008783D2000780FD00F70FB2004F
:105E50000700E000940032004220A9004200A9009F
:105E60000638E10091003200980033000900A100DB
:105E70000910A0000684530007037800F10FB20058
:105E80000170A000F30FB2000370A0008702200091
:105E90000838E100110033004220A9004200A900A7
:105EA0008180D3000080D3000804E900FAFF3A00A3
:105EB0000D003700870220000838E1000900330098
:105EC0004220A9004200A9008381D3000281D300AF
:105ED0000804E900FAFF3A000F00370002007800DA
:105EE00083007800430037000BF0A6001100370054
:105EF0000940A7008C0578000000EA00020032008B
:105F000081C0EA00010037008100EA000940A700D3
:105F10002B003700070037000BF0A6000500370004
:105F20000201EA000200320083C1EA0001003700EA
:105F30008301EA00F50FB2004220A9004200A90047
:105F40000200400083C048004200AF000930A000BA
:105F50000900A700090037000910A7000100370059
:105F60000B0037000BF0A700150037000930A70021
:105F7000290037000960A0001E0037000BF0A700C1
:105F80000F0037000930A700230037001900370041
:105F90000920A1000BF0A700040037008A05780053
:105FA0000930A7001C0037002B0037000940A00073
:105FB00001C8B2000170A700CDFF37008A05780044
:105FC000F10FB200810370000A0032000170A700D7
:105FD000080037004220A9004200A9000080D2003A
:105FE0008180D2000603E9004220AF00260037007E
:105FF000F6FF37000900A7008A0578000910A700FE
:106000008C0578000950A6000F0037000AF0A700A1
:106010000080A000100037004200A80081C0D3001B
:106020000080D3004200AF000950A0000603E80042
:106030000900A7008A0578000910A7008C057800E0
:106040004220AF00100037000960A7008A057800E1
:106050000970A7008C057800010170002300320050
:106060000170A1000680FD004220A9004200A900A5
:106070000683D30081006B0001F0A0000BF0A600A6
:1060800001F0A100190037000000200001002000ED
:10609000160037000AF0A70083016C0002007800A8
:1060A000830078001100370010003700F30FB200B2
:1060B0000370A000F10FB2000170A0000BF0A70068
:1060C0000370A1000920A00093FF370007045300CC
:1060D000F10FB2000170A000F30FB2000370A00036
:1060E0000910A1000900A00072FF3700250120005F
:1060F00003000900CF127800CF02780000000600EC
:10610000851F7800C500200004000900B51F780035
:106110008004EB008384680001037800800278002B
:1061200003047800820378008180D2000180FD00A2
:106130008180FB000100E0004E0032008381D2002C
:106140000380FD008381FB000300E0004900320072
:106150000000EB0003C0500003003900F047B0001E
:1061600044003100030037001048B10041003900FD
:106170004000320085007800060178000270A0001F
:10618000F20FB200F80FB2000870A0009A012000D0
:106190008001EB000002EB008780500008015900ED
:1061A000020033000400310004003A008780400000
:1061B00008014900010037000400A0000A05E900B9
:1061C000070032004200A9008180D2000281D20083
:1061D0004200A9000482D2008381D200EEFF370082
:1061E0000005EB000380A700010037000600370020
:1061F0004200A9008381D3000370A1000482D30070
:106200000A85D200020037000000E90019003200C0
:106210000AF0A700050039008180D2000281D20077
:106220008780500008015900090039000402E80085
:1062300007003A008301E80005003A000000E8008A
:106240000C003200020037000000E90009003200B3
:106250000080FD008080D30001F0A00009F0A600BE
:1062600001F0A1000370A10081C069000400780062
:10627000030037000000200001002000000037006C
:106280004501200004000900CF127800CF027800F9
:1062900000000600000178008101780001407800CC
:1062A0000080FD0000F0A0008180D2000180FD0090
:1062B0008180FB00E408200081405200060032008B
:1062C0000000E000040032004200A9000080D3007A
:1062D0008100E900FAFF3A0003F0A600020037004F
:1062E0000000EA000000370000000600851F78006B
:1062F000E0CFB30031EDB70000C6B30036EDB70014
:10630000C0C0B30037EDB700304DE20003003A00E3
:1063100000C2B30038EDB700230037008469800065
:106320006124E10003003A00C0CEB30038EDB700AD
:106330001D003700846980006224E10003003A00F8
:10634000C0CEB30038EDB700170037008469800075
:106350006324E10003003A0000CDB30038EDB7003C
:1063600011003700846980006424E10003003A00D2
:1063700000CBB30038EDB7000B0037008469800014
:106380006524E10003003A0000C9B30038EDB7000E
:1063900005003700846980006624E10002003A00AD
:1063A00000C7B30038EDB70032CDBF0035EDB70000
:1063B00033CDBF0034EDB700D322A8002800090078
:1063C00000000000DEC2A800290009000000000053
:1063D000D722A900D322A90028000900000000004C
:1063E000E2C2A900DEC2A90021CCB30062280200EB
:1063F000000000006104E10003003A0040C0B30067
:1064000000E0B7004800370001C2B3006228020074
:10641000000000006104E10003003A0050C0B30036
:1064200000E0B7004000370031CDBF0080007800A9
:1064300062280200000000006104E10003003A004D
:1064400060C0B30000E0B70037003700A1698000EA
:1064500062280200000000006104E10003003A002D
:1064600070C0B30000E0B7002F00370035CDBF008B
:106470008000780062280200000000006104E10052
:1064800003003A0080C0B30000E0B70026003700E8
:10649000B169800062280200000000006104E10090
:1064A00003003A0090C0B30000E0B7001E003700C0
:1064B00037CDBF0080007800622802000000000095
:1064C0006104E10003003A00A0C0B30000E0B7009F
:1064D00015003700C169800062280200000000003A
:1064E0006104E10003003A00B0C0B30000E0B7006F
:1064F0000D003700D322A90000000000DEC2A80072
:10650000E0C2AE00FEFF37002800090000000000D6
:106510000100090000000000D322A80028000900A3
:10652000000000000060EF00CF02780000000600CD
:10653000E70160004300DE00010040000000A7000A
:10654000E88141000000A1000204E0001098AD00C5
:1065500000000600851F78006229EF007069EF00D7
:10656000DE42A800E042AE000300370010C0B300D6
:1065700000E0B700460037001200090000000000EC
:10658000F0C0B30031EDB700846980004822DE001E
:10659000F4CFB20012003200E262A900DE62A9006C
:1065A0001200090000000000E262A800DE62A900FB
:1065B000DE42A800E042AE00050037002196200030
:1065C00031CDBF000160EF004220A9001180AD0075
:1065D0001200090000000000316DED00EAFF3700F5
:1065E000E262A900DE62A9001200090000000000BA
:1065F000E262A800DE62A9001200090000000000AB
:1066000020C0B30031EDB700846980004822DE006D
:10661000F4CFB20015003200E262A900DE62A900E8
:106620001200090000000000DE42A800E042AE00B7
:10663000080037000197200031CDBF000160EF0056
:1066400012002000821F78004F017800983202006B
:1066500000000000E262A800DE62A900120009004A
:1066600000000000316DED00E7FF3700E262A90095
:10667000DE62A9001200090000000000E262A8002A
:10668000DE62A90012000900000000000060EF00B7
:10669000CF02780000000600851F7800861F780072
:1066A0007229EF007429EF00AA32020000000000F6
:1066B0006104E10001003A00FBFF37006809F800BF
:1066C0006A09F9006829EF00104B80006829B700BB
:1066D000F44A80004822DE00704242000440780004
:1066E0005FE9B700F44A80004822DE007924E10027
:1066F00033003C00AA320200000000006104E10007
:1067000001003A00FBFF3700104B80006C29B700F6
:10671000F44A80004822DE007042420004407800C3
:106720005FE9B700F44A80004822DE007040520062
:1067300030EDB700846980007A24E100090032005E
:106740006829D4006AA9D6006DE9AE0001003700BF
:106750006809A8006C29D4006EA9D600306DEC0041
:10676000F4FF3700F44A80004822DE007A405200ED
:106770005FE9B7006809F8007209F900544B80001E
:10678000F43FB200A44B8800306DEF0030CDBF0065
:106790005F49E300090032006829D4006AA9D600E5
:1067A0006DE9AE00010037006809A8006C29D4002B
:1067B0006EA9D600306DEC00F4FF370013003700EF
:1067C000F44A80004822DE007A4052005FE9B700B8
:1067D000F44A80004822DE000960EF00454B80004B
:1067E000564B80000402E8000402E9000300320076
:1067F0000603D1008582D300FBFF3700954B88004C
:1068000006027800F43FB200A44B88004F037800E2
:10681000CF02780000000600670160004300DE0040
:1068200001004000104078000010A5000000EB00BF
:106830004200AF000000E80000000600316DEF00EC
:106840008509A9008229EF0090C1B30030EDB7009F
:1068500084698000F4CFB20012003200219720003A
:1068600030CDBF000160EF000C34020000000000DA
:106870000000A3000800390031CDBF000160EF0027
:106880004100DD0004BD200004004000100078003D
:106890008289B600104C8800316DEC00306DED003F
:1068A000EBFF3700144C8000F43FB200144C88001A
:1068B000104C8000040CE30005003A008509A80094
:1068C00010C6B30084E9B700200037001F0037006E
:1068D000104C8000060CE30005003A008509A80072
:1068E00020C6B30084E9B70018003700170037004E
:1068F000104C8000080CE30005003A008509A80050
:1069000030C6B30084E9B700100037000F0037002D
:10691000104C80000A0CE30005003A008509A8002D
:1069200030C4B30084E9B70008003700070037001F
:10693000104C80000C0CE30004003A008509A8000C
:1069400040C6B30084E9B70000003700000006002D
:10695000E262A800DE62A9005F69EF008169EF00D2
:106960009E2BEF0000C3B30084E9B7008509A9009E
:106970007229EF007429EF007169EF00AA3202005A
:10698000000000004C330200000000001E34020032
:10699000000000008F69EF008D69EF008E69EF0045
:1069A00002002000419920000200780092130200AA
:1069B00000000000805878000201E8000004E000B8
:1069C0004220AE00F8FF3700C76BEF008629EF00CA
:1069D00002002000E199200002007800A8130200C4
:1069E00000000000805878000201E8000004E00088
:1069F0004220AE00F8FF37000200200021AA20004C
:106A000002007800E01302000000000080587800C7
:106A10000201E8000004E0004220AE00F8FF370069
:106A200002002000E1AD200002007800E013020027
:106A300000000000805878000201E8000004E00037
:106A40004220AE00F8FF370002002000A1B1200074
:106A500002007800E0130200000000008058780077
:106A60000201E8000004E0004220AE00F8FF370019
:106A70000200200061B5200002007800E01302004F
:106A800000000000805878000201E8000004E000E7
:106A90004220AE00F8FF37000200200001A22000D3
:106AA00002007800A813020000000000805878005F
:106AB0000201E8000004E0004220AE00F8FF3700C9
:106AC0000200200001AC200002007800E013020068
:106AD00000000000805878000201E8000004E00097
:106AE0004220AE00F8FF370002002000C1AF2000B6
:106AF00002007800E01302000000000080587800D7
:106B00000201E8000004E0004220AE00F8FF370078
:106B10000200200081B3200002007800E013020090
:106B200000000000805878000201E8000004E00046
:106B30004220AE00F8FF37000200200041B72000DD
:106B400002007800E0130200000000008058780086
:106B50000201E8000004E0004220AE00F8FF370028
:106B60008069EF00982BEF009A2BEF00922BEF003B
:106B7000942BEF0000000600851F7800820178004A
:106B8000820278004200A9008381D2000380FD00C8
:106B9000F30FB2000338B000F207B2003600200055
:106BA0000002EB004200A9000281D3008180D300E3
:106BB0000080D3004200AF000402E8000603E900B1
:106BC000F8FF3A000270A100C419DD0003F0A10033
:106BD00005F0A70003F0A00083016900010178001F
:106BE0008000780004007800CF02780000000600E2
:106BF000881F78002801200004000900B81F7800D1
:106C00008005EB006066B800030478008704780014
:106C1000FA7F20004200A9004220A90044C4DE00FF
:106C2000080465000800E000700032004200A9007E
:106C30004220A900C4CCDE00890465000900E00000
:106C40006A0032000884440009B0A700040037003D
:106C5000F83FB100650032006400390003003700DE
:106C60001A40200085424500600031008786690097
:106C70004200A9004220A900F300B2000340A00096
:106C8000F700B2000740A000881F78000124B80078
:106C9000002DB8000A0544008B854C000C80B00024
:106CA0000224B8008B0544000C864C00012CB8006F
:106CB0008B0544000C864C000034B8000005EB0046
:106CC0008B0544000C864C000A80B0008005EB0068
:106CD0000324B8000C0644000A854C000B80B00069
:106CE000022CB8000C0644000A854C000B80B00052
:106CF0000134B8000C0644000A854C000B80B0003B
:106D0000003CB8000C0644000A854C000B80B00023
:106D10000C0078000006EB00032CB8000A054400C4
:106D20008B854C000C80B0000234B8000A0544008A
:106D30008B854C000C80B0000334B8008B054400F8
:106D40000C864C00013CB8000A0544008B854C00C1
:106D50000C80B000023CB8008B0544000C864C004F
:106D6000033CB8000C0644008A0078000B01780050
:106D70008C017800540020004200A9008381D300D8
:106D80000281D3008180D3000080D3000402E90097
:106D9000F9FF3A004F0478000804E800010370008E
:106DA00001003200020037000303710008003200C6
:106DB0000340A700060037004200A9000080D2006F
:106DC0008180D2000281D2008381D2000804E900D0
:106DD0004444DD0003F0A1000DF0A70003F0A00083
:106DE0000340A10083016C00030037006000B8007D
:106DF0006001B80000003700A8012000040009006D
:106E00004F1478004F04780000000600881F7800B7
:106E1000891F78008A1F78008784690009F0A6001E
:106E2000060037004200A9004220A90003F0A60096
:106E3000340037004200A80032003700FA7F2000FB
:106E4000030478008704780044C4DE000804650069
:106E5000C4CCDE00890465000885540005003200BA
:106E600003F0A600270037001000200042E0B60023
:106E7000240037000304780087047800F301B2008F
:106E8000F701B2000340A1000740A10003C5530071
:106E90000500320008F0A6001A003700100020009C
:106EA00042E0B6001700370002055300050032002B
:106EB00008F0A600130037001000200042E0B600E2
:106EC00010003700018552000500320008F0A600CE
:106ED0000C0037001000200042E0B6000900370027
:106EE000000552000500320008F0A600050037003A
:106EF0001000200042E0B600020037004200A90066
:106F0000000037004F057800CF0478004F04780068
:106F100000000600851F7800C5002000050009005C
:106F2000B51F78000304780082037800010378001D
:106F300080027800830478003B472000C499DE007B
:106F4000FA7F20008301650083855500F801B200B7
:106F50000840A0000000EB008000EB000001EB0007
:106F60008001EB004200A9000884D3008783D3008E
:106F70000683D3008582D3008381D3000281D300AE
:106F80008180D3000080D3008B05E900F5FF3A0033
:106F900009F0A600050037000000EA008180EA0041
:106FA0000281EA008381EA000000370065012000C9
:106FB00005000900CF127800CF027800000006001B
:106FC0008C1F78008D1F78000004EB008004EB001C
:106FD0000005EB008005EB000006EB008006EB00EF
:106FE000E8002000090020001000FA000C377C00A7
:106FF0000884E900FDFF3B0005046A0002003A0036
:1070000007046B002F0032000004EB000D04200089
:107010000D0420004200A9000080D2008180D2002F
:107020000281D2008381D2000884D2008984D200F8
:107030000A85D2008B85D2000758E10005003A008E
:1070400006D0E10003003A0005C8E10001003A0063
:1070500004C0E100050039000404540085845C008C
:1070600006055D0087855D004200A800080F7800D6
:10707000190798002A0798003B0798004E049000D3
:10708000DE0490006E059000FE0590000884D2009A
:107090008984D2000A85D2008B85D20048079800E7
:1070A000590798006A0798007B0798001E0478002B
:1070B0009E0490002E059000BE0590008D06E9000C
:1070C000D4FF3A004E009000DE0090006E01900068
:1070D000FE0190000080FA0000003700CF06780023
:1070E0004F06780000000600851F7800C5002000CC
:1070F00007000900B51F78000900E0001300320006
:107100002800FA00680220000006EB000C377C0023
:107110000884E900FDFF3B0039179800470224006E
:107120000003EB006022B8002917980047022400F2
:107130000003EB006022B800F835020000000000F8
:10714000AE1490008904E900F7FF3A00D71C240030
:1071500056D62C006022B800000F9800110F98003E
:10716000220F9800330F980003F0A10006370200A9
:10717000000000004200AE000E0037000E08900034
:107180009E0890002E099000BE099000A8002000E3
:1071900008179800A5B9230004A02C006033B8009C
:1071A000440F9800550F9800660F9800770F9800CD
:1071B0000E0037000E0890009E0890002E099000E7
:1071C000BE09900048012000081798000400200024
:1071D000859E28004630220077AC2800440F980096
:1071E000550F9800660F9800770F980000057800FB
:1071F00003F0A7004D0037000A00780003F0A1005B
:107200008A370200000000009E1490008004EB000A
:10721000191798004E0A9000DE0A90006E0B90003D
:10722000FE0B90009E169000E03702000000000068
:107230009E1690000D00A7002C003700080F980044
:10724000190F98002A0F9800310F98009E16900091
:107250000D00A2001D1798009E1690000D10A700AB
:10726000060037009E1690000000E0001300320078
:107270009E1690000D10A0001D1798000E12900091
:10728000BE169000800278000D20E10005003A0053
:107290003D1798003322AF00FEFF3700E4022000C4
:1072A000A41188003D179800050078000003B00085
:1072B0003322AF00FEFF3700A01188008E16900029
:1072C0008D06E9001E0032000D1798004E08900050
:1072D000DE0890006E099000FE099000A4002000D6
:1072E0008002EB006033B800CEFF3700400F9800FB
:1072F000510F9800620F9800730F980000027800F9
:107300008102780002037800830378000E08900061
:107310009E0890002E099000BE0990009E169000D5
:107320000D00A2001D179800BEFF37003322AF00EA
:10733000FEFF3700D4022000A4118800AFFF370001
:10734000000000000080FA00A501200007000900ED
:10735000CF127800CF02780000000600851F780069
:10736000861F7800C46980004822DE0003032000E5
:10737000041CE100020036007100370006003700EF
:10738000C46980004822DE0093032000041CE10051
:10739000010031006A0037006009E20003003A0092
:1073A00014002000044B880017003700044B8000B5
:1073B0006120E10003003A0064012000044B8800D2
:1073C00011003700044B80007620E10003003A00F2
:1073D000B4022000044B88000B003700044B8000EF
:1073E000B482B20003003A0004042000044B880079
:1073F00005003700044B80000484B20002003A000C
:1074000014002000044B88004369EF00144A8000F8
:107410004822DE0033032000041CE100480036004F
:10742000C46980004822DE0043032000041CE10000
:107430000E003900C46980004822DE000443B10018
:107440000440780000E0B700340320000400B800D6
:10745000144A80004822DE0004404000021002006E
:107460000000000044E9B70012003700C469800042
:107470004822DE0053032000041CE1000D003E0002
:10748000C46980004822DE005443B1000440780003
:1074900000E0B700340320000400B800144A800064
:1074A0004822DE0004404000CA1002000000000034
:1074B00044E9B7004349E20006003A0060C9BF0052
:1074C0003AEDB7003B6DEF00A6200200000000007F
:1074D00015003700144A80004822DE007124E100C4
:1074E00007003A0060C9BF003AEDB70010C0B30012
:1074F0003BEDB700A6200200000000000A003700A4
:10750000144A80004822DE0024C2B20006003A007D
:1075100060C9BF003AEDB70020C0B3003BEDB70033
:10752000A62002000000000044C9BF003AEDB700E9
:10753000CC200200000000004369EC00B3FF3700DC
:107540004F037800CF02780000000600851F780006
:10755000C500200007000900B51F78000900E00001
:10756000130032002800FA00680220000006EB0039
:107570000C377C000884E900FDFF3B0039179800B8
:10758000470224000003EB006022B800291798008E
:10759000470224000003EB006022B800F835020027
:1075A00000000000AE1490008904E900F7FF3A00E3
:1075B000D71C240056D62C006022B800000F98007B
:1075C000110F9800220F9800330F980003F0A100CC
:1075D00006370200000000004200AE000E00370037
:1075E0000E0890009E0890002E099000BE099000A1
:1075F000A800200008179800A5B9230004A02C00BB
:107600006033B800440F9800550F9800660F98003B
:10761000770F98000E0037000E0890009E0890002B
:107620002E099000BE09900048012000081798001C
:1076300004002000859E28004630220077AC2800F8
:10764000440F9800550F9800660F9800770F980028
:107650000005780003F0A7004D0037000A0078000D
:1076600003F0A1008A370200000000009E14900081
:107670008004EB00191798004E0A9000DE0A900073
:107680006E0B9000FE0B90009E169000E0370200FB
:10769000000000009E1690000D00A7002C0037008F
:1076A000080F9800190F98002A0F9800310F9800C2
:1076B0009E1690000D00A2001D1798009E169000C7
:1076C0000D10A700060037009E1690000000E00095
:1076D000130032009E1690000D10A0001D17980098
:1076E0000E129000BE169000800278000D20E1007E
:1076F00005003A003D179800E0C2B30039EDB7002D
:10770000AE390200000000003D1798000500780027
:107710000003B00039EDB700AE39020000000000F0
:107720008E1690008D06E9001E0032000D1798009D
:107730004E089000DE0890006E099000FE0990004F
:10774000A40020008002EB006033B800CEFF3700B9
:10775000400F9800510F9800620F9800730F980027
:107760000002780081027800020378008303780029
:107770000E0890009E0890002E099000BE0990000F
:107780009E1690000D00A2001D179800BEFF370046
:10779000D0C2B30039EDB700AE39020000000000DE
:1077A000AFFF3700000000000080FA00A5012000B4
:1077B00007000900CF127800CF0278000000060011
:1077C000851F7800861F7800846980006124E100AD
:1077D00001003A000900370034618000449FB20084
:1077E00005003200262CEC0010C0B30000E0B7000A
:1077F0007600370001003700262CEF00D322A800C6
:107800002800090000000000DEC2A80029000900CD
:1078100000000000D722A900D322A90028000900F7
:1078200000000000E2C2A900DEC2A90031CCB30012
:1078300062280200000000006104E10003003A0039
:1078400010C0B30000E0B700600037001100200056
:10785000811F7800CF0078001E2902000000000080
:1078600013ECB70011002000811F7800CF007800D2
:107870001E2902000000000020ECB70011002000CB
:10788000811F7800CF0078001E2902000000000050
:1078900021ECB70001002000811F7800CF007800A4
:1078A0001E2902000000000022ECB700D322A9002C
:1078B00000000000DEC2A800E0C2AE00FEFF3700FC
:1078C000280009000000000001000900000000007D
:1078D000D322A80028000900000000000608A90023
:1078E000224CAF000608A80020CCBF002DECB7004A
:1078F00001002000010078000816020000000000CE
:107900008100E8003322AF00FEFF3700A01188009D
:10791000600020000008E600F6FF37002DCCBF0015
:107920000160EF0034002800C824020000000000BD
:107930003322AF00FEFF3700A4002000A41188000E
:107940003322AF00FEFF3700D4002000A4118800CE
:10795000C0C3B3003AEDB70040C0B3003BEDB70081
:10796000A6200200000000002D4CE2000D003A00AD
:10797000050020000500780022160200000000002B
:107980000040B3004220AF00050037008502E80048
:1079900036EDB7002424020000000000F5FF370098
:1079A000090037002DCCBF00800278000B60EF008B
:1079B00006002000050078008600780034002000D2
:1079C000E22B0200000000000060EF004F0378008F
:1079D000CF02780000000600851F7800861F78001F
:1079E000871F7800881F7800214DE2003A003A0096
:1079F0001069800021698000024022004397240022
:107A0000D02D0200000000006069880071698800C4
:107A1000106980002169800062662E00E32A24003C
:107A20008E2E020000000000090031000800320024
:107A3000A0992100812D2400126980002369800013
:107A40008E2E0200000000000100310003003A0009
:107A500010C0B30000E0B7007C0637004300A90067
:107A60006069800071698000024E240033B22400F6
:107A7000F62E02000000000080027800010378006A
:107A80000500780086007800020020000300240032
:107A9000D02D02000000000080037800010478006F
:107AA000070078008800780002002500337C24005D
:107AB00080300200000000003069880041698800C1
:107AC00030698000416980004A31020000000000F6
:107AD0005069880039013700046980004822DE00BF
:107AE0006124E10004003200046980004822DE00C5
:107AF0006224E1003A003A001069800021698000A8
:107B000002002000A3472400D02D02000000000046
:107B100060698800716988001069800021698000AF
:107B200002002000F33024008E2E0200000000002E
:107B3000090031000800320000002E00514D2400E1
:107B400012698000236980008E2E02000000000070
:107B50000100310003003A0010C0B30000E0B7009C
:107B60003A0637004300A90060698000716980000F
:107B7000024E240033B22400F62E02000000000062
:107B80008002780001037800050078008600780004
:107B900002002000031A2400D02D02000000000083
:107BA00080037800010478000700780088007800DE
:107BB00002002400C369240080300200000000009D
:107BC000306988004169880030698000416980001F
:107BD0004A3102000000000050698800F7003700B9
:107BE000046980004822DE006324E1003A003A0084
:107BF000106980002169800002002000A347240052
:107C0000D02D0200000000006069880071698800C2
:107C1000106980002169800002002B00F3502400CD
:107C20008E2E020000000000090031000800320022
:107C300000802600F1592400126980002369800029
:107C40008E2E0200000000000100310003003A0007
:107C500010C0B30000E0B700FC0537004300A900E6
:107C60006069800071698000024E240033B22400F4
:107C7000F62E020000000000800278000103780068
:107C80000500780086007800020020000318240018
:107C9000D02D02000000000080037800010478006D
:107CA000070078008800780002002400C3612400E7
:107CB00080300200000000003069880041698800BF
:107CC00030698000416980004A31020000000000F4
:107CD00050698800B9003700046980004822DE003E
:107CE0006424E1003A003A001069800021698000B4
:107CF00002002000A3472400D02D02000000000055
:107D000060698800716988001069800021698000BD
:107D100002802300535B24008E2E0200000000002E
:107D2000090031000800320000C02B0081652400EA
:107D300012698000236980008E2E0200000000007E
:107D40000100310003003A0010C0B30000E0B700AA
:107D5000BE0537004300A90060698000716980009A
:107D6000024E240033B22400F62E02000000000070
:107D70008002780001037800050078008600780012
:107D80000200200003122400D02D02000000000099
:107D900080037800010478000700780088007800EC
:107DA00002002400C36124008030020000000000B3
:107DB000306988004169880030698000416980002D
:107DC0004A31020000000000506988007B00370043
:107DD000046980004822DE006524E1003A003A0090
:107DE000106980002169800002002000A347240060
:107DF000D02D0200000000006069880071698800D1
:107E0000106980002169800002C02A0033632400C9
:107E10008E2E020000000000090031000800320030
:107E200000A02900416924001269800023698000B4
:107E30008E2E0200000000000100310003003A0015
:107E400010C0B30000E0B700800537004300A90070
:107E50006069800071698000024E240033B2240002
:107E6000F62E020000000000800278000103780076
:107E7000050078008600780002002000031024002E
:107E8000D02D02000000000080037800010478007B
:107E9000070078008800780002002400C3612400F5
:107EA00080300200000000003069880041698800CD
:107EB00030698000416980004A3102000000000002
:107EC000506988003D003700046980004822DE00C8
:107ED0006624E10039003A001069800021698000C1
:107EE00002002000A3472400D02D02000000000063
:107EF00060698800716988001069800021698000CC
:107F000002E02800836824008E2E0200000000009A
:107F1000090031000800320000A02E00B16C2400DE
:107F200012698000236980008E2E0200000000008C
:107F30000100310003003A0010C0B30000E0B700B8
:107F4000420537004300A900606980007169800024
:107F5000024E240033B22400F62E0200000000007E
:107F60008002780001037800050078008600780020
:107F700002002000030C2400D02D020000000000AD
:107F800080037800010478000700780088007800FA
:107F900002002400C36124008030020000000000C1
:107FA000306988004169880030698000416980003B
:107FB0004A310200000000005069880021CDBF0056
:107FC00030EDB7002A0DF800320DF90076310200CD
:107FD0000000000021CDBF000FECB700220DF8001B
:107FE0000808F900240DF8000A08F9002A0DF80025
:107FF000100CF9000F4CE20002003A00A834020015
:10800000000000000F4CE200CD003A004300A90040
:108010004040800051408000F226210033B0230010
:10802000F62E0200000000008002780001037800B4
:1080300001002000010078005A1602000000000034
:108040008100E8003322AF00FEFF3700A011880056
:10805000500020000008E600F6FF37000000200076
:108060008500780006017800BC35020000000000A1
:10807000290020007438020000000000B100200038
:10808000010078005A160200000000008100E8009C
:108090003322AF00FEFF3700A0118800E00020006F
:1080A0000008E600F6FF37003A6DEF003B6DEF0089
:1080B000A6200200000000006029EF004300A90094
:1080C0004040800051408000F226210033A8230068
:1080D000F62E020000000000800278000103780004
:1080E000050078008600780002002000832C240020
:1080F0008E2E020000000000330039004300A9006A
:108100004040800051408000F226210033B023001F
:10811000F62E0200000000008002780001037800C3
:10812000000020008500780006017800BC350200C0
:108130000000000029002000A63A02000000000014
:1081400070C2B3003AEDB70020C0B3003BEDB700FA
:10815000A62002000000000000CEB3003AEDB700F8
:10816000CC2002000000000000CEB3003AEDB700C2
:10817000CC2002000000000000CEB3003AEDB700B2
:10818000CC20020000000000B0C3B3003AEDB700FD
:1081900020C0B3003BEDB700A620020000000000A5
:1081A0003A6DEF00CC200200000000003A6DEF00B5
:1081B000CC200200000000003A6DEF00CC2002004D
:1081C00000000000320037004300A900404080005A
:1081D00051408000F226210033B02300F62E020029
:1081E00000000000800278000103780000002000F9
:1081F0008500780006017800BC3502000000000010
:1082000019002000A63A02000000000070C2B3006E
:108210003AEDB70020C0B3003BEDB700A620020046
:10822000000000003A6DEF00CC20020000000000CA
:108230003A6DEF00CC200200000000003A6DEF0024
:10824000CC20020000000000B0C3B3003AEDB7003C
:1082500020C0B3003BEDB700A620020000000000E4
:1082600000CEB3003AEDB700CC20020000000000C1
:1082700000CEB3003AEDB700CC20020000000000B1
:1082800000CEB3003AEDB700CC20020000000000A1
:1082900030C0B30030EDB7002E2402000000000013
:1082A0003A6DEF0030C0B3003BEDB700A6200200EE
:1082B0000000000006E8A900050020000500780085
:1082C00076160200000000000040B3004220AF001C
:1082D000050037008502E80036EDB70024240200CF
:1082E00000000000F5FF370028C8BF0036EDB700DA
:1082F000242402000000000027C8BF00800278008C
:108300000B60EF0006002000050078008600780072
:1083100004002000E22B02000000000000C2B300B5
:1083200036EDB700242402000000000000C2B300B4
:1083300036EDB700242402000000000036043700A8
:10834000746080004822DE006124E10094003A005D
:1083500001002000010078008616020000000000E5
:108360008100E8003322AF00FEFF3700A011880033
:10837000300020000008E600F6FF37000000200073
:108380004140800052408000BC35020000000000E7
:108390002900200074380200000000009100200035
:1083A0000100780086160200000000008100E8004D
:1083B0003322AF00FEFF3700A0118800C00020006C
:1083C0000008E600F6FF37003A6DEF003B6DEF0066
:1083D000A6200200000000006029EF004300A90071
:1083E0004040800051408000F226210033A8230045
:1083F000F62E0200000000008002780001037800E1
:10840000000020008500780006017800BC350200DD
:108410000000000019002000A63A02000000000041
:1084200070C2B3003AEDB70020C0B3003BEDB70017
:10843000A6200200000000003A6DEF00CC200200F0
:10844000000000003A6DEF00CC20020000000000A8
:108450003A6DEF00CC20020000000000B0C3B30072
:108460003AEDB70020C0B3003BEDB700A6200200F4
:108470000000000000CEB3003AEDB700CC200200AF
:108480000000000000CEB3003AEDB700CC2002009F
:108490000000000000CEB3003AEDB700CC2002008F
:1084A0000000000030C0B30030EDB7002E24020001
:1084B000000000003A6DEF0030C0B3003BEDB700A4
:1084C000A62002000000000006E8A9000500200028
:1084D00005007800A0160200000000000040B30074
:1084E0004220AF00050037008502E80036EDB700F6
:1084F0002424020000000000F5FF370028C8BF0058
:1085000036EDB700242402000000000027C8BF0099
:10851000800278000B60EF00060020000500780064
:108520008600780004002000E22B0200000000001A
:1085300000C2B30036EDB7002424020000000000A2
:1085400000C2B30036EDB700242402000000000092
:1085500010C4B3003AEDB70030C0B3003BEDB70034
:10856000A62002000000000006E8A9000500200087
:1085700005007800B0160200000000000040B300C3
:108580004220AF00050037008502E80036EDB70055
:108590002424020000000000F5FF37009E0337008E
:1085A000746080004822DE006224E10094003A00FA
:1085B0000100200001007800C01602000000000049
:1085C0008100E8003322AF00FEFF3700A0118800D1
:1085D000300020000008E600F6FF37000000200011
:1085E0004140800052408000BC3502000000000085
:1085F00029002000743802000000000091002000D3
:1086000001007800C0160200000000008100E800B0
:108610003322AF00FEFF3700A0118800C000200009
:108620000008E600F6FF37003A6DEF003B6DEF0003
:10863000A6200200000000006029EF004300A9000E
:108640004040800051408000F226210033A82300E2
:10865000F62E02000000000080027800010378007E
:10866000000020008500780006017800BC3502007B
:108670000000000019002000A63A020000000000DF
:1086800070C2B3003AEDB70020C0B3003BEDB700B5
:10869000A6200200000000003A6DEF00CC2002008E
:1086A000000000003A6DEF00CC2002000000000046
:1086B0003A6DEF00CC20020000000000B0C3B30010
:1086C0003AEDB70020C0B3003BEDB700A620020092
:1086D0000000000000CEB3003AEDB700CC2002004D
:1086E0000000000000CEB3003AEDB700CC2002003D
:1086F0000000000000CEB3003AEDB700CC2002002D
:108700000000000030C0B30030EDB7002E2402009E
:10871000000000003A6DEF0030C0B3003BEDB70041
:10872000A62002000000000006E8A90005002000C5
:1087300005007800DA160200000000000040B300D7
:108740004220AF00050037008502E80036EDB70093
:108750002424020000000000F5FF370028C8BF00F5
:1087600036EDB700242402000000000027C8BF0037
:10877000800278000B60EF00060020000500780002
:108780008600780004002000E22B020000000000B8
:1087900000C2B30036EDB700242402000000000040
:1087A00000C2B30036EDB700242402000000000030
:1087B00010C4B3003AEDB70030C0B3003BEDB700D2
:1087C000A62002000000000006E8A9000500200025
:1087D00005007800B0160200000000000040B30061
:1087E0004220AF00050037008502E80036EDB700F3
:1087F0002424020000000000F5FF370006033700C4
:10880000746080004822DE006324E10099003A0091
:108810000100200001007800EA16020000000000BC
:108820008100E8003322AF00FEFF3700A01188006E
:10883000400020000008E600F6FF3700000020009E
:108840004140800052408000BC3502000000000022
:10885000290020007438020000000000A100200060
:1088600001007800EA160200000000008100E80024
:108870003322AF00FEFF3700A0118800D000200097
:108880000008E600F6FF37003A6DEF003B6DEF00A1
:10889000A6200200000000006029EF004300A900AC
:1088A0004040800051408000F226210033A8230080
:1088B000F62E02000000000080027800010378001C
:1088C00005007800860078000200200003122400D2
:1088D000803002000000000080037800010478006E
:1088E000000020008700780008017800BC350200F5
:1088F0000000000019002000A63A0200000000005D
:1089000070C2B3003AEDB70020C0B3003BEDB70032
:10891000A6200200000000003A6DEF00CC2002000B
:10892000000000003A6DEF00CC20020000000000C3
:108930003A6DEF00CC20020000000000B0C3B3008D
:108940003AEDB70020C0B3003BEDB700A62002000F
:10895000000000003A6DEF00CC2002000000000093
:108960003A6DEF00CC200200000000003A6DEF00ED
:10897000CC2002000000000030C0B30030EDB70092
:108980002E240200000000003A6DEF0030C0B3005A
:108990003BEDB700A62002000000000006E8A90099
:1089A0000500200005007800061702000000000006
:1089B0000040B3004220AF00050037008502E80008
:1089C00036EDB7002424020000000000F5FF370058
:1089D00028C8BF0036EDB7002424020000000000C4
:1089E00027C8BF00800278000B60EF00060020005F
:1089F000050078008600780004002000E22B0200C9
:108A00000000000000C2B30036EDB70024240200CD
:108A10000000000000C2B30036EDB70024240200BD
:108A20000000000010C4B3003AEDB70030C0B3003E
:108A30003BEDB700A62002000000000006E8A900F8
:108A40000500200005007800B016020000000000BC
:108A50000040B3004220AF00050037008502E80067
:108A600036EDB7002424020000000000F5FF3700B7
:108A700069023700746080004822DE006424E1004F
:108A800026013A00010020000100780018170200BA
:108A9000000000008100E8003322AF00FEFF370035
:108AA000A0118800400020000008E600F6FF370013
:108AB000000020004140800052408000BC35020090
:108AC00000000000290020007438020000000000AF
:108AD000A10020000100780018170200000000002B
:108AE0008100E8003322AF00FEFF3700A0118800AC
:108AF000D00020000008E600F6FF3700404080006C
:108B00005140800002002400C36124008E2E020028
:108B1000000000007B0039003A6DEF003B6DEF0074
:108B2000A6200200000000006029EF004300A90019
:108B30004040800051408000F226210033A82300ED
:108B4000F62E020000000000800278000103780089
:108B5000050078008600780002002000031224003F
:108B600080300200000000008003780001047800DB
:108B7000000020008700780008017800BC35020062
:108B80000000000019002000A63A020000000000CA
:108B900070C2B3003AEDB70020C0B3003BEDB700A0
:108BA000A6200200000000003A6DEF00CC20020079
:108BB000000000003A6DEF00CC2002000000000031
:108BC0003A6DEF00CC20020000000000B0C3B300FB
:108BD0003AEDB70020C0B3003BEDB700A62002007D
:108BE000000000003A6DEF00CC2002000000000001
:108BF0003A6DEF00CC200200000000003A6DEF005B
:108C0000CC2002000000000030C0B30030EDB700FF
:108C10002E240200000000003A6DEF0030C0B300C7
:108C20003BEDB700A62002000000000006E8A90006
:108C30000500200005007800341702000000000045
:108C40000040B3004220AF00050037008502E80075
:108C500036EDB7002424020000000000F5FF3700C5
:108C600028C8BF0036EDB700242402000000000031
:108C700027C8BF00800278000B60EF0006002000CC
:108C8000050078008600780004002000E22B020036
:108C90000000000000C2B30036EDB700242402003B
:108CA0000000000000C2B30036EDB700242402002B
:108CB0000000000010C4B3003AEDB70030C0B300AC
:108CC0003BEDB700A62002000000000006E8A90066
:108CD0000500200005007800B0160200000000002A
:108CE0000040B3004220AF00050037008502E800D5
:108CF00036EDB7002424020000000000F5FF370025
:108D00008500370000002400C1612400424080003B
:108D1000534080008E2E0200000000000100310050
:108D20007D003A003A6DEF003B6DEF00A620020097
:108D3000000000006029EF004300A90040408000CF
:108D400051408000F226210033A82300F62E0200B5
:108D50000000000080027800010378000500780020
:108D60008600780002002000A34724008030020023
:108D7000000000008003780001047800000020005B
:108D80008700780008017800BC3502000000000070
:108D900029002000A63A02000000000070C2B300C3
:108DA0003AEDB70020C0B3003BEDB700A6200200AB
:108DB0000000000000CEB3003AEDB700CC20020066
:108DC0000000000000CEB3003AEDB700CC20020056
:108DD0000000000000CEB3003AEDB700CC20020046
:108DE00000000000B0C3B3003AEDB70020C0B300EC
:108DF0003BEDB700A6200200000000003A6DEF0036
:108E0000CC200200000000003A6DEF00CC200200F0
:108E1000000000003A6DEF00CC20020000000000CE
:108E200030C0B30030EDB7002E2402000000000077
:108E30003A6DEF0030C0B3003BEDB700A620020052
:108E40000000000006E8A9000500200005007800E9
:108E500034170200000000000040B3004220AF00C1
:108E6000050037008502E80036EDB7002424020033
:108E700000000000F5FF370028C8BF0036EDB7003E
:108E8000242402000000000027C8BF0080027800F0
:108E90000B60EF00060020000500780086007800D7
:108EA00004002000E22B02000000000000C2B3001A
:108EB00036EDB700242402000000000000C2B30019
:108EC00036EDB700242402000000000010C4B300F7
:108ED0003AEDB70030C0B3003BEDB700A62002006A
:108EE0000000000006E8A900050020000500780049
:108EF00046170200000000000040B3004220AF000F
:108F0000050037008502E80036EDB7002424020092
:108F100000000000F5FF37003F013700746080005B
:108F20004822DE006524E1009C003A000100200098
:108F30000100780056170200000000008100E800E0
:108F40003322AF00FEFF3700A01188004000200050
:108F50000008E600F6FF37000000200041408000D6
:108F600052408000BC3502000000000029002000B3
:108F70007438020000000000A10020000100780009
:108F800056170200000000008100E8003322AF0005
:108F9000FEFF3700A0118800D00020000008E60086
:108FA000F6FF37003A6DEF003B6DEF00A6200200A0
:108FB000000000006029EF004300A900404080004D
:108FC00051408000F226210033A82300F62E020033
:108FD000000000008002780001037800050078009E
:108FE0008600780002002000A347240080300200A1
:108FF00000000000800378000104780000002000D9
:109000008700780008017800BC35020000000000ED
:1090100029002000A63A02000000000070C2B30040
:109020003AEDB70020C0B3003BEDB700A620020028
:109030000000000000CEB3003AEDB700CC200200E3
:109040000000000000CEB3003AEDB700CC200200D3
:109050000000000000CEB3003AEDB700CC200200C3
:1090600000000000B0C3B3003AEDB70020C0B30069
:109070003BEDB700A6200200000000003A6DEF00B3
:10908000CC200200000000003A6DEF00CC2002006E
:10909000000000003A6DEF00CC200200000000004C
:1090A00030C0B30030EDB7002E24020000000000F5
:1090B0003A6DEF0030C0B3003BEDB700A6200200D0
:1090C0000000000006E8A900050020000500780067
:1090D00072170200000000000040B3004220AF0001
:1090E000050037008502E80036EDB70024240200B1
:1090F00000000000F5FF370028C8BF0036EDB700BC
:10910000242402000000000027C8BF00800278006D
:109110000B60EF0006002000050078008600780054
:1091200004002000E22B02000000000000C2B30097
:1091300036EDB700242402000000000000C2B30096
:1091400036EDB700242402000000000010C4B30074
:109150003AEDB70030C0B3003BEDB700A6200200E7
:109160000000000006E8A9000500200005007800C6
:1091700046170200000000000040B3004220AF008C
:10918000050037008502E80036EDB7002424020010
:1091900000000000F5FF37009F003700746080007A
:1091A0004822DE006624E1009B003A000100200016
:1091B0000100780084170200000000008100E80030
:1091C0003322AF00FEFF3700A011880040002000CE
:1091D0000008E600F6FF3700000020004140800054
:1091E00052408000BC350200000000002900200031
:1091F0007438020000000000A10020000100780087
:1092000084170200000000008100E8003322AF0054
:10921000FEFF3700A0118800D00020000008E60003
:10922000F6FF37003A6DEF003B6DEF00A62002001D
:10923000000000006029EF004300A90040408000CA
:1092400051408000F226210033A82300F62E0200B0
:10925000000000008002780001037800050078001B
:109260008600780002002000A3472400803002001E
:109270000000000080037800010478000000200056
:109280008700780008017800BC350200000000006B
:1092900029002000A63A02000000000070C2B300BE
:1092A0003AEDB70020C0B3003BEDB700A6200200A6
:1092B0000000000000CEB3003AEDB700CC20020061
:1092C0000000000000CEB3003AEDB700CC20020051
:1092D0000000000000CEB3003AEDB700CC20020041
:1092E00000000000B0C3B3003AEDB70020C0B300E7
:1092F0003BEDB700A6200200000000003A6DEF0031
:10930000CC200200000000003A6DEF00CC200200EB
:10931000000000003A6DEF00CC20020000000000C9
:1093200030C0B30030EDB7002E2402000000000072
:109330003A6DEF0030C0B3003BEDB700A62002004D
:109340000000000006E8A9000500200005007800E4
:10935000A0170200000000000040B3004220AF0050
:10936000050037008502E80036EDB700242402002E
:1093700000000000F5FF370028C8BF0036EDB70039
:10938000242402000000000027C8BF0080027800EB
:109390000B60EF00060020000500780086007800D2
:1093A00004002000E22B02000000000000C2B30015
:1093B00036EDB700242402000000000000C2B30014
:1093C00036EDB700242402000000000010C4B300F2
:1093D0003AEDB70030C0B3003BEDB700A620020065
:1093E0000000000006E8A900050020000500780044
:1093F00046170200000000000040B3004220AF000A
:10940000050037008502E80036EDB700242402008D
:1094100000000000F5FF370040C0B30030EDB7009A
:109420002E2402000000000050C0B30030EDB70051
:109430002E2402000000000010C0B30030EDB70081
:10944000E03B0200000000000060EF004F047800E5
:10945000CF0378004F037800CF02780000000600A9
:10946000851F7800861F7800871F78000E6CEF003C
:10947000D222EF0004802000B41688000000000013
:1094800000000000F43F200094168800D742A80096
:10949000D342A900000000000000000000C3B30098
:1094A0001CEDB7001D6DEF00B428020000000000A5
:1094B00050C3B3001CEDB7001D6DEF00B4280200CF
:1094C00000000000562402000000000056240200A4
:1094D0000000000010C0B3003AEDB7003B6DEF0094
:1094E000A620020000000000050020000500780012
:1094F000B8180200000000000040B3004220AF0096
:10950000050037008502E80036EDB700242402008C
:1095100000000000F5FF370010C0B3003AEDB700BF
:1095200030C0B3003BEDB700A620020000000000F1
:109530000500200005007800D2180200000000009D
:109540000040B3004220AF00050037008502E8006C
:1095500036EDB7002424020000000000F5FF3700BC
:1095600010C0B3003AEDB70040C0B3003BEDB70008
:10957000A620020000000000050020000500780081
:10958000EC180200000000000040B3004220AF00D1
:10959000050037008502E80036EDB70024240200FC
:1095A00000000000F5FF37000500200005007800EE
:1095B00008190200000000000040B3004220AF0084
:1095C000060037008502E8003322AF00FEFF3700B7
:1095D00034E2B7003562EF00F4FF370005002000E9
:1095E0000500780028190200000000000040B300C8
:1095F0004220AF00060037008502E8003322AF00AA
:10960000FEFF370034E2B7003562EF00F4FF3700A9
:109610000500200005007800461902000000000047
:109620000040B3004220AF00060037008502E8008A
:109630003322AF00FEFF370034E2B7003562EF009F
:10964000F4FF3700D242A800D442AE000100370038
:10965000FCFF3700D282A800D482AE0001003700A0
:10966000FCFF370010C0B3000EECB700D262A800B8
:10967000D462AF0008003700D242A800D442AF0045
:1096800005003700D282A800D482AF000200370064
:1096900000000000F5FF3700D282A800D482AF009E
:1096A00001003700F3003700BC2C0200000000006E
:1096B000562402000000000010C0B3003AEDB700CD
:1096C0003B6DEF00A6200200000000000500200016
:1096D0000500780064190200000000000040B3009B
:1096E0004220AF00050037008502E80036EDB700E4
:1096F0002424020000000000F5FF370010C0B30072
:109700003AEDB70020C0B3003BEDB700A620020041
:10971000000000000500200005007800801902000C
:10972000000000000040B3004220AF0005003700F9
:109730008502E80036EDB700242402000000000096
:10974000F5FF370010C0B3003AEDB70030C0B300EA
:109750003BEDB700A620020000000000050020003D
:10976000050078009C190200000000000040B300D2
:109770004220AF00050037008502E80036EDB70053
:109780002424020000000000F5FF370010C0B300E1
:109790003AEDB70040C0B3003BEDB700A620020091
:1097A000000000000500200005007800B819020044
:1097B000000000000040B3004220AF000500370069
:1097C0008502E80036EDB700242402000000000006
:1097D000F5FF370010C0B3003AEDB70050C0B3003A
:1097E0003BEDB700A62002000000000005002000AD
:1097F00005007800D4190200000000000040B3000A
:109800004220AF00050037008502E80036EDB700C2
:109810002424020000000000F5FF370005002000AE
:1098200005007800F0190200000000000040B300BD
:109830004220AF00060037008502E8003322AF0067
:10984000FEFF370034E2B7003562EF00F4FF370067
:109850000500200005007800141A02000000000036
:109860000040B3004220AF00060037008502E80048
:109870003322AF00FEFF370034E2B7003562EF005D
:10988000F4FF37000500200005007800321A0200BE
:10989000000000000040B3004220AF000600370087
:1098A0008502E8003322AF00FEFF370034E2B70044
:1098B0003562EF00F4FF3700050020000500780056
:1098C0005C1A0200000000000040B3004220AF001C
:1098D000060037008502E8003322AF00FEFF3700A4
:1098E00034E2B7003562EF00F4FF3700D282A800FF
:1098F000D482AF00FDFF3700409C2000641F0200AF
:109900000000000056240200000000000828EF00BC
:10991000442C24005440880005002000462C2400DC
:10992000216DEF001569880026698800EC3C020073
:10993000000000003A6DEF0030C0B3003BEDB7000F
:10994000A6200200000000000500200005007800AD
:109950007C1A0200000000000040B3004220AF006B
:10996000050037008502E80036EDB7002424020028
:1099700000000000F5FF3700D282A800D482AF00BB
:109980003C003700D262A800D462AE001A00370053
:10999000D262A800D462AE0004003700500020005C
:1099A000641F020000000000F9FF3700A0C2B300EE
:1099B00028E8B7004300A8004040800051408000E4
:1099C000D2CC2C00C3D42300F62E020000000000ED
:1099D0004040880051408800216DEF000808F800E1
:1099E000220DF9000A08F800240DF900EC3C0200F1
:1099F000000000001C003700D242A800D442AE0094
:109A000019003700D242A800D442AE00040037004B
:109A100050002000641F020000000000F9FF370022
:109A2000A0C2B30028E8B7004300A900404080006E
:109A300051408000D2CC2C00C3D42300F62E02006B
:109A4000000000004040880051408800216DEF0078
:109A50000808F800220DF9000A08F800240DF900A2
:109A6000EC3C02000000000020C0B3000EECB70088
:109A7000C1FF37007A25020000000000CF03780004
:109A80004F037800CF02780000000600851F7800A1
:109A9000C500200003000900B51F780000F0A600F3
:109AA000020037000000EA000480A0008002EB0002
:109AB000800378008404780004F0A1000404E0002E
:109AC00006003A0009F0A700020037000500200058
:109AD0000F003700050020000D003700E64252005D
:109AE0000A0039000003200009F0A600000220004F
:109AF0003322AF00FEFF3700A01188008502E90085
:109B0000FBFF3B0055002000010037008402780075
:109B10006400200005E0A00009F0A70005F0A00007
:109B200008712200110009008883D800DA4D020074
:109B30000000000081037800883E20001100090029
:109B40008883D800DA4D020000000000810378000D
:109B500048062000110009008883D800DA4D020071
:109B60000000000081037800A80020001100090017
:109B70008883D800DA4D0200000000000980A600AA
:109B800005003700D00220003322AF00FEFF37006F
:109B9000A01188000980A1000003200000C040003F
:109BA000500188003322AF00FEFF3700A01188006B
:109BB00020003700060320000000E0000E003A00FD
:109BC00005E0A600160037000402E9000524E100C4
:109BD000020032004200AF00000006000000E0007A
:109BE00005003A0005E0A6000D00370005F0A600CC
:109BF000060220000A00370005E0A1000980A60047
:109C00000700370000057800D00220003322AF00A3
:109C1000FEFF3700A01188000980A1000A0078002B
:109C2000004043003322AF00FEFF3700A011880040
:109C3000000006002501200003000900CF12780073
:109C4000CF02780000000600851F7800861F78008C
:109C500080C0B30029ECB70000C2B3002AECB70003
:109C600070C2B3001CEDB7002ACCBF001DEDB700D9
:109C7000B42802000000000080C2B3001CEDB70051
:109C800029CCBF001DEDB700B42802000000000081
:109C9000550CA9005624020000000000A0C0B3002B
:109CA0003AEDB70050C0B3003BEDB700A62002006C
:109CB00000000000050020000500780016180200D2
:109CC000000000000040B3004220AF000500370054
:109CD0008502E80036EDB7002424020000000000F1
:109CE000F5FF370005002000050078002E1802005F
:109CF000000000000040B3004220AF000600370023
:109D00008502E8003322AF00FEFF370034E2B700DF
:109D10003562EF00F4FF3700803E2000641F020030
:109D20000000000070C2B3001CEDB70000C8B30013
:109D30001DEDB700B428020000000000400620001E
:109D4000641F02000000000070C2B3001CEDB700E9
:109D500000CCB3001DEDB700B428020000000000E5
:109D600040062000641F0200000000004300A8001D
:109D70004040800051408000D2CC2C00C3D423004E
:109D8000F62E02000000000040408800514088008C
:109D9000216DEF000808F800220DF9000A08F8000C
:109DA000240DF900EC3C02000000000040062000F9
:109DB000641F020000000000536CEF0094628000FA
:109DC0004822DE0004C4B2006E00320070C2B3004C
:109DD0001CEDB70053CCBF001DEDB700B428020046
:109DE0000000000040062000641F02000000000088
:109DF000D322A8002800090000000000DEC2A8004D
:109E00002900090000000000D722A900D322A900E0
:109E10002800090000000000E2C2A900DEC2A9007B
:109E200031CCB30062280200000000006104E100B0
:109E300001003A000000000011002000811F78009E
:109E4000CF0078001E2902000000000013ECB700CC
:109E500001002000811F7800CF0078001E29020039
:109E60000000000020ECB700D322A9000000000091
:109E7000DEC2A800E0C2AE00FEFF370028000900E5
:109E8000000000000100090000000000D322A8002B
:109E9000280009000000000020CCBF0097ECB700AC
:109EA000946280004822DE0063C5200083024200E5
:109EB00097CCBF00804A7800946280004822DE0080
:109EC00063C5200003004200904278003322AF00B7
:109ED000FEFF370004022000A41188003322AF00E7
:109EE000FEFF370054072000A411880053CCBF00A8
:109EF0000160EF0004002000C82402000000000000
:109F00003322AF00FEFF3700D4032000A4118800E5
:109F1000054078000160EF0004002000C824020022
:109F2000000000003322AF00FEFF370004022000D3
:109F3000A4118800A0C0B3003AEDB70050C0B30030
:109F40003BEDB700A6200200000000000500200045
:109F50000500780048180200000000000040B3002F
:109F60004220AF00050037008502E80036EDB7005B
:109F70002424020000000000F5FF3700536CEC00C1
:109F80008EFF37004300A900404080005140800010
:109F9000D2CC2C00C3DC2300F62E0200000000000F
:109FA0008002780001037800216DEF0015698800B8
:109FB00026698800EC3C02000000000040062000FA
:109FC000641F020000000000536CEF0094628000E8
:109FD0004822DE0004C4B2006E00320070C2B3003A
:109FE0001CEDB70053CCBF001DEDB700B428020034
:109FF0000000000040062000641F02000000000076
:10A00000D322A8002800090000000000DEC2A8003A
:10A010002900090000000000D722A900D322A900CE
:10A020002800090000000000E2C2A900DEC2A90069
:10A0300031CCB30062280200000000006104E1009E
:10A0400001003A000000000011002000811F78008C
:10A05000CF0078001E2902000000000013ECB700BA
:10A0600001002000811F7800CF0078001E29020027
:10A070000000000020ECB700D322A900000000007F
:10A08000DEC2A800E0C2AE00FEFF370028000900D3
:10A09000000000000100090000000000D322A80019
:10A0A000280009000000000020CCBF0097ECB7009A
:10A0B000946280004822DE0083C9200083024200AF
:10A0C00097CCBF00804A7800946280004822DE006E
:10A0D00083C9200003004200904278003322AF0081
:10A0E000FEFF370004022000A41188003322AF00D5
:10A0F000FEFF3700F4062000A411880053CCBF00F7
:10A100000160EF0004002000C824020000000000ED
:10A110003322AF00FEFF3700D4032000A4118800D3
:10A12000054078000160EF0004002000C824020010
:10A13000000000003322AF00FEFF370004022000C1
:10A14000A4118800A0C0B3003AEDB70050C0B3001E
:10A150003BEDB700A6200200000000000500200033
:10A160000500780048180200000000000040B3001D
:10A170004220AF00050037008502E80036EDB70049
:10A180002424020000000000F5FF3700536CEC00AF
:10A190008EFF3700526CEF009462800004C4B2005E
:10A1A0002A003200946280000960EF00A3CD2000F5
:10A1B00083024200946280000960EF0083C920009E
:10A1C0000300420010437800946280000960EF00B1
:10A1D00063C5200003004200104078000040530097
:10A1E000804A7800946280000960EF00A3CD2000CF
:10A1F0000300420090427800010020000100780036
:10A2000060180200000000008100E8003322AF0067
:10A21000FEFF3700A0118800400020000008E60083
:10A22000F6FF37000500FB0004002000464D020049
:10A23000000000003322AF00FEFF370004022000C0
:10A24000A4118800526CEC00D3FF37001B6DEF00A7
:10A25000D46880004822DE0024C3B20037003200F8
:10A26000550CAE000100370034003700010020001B
:10A270000100780076180200000000008100E8006C
:10A280003322AF00FEFF3700A011880050002000ED
:10A290000008E600F6FF37001BCDBF000000FB0002
:10A2A00004002000C8240200000000003322AF0098
:10A2B000FEFF370004022000A411880050C0B30044
:10A2C00052ECB70094628000C4C3B200190032009F
:10A2D000946280000960EF00A3CD200003004200DB
:10A2E00010407800D9ECB70052CCBF0054ECB70056
:10A2F00004002000D3688000C819DE00034052002B
:10A30000C46680004822DE000024E100070035001A
:10A31000D9CCBF00D46880004822DE000024E100D0
:10A3200002003500550CA80002003700526CEC000A
:10A33000E4FF37001B6DEC00C5FF370070C2B300AF
:10A340001CEDB70054CCBF001DEDB700B4280200CF
:10A350000000000040062000641F02000000000012
:10A3600054CCBF002AECB7000100200001007800A7
:10A370008C180200000000008100E8003322AF00CA
:10A38000FEFF3700A0118800500020000008E60002
:10A39000F6FF37002ACCBF000160EF003400200038
:10A3A000C8240200000000003322AF00FEFF370087
:10A3B00004022000A41188003322AF00FEFF370002
:10A3C00004022000A41188003322AF00FEFF3700F2
:10A3D00004022000A411880050C0B30030EDB70083
:10A3E0002E24020000000000A0C0B3003AEDB70028
:10A3F00050C0B3003BEDB700A620020000000000F3
:10A400000500200005007800A618020000000000EA
:10A410000040B3004220AF00050037008502E8008D
:10A4200036EDB7002424020000000000F5FF3700DD
:10A43000556180000B60EF000600200005007800E9
:10A440008600780034002000E22B020000000000AB
:10A450002ACCBF001EEDB700D41F2000E46888009E
:10A46000362B020000000000007D2000641F020067
:10A470000000000050C0B30030EDB7002E240200F1
:10A48000000000004300A8004040800051408000D0
:10A49000D2CC2C00C3D42300F62E02000000000012
:10A4A0008002780001037800216DEF0015698800B3
:10A4B00026698800EC3C0200000000004F03780091
:10A4C000CF02780000000600746080006224E10082
:10A4D000010032000A003700244E02000000000094
:10A4E000BC2C02000000000010C0B3001EEDB7003D
:10A4F000C41F2000E4688800362B02000000000022
:10A50000000006005C4CE200560032000F4CE200F6
:10A510000A003A004300A9004040800051408000FA
:10A52000D2CC2C00C3D42300F62E02000000000081
:10A53000A0608800B1608800490037007460800026
:10A540004822DE006124E1000400320074608000D3
:10A550004822DE006224E1000A003A004300A9001C
:10A5600040408000514080000200200003F823009A
:10A57000F62E020000000000A0608800B160880094
:10A5800037003700746080004822DE006324E10059
:10A590000A003A004300A90040408000514080007A
:10A5A0000200200003F22300F62E0200000000004B
:10A5B000A0608800B16088002900370074608000C6
:10A5C0004822DE006424E1000A003A004300A900AA
:10A5D00040408000514080000200200003F823002A
:10A5E000F62E020000000000A0608800B160880024
:10A5F0001B003700746080004822DE006524E10003
:10A600000A003A004300A900404080005140800009
:10A610000200200003FA2300F62E020000000000D2
:10A62000A0608800B16088000D0037007460800071
:10A630004822DE006624E10009003A004300A90038
:10A640004040800051408000F2282C0053FD230040
:10A65000F62E020000000000A0608800B1608800B3
:10A66000570037005C4CE20055003A000F4CE20006
:10A670000A003A004300A80040408000514080009A
:10A68000D2CC2C00C3D42300F62E02000000000020
:10A69000A0608800B16088004900370074608000C5
:10A6A0004822DE006124E100040032007460800072
:10A6B0004822DE006224E1000A003A004300A800BC
:10A6C00040408000514080000200200003F8230039
:10A6D000F62E020000000000A0608800B160880033
:10A6E00037003700746080004822DE006324E100F8
:10A6F0000A003A004300A80040408000514080001A
:10A700000200200003F22300F62E020000000000E9
:10A71000A0608800B1608800290037007460800064
:10A720004822DE006424E1000A003A004300A80049
:10A7300040408000514080000200200003F82300C8
:10A74000F62E020000000000A0608800B1608800C2
:10A750001B003700746080004822DE006524E100A1
:10A760000A003A004300A8004040800051408000A9
:10A770000200200003FA2300F62E02000000000071
:10A78000A0608800B16088000D0037007460800010
:10A790004822DE006624E10009003A004300A800D8
:10A7A0004040800051408000F2282C0053FD2300DF
:10A7B000F62E020000000000A0608800B160880052
:10A7C0000FCCBF0021EDB700140CF800220DF900EA
:10A7D000160CF800240DF900EC3C0200000000000B
:10A7E0000060EF0000000600044C80004822DE00FC
:10A7F0006424E10001003A008169EF008149E20030
:10A8000009003A00244C800014C6B20006003A0049
:10A8100010C0B30081E9B7007609F8007809F900A3
:10A820003500370033003700044C80004822DE003A
:10A830006124E10009003A00244C800024C6B200E3
:10A8400006003A0020C0B30081E9B7007609F8009D
:10A850007A09F9002800370026003700044C8000F0
:10A860004822DE006224E10009003A00244C800006
:10A8700034C6B20006003A0030C0B30081E9B70028
:10A880007609F8007C09F9001B0037001900370031
:10A89000044C80004822DE006224E10009003A00F6
:10A8A000244C800034C4B20006003A0030C0B3002B
:10A8B00081E9B7007609F8007C09F9000E0037003D
:10A8C0000C003700044C80004822DE006324E100C5
:10A8D00008003A00244C800044C6B20005003A004B
:10A8E00040C0B30081E9B7007609F8007E09F9009D
:10A8F000010037008169EF0000000600851F780025
:10A90000861F780000027800810278000000EB00CA
:10A910008000EB0085016A00110032000001EB00AD
:10A92000610B20000270A700070037004200A90059
:10A930000482D2008582D2000080D2000281D2003F
:10A940008100E900F7FF3A000180FD004200A90004
:10A950008180D30001F0A1000270A1008140690054
:10A960004F037800CF02780000000600851F7800B2
:10A970008102780000017800640B20008180D20001
:10A980000180FD00F10FB2000142520085417800C4
:10A990000370A000F30FB2000000EB008000EB009A
:10A9A0004200A9008381D3000281D3008180D300BB
:10A9B0000080D3000402E900F9FF3A0005F0A60088
:10A9C000060037000000EA00020032008180EA0041
:10A9D000020037008100EA0000003700CF02780053
:10A9E00000000600851F7800861F780000027800AE
:10A9F000810278000000EB008000EB000600A1005F
:10AA000005F0A600060037000600A0000402EA00D8
:10AA1000020032008582EA00010037008502EA0068
:10AA200085016A00130032000001EB00610B200079
:10AA30000270A700070037004200A9000482D2007C
:10AA40008582D2000080D2000281D2008100E9001C
:10AA5000F7FF3A000180FD004200A9008180D30089
:10AA600001F0A1000270A100814069000600A7006A
:10AA700001F0A0004F037800CF027800000006002C
:10AA8000851F7800C500200003000900B51F78006D
:10AA90000202B80003F0A600020037000383B900E9
:10AAA000010037000303B8004200A90085024300FB
:10AAB00060844B0001F0A60002003700028BB90051
:10AAC00001003700020BB80085024B0008844B00E0
:10AAD0000980B000038BB90008044B0087834C0049
:10AAE000870178000801780085007800040078006C
:10AAF0002501200003000900CF127800CF02780062
:10AB000000000600851F7800C50020000300090032
:10AB1000B51F7800090020004300AF001900200095
:10AB2000891F78008384680001F0A60005003700C3
:10AB30000000EA000100320001003A008100EA0052
:10AB40008180EA0003F0A600050037000201EA0058
:10AB50000100320001003A008301EA008381EA002B
:10AB600003026900150032000002EB008002EB00D6
:10AB70000003EB008003EB00080220004200A90064
:10AB80000080D2008180D2000482D2008582D2006F
:10AB90000328E10001003A0002A0E10003003900AF
:10ABA0000202520083825A004200A8000683D200AB
:10ABB0008783D2000804E900F0FF3A0009F0A600FC
:10ABC000060037000600EA000100320001003A00EA
:10ABD0008700EA008780EA000300370087007800DA
:10ABE0000600780000003700CF0478000900E0007C
:10ABF000010032000400BE0025012000030009000E
:10AC0000CF127800CF027800000006004300A900B0
:10AC100020638000316380004263800053638000C2
:10AC200082550200000000006063880071638800A4
:10AC30004063800051638000626380007363800022
:10AC40004055020000000000246380000000520014
:10AC5000806388003463800001005A00906388009C
:10AC60006063800071638000826380009363800072
:10AC700000000600851F7800861F78000001EB00A9
:10AC80000103780064C110004211DD000200DD0004
:10AC9000800278000C60EC000C60ED000D003200CA
:10ACA00005007800C42ADD004C00DE00F000B20090
:10ACB0000003B000A20320000200E10001003900FF
:10ACC0000D40B4003322AF00FEFF3700A011880012
:10ACD000F1FF37004F037800CF0278000000060034
:10ACE000851F7800861F7800644080006124E100A1
:10ACF00037003A008042EB000648AF008502E800CA
:10AD00000043EB000668AF000603E80001002000E6
:10AD10000100780034150200000000008100E80006
:10AD20003322AF00FEFF3700A01188008000200012
:10AD30000008E600F6FF3700054078000160EF00EC
:10AD400004002000C8240200000000003322AF00ED
:10AD5000FEFF370004022000A41188003322AF0058
:10AD6000FEFF370064042000A41188003322AF00E6
:10AD7000FEFF3700D4032000A411880006407800AD
:10AD80000160EF0004002000C82402000000000061
:10AD900001012000010078003415020000000000CD
:10ADA0008100E8003322AF00FEFF3700A0118800C9
:10ADB000300120000008E600F6FF370020C8BF0081
:10ADC0000160EF0004002000C82402000000000021
:10ADD000644080006124E10037003A008042EB00CB
:10ADE0000688AF008502E8000043EB0006A8AF002C
:10ADF0000603E8003322AF00FEFF37000402200004
:10AE0000A41188003322AF00FEFF37004404200065
:10AE1000A41188003322AF00FEFF3700D4032000C6
:10AE2000A4118800054078000160EF0004002000B4
:10AE3000C82402000000000051002000010078003A
:10AE400058150200000000008100E8003322AF0026
:10AE5000FEFF3700A0118800900020000008E600E7
:10AE6000F6FF3700064078000160EF000400200084
:10AE7000C824020000000000C1002000010078008A
:10AE800058150200000000008100E8003322AF00E6
:10AE9000FEFF3700A0118800000120000008E60036
:10AEA000F6FF370021C8BF000160EF00040020005A
:10AEB000C824020000000000644080006124E1001A
:10AEC0001E003A0001002000010078007815020001
:10AED000000000008100E8003322AF00FEFF3700D1
:10AEE000A0118800400020000008E600F6FF3700AF
:10AEF0002041800004002000C8240200000000005F
:10AF00008100200001007800781502000000000098
:10AF10008100E8003322AF00FEFF3700A011880057
:10AF2000C00020000008E600F6FF37001041800056
:10AF300004002000C82402000000000064408000DB
:10AF40006124E10020003A000100200001007800A7
:10AF500096150200000000008100E8003322AF00D7
:10AF6000FEFF3700A0118800300020000008E60036
:10AF7000F6FF370059C8BF000160EF0021702200C2
:10AF80003A56020000000000610020000100780035
:10AF900096150200000000008100E8003322AF0097
:10AFA000FEFF3700A0118800A00020000008E60086
:10AFB000F6FF37007DC8BF000160EF00217022005E
:10AFC0003A56020000000000644080006124E10065
:10AFD00014003A000100200001007800B0150200C2
:10AFE000000000008100E8003322AF00FEFF3700C0
:10AFF000A0118800400020000008E600F6FF37009E
:10B000007EC8BF000160EF00217022003A560200A6
:10B01000000000003322AF00FEFF370004022000D2
:10B02000A41188004F037800CF02780000000600CA
:10B03000851F7800C500200006000900B51F7800B4
:10B040007809F8008609F900354C8000CC2ADE002A
:10B050006FC0620059E8B7008809F8008A09F90052
:10B060008609F8008809F900404C80008A09E3004D
:10B070000B003200304C80008809E30008003200E9
:10B080008609E200060032008C69EF0040C1B3007F
:10B090009CEBB7008D69EF008E69EF007D033700F0
:10B0A000D54B8000C52ADE007FC062008CE9B70066
:10B0B0007BC9BF00800278000B60EF0005027800BA
:10B0C000044FB2000440780091E9B70000802000EE
:10B0D0007A09B60080027800048020000520E10093
:10B0E00004003A0091C9BF006B40700091E9B700BD
:10B0F0000300370091C9BF006A40700091E9B700B2
:10B10000844C80004822DE00A4C4B20047023A000A
:10B11000C76BEF00E04B80004100DE00005D88005F
:10B12000A22BEF00D04B8000E10260006128E1001B
:10B1300007003A0004002800035D800004804100FD
:10B14000005D8800145D800060024A00145D880084
:10B15000D04B8000E20260006228E10006003A0065
:10B16000045D800060024200045D8800145D800080
:10B1700061024A00145D8800E04B8000E10260003B
:10B180004428DD00C4EBB700265E80000603FB0008
:10B19000F54B8000CC2ADE006F8062000600400084
:10B1A000C4EBB700F54B8000C62ADE00050078002E
:10B1B000F003B200C5EBB700C66BEF007EA9AF008D
:10B1C000C66BEC00F04B80006F4060009DEBB70059
:10B1D000C64BE2000B003A009DCBBF000160EF00C0
:10B1E0004100DE00C46BB400245E80007724E100DF
:10B1F00003003400245E800078405200C4EBB700A6
:10B200000D0037009DCBBF000160EF004100DE0064
:10B21000245E800000405200C4EBB700245E800032
:10B220006024E10004003D00245E8000784242007A
:10B2300004407800C4EBB700005D8000115D800021
:10B240007E540200000000008002780001037800B4
:10B250004300A8000500780086007800D28C290001
:10B26000B3662400F62E0200000000008003780080
:10B2700001047800070078008800780002002A00A6
:10B28000633B24008030020000000000B65402003E
:10B2900000000000205D8800315D8800005D8000B6
:10B2A000115D80007E5402000000000080027800E2
:10B2B000010378004300A8000500780086007800AC
:10B2C00062062B0093662400F62E020000000000A8
:10B2D0008003780001047800205D8000315D8000EB
:10B2E0007E54020000000000800478000105780010
:10B2F000090078008A00780002002A00633B2400DD
:10B30000D02D020000000000B65402000000000032
:10B310007E540200000000004300A80000017800F5
:10B32000810178000700780088007800F62E02007E
:10B330000000000080057800010678000B0078000E
:10B340008C00780012D02C00431F240080300200B3
:10B3500000000000B654020000000000805D88007C
:10B36000915D8800045D8000C3A623008302520023
:10B37000145D800060035A00205D8000315D800014
:10B380007E54020000000000800378000104780071
:10B39000070078008800780002002A00633B240040
:10B3A000D02D020000000000B65402000000000092
:10B3B0008084520001055B00805D8000915D80000B
:10B3C000F2540200000000008005780001067800B9
:10B3D0000B0078008C00780012D02C00431F240052
:10B3E000D02D020000000000B65402000000000052
:10B3F0000080540081005D00A05D8800B15D880080
:10B40000845D80006E20E10002003A00B20BE20091
:10B4100005003200845D80006F20E10006003A00E4
:10B42000B20BE20004003A0014002000C45D880062
:10B43000BA2BEF0002003700B82BEF00BA2BEF0059
:10B44000205D8000B80BB400D45D8000335D8000C7
:10B4500084804900405D8800515D8800845D8000E3
:10B46000E1025200945D800060035A00C05D8000DC
:10B47000D15D8000C2002000030020004055020082
:10B480000000000000805200E05D880001005B00C9
:10B49000F05D8800C4762000435D80000480410098
:10B4A000405D8800545D800060024A00545D880061
:10B4B00020002000A00BB4008002780000002000D3
:10B4C000A28BB4000003780054132D0004805200B6
:10B4D000605D880060005B00705D88007400200083
:10B4E000446388006A2CEF00AC0BF800640CF90090
:10B4F000AE0BF800660CF9000656020000000000D2
:10B50000E0628800F16288000263880013638800AB
:10B510000463800061024200045E880014638000BE
:10B5200060024A00145E8800045E80006120E10031
:10B530000D003A00C20BE2000B003A0002002000AE
:10B5400081BC20000200780004140200000000000A
:10B55000805878000201E8000004E0004220AE00BC
:10B56000F8FF37005F003700045E80006220E100D2
:10B570000D003A00C20BE2000B003A00020020006E
:10B5800081BC2000020078001414020000000000BA
:10B59000805878000201E8000004E0004220AE007C
:10B5A000F8FF37004F003700045E80006320E100A1
:10B5B0000D003A00C20BE2000B003A00020020002E
:10B5C00081BC20000200780024140200000000006A
:10B5D000805878000201E8000004E0004220AE003C
:10B5E000F8FF37003F003700045E80006420E10070
:10B5F0000D003A00C20BE2000B003A0002002000EE
:10B6000081BC200002007800341402000000000019
:10B61000805878000201E8000004E0004220AE00FB
:10B62000F8FF37002F003700045E80006520E1003E
:10B630000D003A00C20BE2000B003A0002002000AD
:10B6400081BC2000020078004414020000000000C9
:10B65000805878000201E8000004E0004220AE00BB
:10B66000F8FF37001F003700045E80006620E1000D
:10B670000D003A00C20BE2000B003A00020020006D
:10B6800081BC200002007800541402000000000079
:10B69000805878000201E8000004E0004220AE007B
:10B6A000F8FF37000F003700045E80006720E100DC
:10B6B0000C003A00C20BE2000A003A00020020002F
:10B6C00081BC200002007800641402000000000029
:10B6D000805878000201E8000004E0004220AE003B
:10B6E000F8FF3700E45D80006120E1000D003A00C2
:10B6F000BE0BE2000B003A0002002000C1BC20009B
:10B7000002007800741402000000000080587800E5
:10B710000201E8000004E0004220AE00F8FF37001C
:10B72000AF003700E45D80006220E1000D003A00C8
:10B73000BE0BE2000B003A0002002000C1BC20005A
:10B740000200780084140200000000008058780095
:10B750000201E8000004E0004220AE00F8FF3700DC
:10B760009F003700E45D80006320E1000D003A0097
:10B77000BE0BE2000B003A0002002000C1BC20001A
:10B780000200780094140200000000008058780045
:10B790000201E8000004E0004220AE00F8FF37009C
:10B7A0008F003700E45D80006420E1000D003A0066
:10B7B000BE0BE2000B003A0002002000C1BC2000DA
:10B7C00002007800A41402000000000080587800F5
:10B7D0000201E8000004E0004220AE00F8FF37005C
:10B7E0007F003700E45D80006520E1000D003A0035
:10B7F000BE0BE2000B003A0002002000C1BC20009A
:10B8000002007800B41402000000000080587800A4
:10B810000201E8000004E0004220AE00F8FF37001B
:10B820006F003700E45D80006620E1000D003A0003
:10B83000BE0BE2000B003A0002002000C1BC200059
:10B8400002007800C4140200000000008058780054
:10B850000201E8000004E0004220AE00F8FF3700DB
:10B860005F003700E45D80006720E1000D003A00D2
:10B87000BE0BE2000B003A0002002000C1BC200019
:10B8800002007800D4140200000000008058780004
:10B890000201E8000004E0004220AE00F8FF37009B
:10B8A0004F003700E45D80006820E1000D003A00A1
:10B8B000BE0BE2000B003A0002002000C1BC2000D9
:10B8C00002007800E41402000000000080587800B4
:10B8D0000201E8000004E0004220AE00F8FF37005B
:10B8E0003F003700E45D80006920E1000D003A0070
:10B8F000BE0BE2000B003A0002002000C1BC200099
:10B9000002007800F4140200000000008058780063
:10B910000201E8000004E0004220AE00F8FF37001A
:10B920002F003700E45D80006A20E1000D003A003E
:10B93000BE0BE2000B003A0002002000C1BC200058
:10B940000200780004150200000000008058780012
:10B950000201E8000004E0004220AE00F8FF3700DA
:10B960001F003700E45D80006B20E1000D003A000D
:10B97000BE0BE2000B003A0002002000C1BC200018
:10B9800002007800141502000000000080587800C2
:10B990000201E8000004E0004220AE00F8FF37009A
:10B9A0000F003700E45D80006C20E1000C003A00DD
:10B9B000BE0BE2000A003A0002002000C1BC2000D9
:10B9C0000200780024150200000000008058780072
:10B9D0000201E8000004E0004220AE00F8FF37005A
:10B9E000545D80006020E1000F00390004003E003B
:10B9F000445D8000837D20000418E1000A003E00C1
:10BA0000545D80006020E10007003E000400390022
:10BA1000445D8000238020000418E100020039000A
:10BA200010C0B300C7EBB7001A013700844C800088
:10BA30004822DE006A24E10004003200844C8000C9
:10BA40004822DE006B24E10050003A000040EB0089
:10BA50000628AF000000E8006204E1002100390080
:10BA6000844C80004822DE006A24E1000D003A0088
:10BA70003322AF00FEFF370004032000A41188002A
:10BA80003322AF00FEFF370014042000A411880009
:10BA90003322AF00FEFF370004022000A41188000B
:10BAA00010003700844C80004822DE006B24E10047
:10BAB0000C003A003322AF00FEFF370004032000E1
:10BAC000A41188003322AF00FEFF370024042000B9
:10BAD000A41188003322AF00FEFF370004022000CB
:10BAE000A4118800D04B8000E3026000054078007C
:10BAF00092E9B7009269D400944C80006142420000
:10BB00000440780000E0B7000080FB00449920006A
:10BB100004034000F04B8000F00FB200004B7800AF
:10BB2000944C80000960EF0043992000830242009A
:10BB30007FC9BF00000378000D60EF0006007800A9
:10BB4000F00FB200804A78008D69EF008E69EF0037
:10BB5000004020007A09B6008002780004402000EE
:10BB60000520E10002003A0010C0B3008DE9B700E3
:10BB7000D04B8000F00260007028E10002003A0023
:10BB800010C0B3008EE9B700C2003700844C8000BB
:10BB90004822DE00A4C2B20072003A00D04B8000FE
:10BBA000F00260007028E10003003A0010C0B3000A
:10BBB0009DE9B700010037009D69EF00D04B800080
:10BBC000EF0260000540780093E9B7009369D40064
:10BBD0009369D4009D49E2002F003A00944C800004
:10BBE0004822DE00634242000440780000E0B700D3
:10BBF0000080FB00E499200004034000F04B80002B
:10BC0000F00FB200004B7800944C80004822DE0018
:10BC1000624242000440780000E0B7000080FB0070
:10BC2000E4992000040340007FC9BF00800378002E
:10BC30000F60EF0007007800F00FB200004B7800B3
:10BC4000944C80004822DE006142420004407800AB
:10BC500000E0B7000080FB00E499200004034000EE
:10BC6000E04B8000F00FB200004B7800944C800055
:10BC70004822DE00E3992000830242007DC9BF0014
:10BC8000000378000D60EF0006007800F00FB200AE
:10BC9000804A780032003700E44C80004822DE0001
:10BCA0006124E1002E003A00944C80004822DE001E
:10BCB000634242000440780000E0B7000080FB00CF
:10BCC00004A2200004034000F04B8000F00FB200FB
:10BCD000004B7800944C80004822DE006242420013
:10BCE0000440780000E0B7000080FB0004A22000C0
:10BCF000040340007FC9BF00800378000F60EF009D
:10BD000007007800F00FB200004B7800944C8000E0
:10BD10004822DE00614242000440780000E0B700A3
:10BD20000080FB0004A2200004034000E04B8000E0
:10BD3000F00FB200004B7800944C80004822DE00E7
:10BD400003A22000830242007DC9BF0000037800E7
:10BD50000D60EF0006007800F00FB200804A780016
:10BD60004C003700844C80004822DE00A4C3B2009F
:10BD700015003A007DE9AE000100370045003700AC
:10BD80007DC9AF0007003700E54B8000C62ADE0002
:10BD900005027800F443B200044078007DE8B70063
:10BDA000080037007DC9AE0006003700E54B800073
:10BDB000C62ADE0005027800F443B2000440780091
:10BDC0007EE8B70033003700844C80004822DE0054
:10BDD000A4C8B2002F003A0010C0B3008FE9B7002A
:10BDE0007A09F8001A08F9007C09F8001C08F90023
:10BDF0007E09F8001E08F9000648A9001A88AF005D
:10BE00000648A8000668A9001A68AF000668A800DE
:10BE1000D04080006740600020E8B70000002400A8
:10BE20001C08B60080027800040024000520E10010
:10BE300002003A0006A8A8000100370006A8A900E1
:10BE4000000028001C08B6008002780004002800CA
:10BE50000520E10002003A000688A8000100370032
:10BE60000688A9001C08F8002408F900F07F2000CB
:10BE70002428B600E5408000CB2ADE0067C06200BF
:10BE800021E8B7001E08F8002208F90070560200E9
:10BE9000000000008501200006000900CF12780094
:10BEA000CF02780000000600851F78005F69EF0070
:10BEB000844B80004822DE007024E1000700390036
:10BEC000AA320200000000000004E00002003A0074
:10BED0007169EF00010037001F0037006429D400AA
:10BEE00066A9D60063E9AE00010037006409A80026
:10BEF0006229D4006409F8007209F900344B80000B
:10BF0000F43FB200A44B88007169EC0004012000EA
:10BF1000834B8000C819DE00034052005FE9B70080
:10BF20006209F8006809F9006A29EF00844B800073
:10BF30004822DE000960EF000402E8000402E90084
:10BF4000030032006A29D50068A9D700FBFF37003B
:10BF50006C29EF006E29EF00CF0278000000060088
:10BF6000851F78008509AE0018003700A400200066
:10BF7000904B8000A14B80000402E8000402E9001D
:10BF8000030032008100D1000080D300FBFF3700A6
:10BF9000B04B8800F453020000000000044C800005
:10BFA0004822DE006424E10003003A001858020031
:10BFB000000000009E2BEF004C3302000000000048
:10BFC0001E340200000000000C0037008509AF009D
:10BFD0000A0037009E2BEC00F45C8000439C20009C
:10BFE0000418E10001003C009E2BEF00545F0200AA
:10BFF000000000001E34020000000000CF027800A4
:10C0000000000600851F7800C50020000700090019
:10C01000B51F78000900E000130032002800FA0084
:10C02000680220000006EB000C377C000884E90061
:10C03000FDFF3B0039179800470224000003EB0086
:10C040006022B80029179800470224000003EB0083
:10C050006022B800F835020000000000AE14900025
:10C060008904E900F7FF3A00D71C240056D62C00BB
:10C070006022B800000F9800110F9800220F98005E
:10C08000330F980003F0A100063702000000000003
:10C090004200AE000E0037000E0890009E0890008F
:10C0A0002E099000BE099000A800200008179800F3
:10C0B000A5B9230004A02C006033B800440F9800F9
:10C0C000550F9800660F9800770F98000E00370004
:10C0D0000E0890009E0890002E099000BE09900066
:10C0E000480120000817980004002000859E2800C1
:10C0F0004630220077AC2800440F9800550F980076
:10C10000660F9800770F98000005780003F0A700ED
:10C110004D0037000A00780003F0A1008A370200C2
:10C12000000000009E1490008004EB001917980096
:10C130004E0A9000DE0A90006E0B9000FE0B9000FD
:10C140009E169000E0370200000000009E1690004E
:10C150000D00A7002C003700080F9800190F980059
:10C160002A0F9800310F98009E1690000D00A20033
:10C170001D1798009E1690000D10A70006003700AE
:10C180009E1690000000E000130032009E16900002
:10C190000D10A0001D1798000E129000BE16900002
:10C1A000800278000D20E10005003A003D1798005C
:10C1B0003322AF00FEFF3700E4022000A411880004
:10C1C0003D179800050078000003B0003322AF004F
:10C1D000FEFF3700A01188008E1690008D06E90042
:10C1E0001E0032000D1798004E089000DE089000E7
:10C1F0006E099000FE099000A40020008002EB0070
:10C200006033B800CEFF3700400F9800510F980000
:10C21000620F9800730F9800000278008102780086
:10C2200002037800830378000E0890009E089000B7
:10C230002E099000BE0990009E1690000D00A200ED
:10C240001D179800BEFF37003322AF00FEFF3700F6
:10C25000D4022000A4118800AFFF370000000000C6
:10C260000080FA00A501200007000900CF12780025
:10C27000CF02780000000600851F7800100CF8003F
:10C280003208F9000100200001007800FE1D0200C4
:10C29000000000008100E8003322AF00FEFF3700FD
:10C2A000A0118800F00020000008E600F6FF37002B
:10C2B00027C8BF000160EF0004002000C82402006E
:10C2C000000000002101200001007800FE1D020096
:10C2D000000000008100E8003322AF00FEFF3700BD
:10C2E000A0118800500120000008E600F6FF37008A
:10C2F0000100200001007800221E02000000000062
:10C300008100E8003322AF00FEFF3700A011880053
:10C31000700020000008E600F6FF37000000200053
:10C320004140800052408000BC3502000000000007
:10C330002900200002600200000000003322AF004C
:10C34000FEFF370004022000A41188000100200035
:10C35000010078003E1E0200000000008100E8009D
:10C360003322AF00FEFF3700A011880060002000DC
:10C370000008E600F6FF370080608000040020001F
:10C38000C8240200000000003322AF00FEFF370087
:10C3900004022000A411880027C8BF000160EF003C
:10C3A0004400DD002CE8B70032C8BF002FE8B7001A
:10C3B00033C8BF0032E8B7003368EF0032C8BF00AF
:10C3C0002EE8B7002CC8BF001CEDB7001D6DEF00B4
:10C3D0002EC8BF001EEDB700362B02000000000083
:10C3E0006441800061424200044078000AE0B700E6
:10C3F000054078001CEDB7001D6DEF002FC8BF0091
:10C400001EEDB700362B02000000000064418000E2
:10C410006A424200044078000AE0B7000540780014
:10C420001CEDB7001D6DEF000FCCBF001EEDB70077
:10C43000362B02000000000000C5B30028E8B7005A
:10C440000F4CE200CD003A004300A90040408000BC
:10C4500051408000F226210033B02300F62E020066
:10C460000000000080027800010378000100200035
:10C47000010078005A160200000000008100E80068
:10C480003322AF00FEFF3700A011880050002000CB
:10C490000008E600F6FF3700000020008500780065
:10C4A00006017800BC3502000000000029002000D1
:10C4B0007438020000000000B10020000100780084
:10C4C0005A160200000000008100E8003322AF008D
:10C4D000FEFF3700A0118800E00020000008E60001
:10C4E000F6FF37003A6DEF003B6DEF00A62002002B
:10C4F000000000006029EF004300A90040408000D8
:10C5000051408000F226210033A82300F62E0200BD
:10C510000000000080027800010378000500780028
:10C520008600780002002000832C24008E2E02005A
:10C5300000000000330039004300A90040408000A3
:10C5400051408000F226210033B02300F62E020075
:10C550000000000080027800010378000000200045
:10C560008500780006017800BC350200000000005C
:10C5700029002000A63A02000000000070C2B300AB
:10C580003AEDB70020C0B3003BEDB700A620020093
:10C590000000000000CEB3003AEDB700CC2002004E
:10C5A0000000000000CEB3003AEDB700CC2002003E
:10C5B0000000000000CEB3003AEDB700CC2002002E
:10C5C00000000000B0C3B3003AEDB70020C0B300D4
:10C5D0003BEDB700A6200200000000003A6DEF001E
:10C5E000CC200200000000003A6DEF00CC200200D9
:10C5F000000000003A6DEF00CC20020000000000B7
:10C60000320037004300A9004040800051408000C4
:10C61000F226210033B02300F62E020000000000B5
:10C620008002780001037800000020008500780077
:10C6300006017800BC35020000000000190020004F
:10C64000A63A02000000000070C2B3003AEDB70045
:10C6500020C0B3003BEDB700A620020000000000A0
:10C660003A6DEF00CC200200000000003A6DEF00B0
:10C67000CC200200000000003A6DEF00CC20020048
:10C6800000000000B0C3B3003AEDB70020C0B30013
:10C690003BEDB700A62002000000000000CEB30072
:10C6A0003AEDB700CC2002000000000000CEB3003D
:10C6B0003AEDB700CC2002000000000000CEB3002D
:10C6C0003AEDB700CC2002000000000030C0B300FB
:10C6D00030EDB7002E240200000000003A6DEF009C
:10C6E00030C0B3003BEDB700A62002000000000000
:10C6F00006E8A90005002000050078007616020073
:10C70000000000000040B3004220AF0005003700E9
:10C710008502E80036EDB700242402000000000086
:10C72000F5FF370028C8BF0036EDB700242402000B
:10C730000000000027C8BF00800278000B60EF00F7
:10C740000600200005007800860078000400200024
:10C75000E22B02000000000000C2B30036EDB7007B
:10C76000242402000000000000C2B30036EDB70030
:10C7700024240200000000003604370074608000AA
:10C780004822DE006124E10094003A00010020000C
:10C790000100780086160200000000008100E80019
:10C7A0003322AF00FEFF3700A011880030002000C8
:10C7B0000008E600F6FF370000002000414080003E
:10C7C00052408000BC35020000000000290020001B
:10C7D0007438020000000000910020000100780081
:10C7E00086160200000000008100E8003322AF003E
:10C7F000FEFF3700A0118800C00020000008E600FE
:10C80000F6FF37003A6DEF003B6DEF00A620020007
:10C81000000000006029EF004300A90040408000B4
:10C8200051408000F226210033A82300F62E02009A
:10C830000000000080027800010378000000200062
:10C840008500780006017800BC3502000000000079
:10C8500019002000A63A02000000000070C2B300D8
:10C860003AEDB70020C0B3003BEDB700A6200200B0
:10C87000000000003A6DEF00CC2002000000000034
:10C880003A6DEF00CC200200000000003A6DEF008E
:10C89000CC20020000000000B0C3B3003AEDB700A6
:10C8A00020C0B3003BEDB700A6200200000000004E
:10C8B00000CEB3003AEDB700CC200200000000002B
:10C8C00000CEB3003AEDB700CC200200000000001B
:10C8D00000CEB3003AEDB700CC200200000000000B
:10C8E00030C0B30030EDB7002E240200000000007D
:10C8F0003A6DEF0030C0B3003BEDB700A620020058
:10C900000000000006E8A9000500200005007800EE
:10C91000A0160200000000000040B3004220AF005B
:10C92000050037008502E80036EDB7002424020038
:10C9300000000000F5FF370028C8BF0036EDB70043
:10C94000242402000000000027C8BF0080027800F5
:10C950000B60EF00060020000500780086007800DC
:10C9600004002000E22B02000000000000C2B3001F
:10C9700036EDB700242402000000000000C2B3001E
:10C9800036EDB700242402000000000010C4B300FC
:10C990003AEDB70030C0B3003BEDB700A62002006F
:10C9A0000000000006E8A90005002000050078004E
:10C9B000B0160200000000000040B3004220AF00AB
:10C9C000050037008502E80036EDB7002424020098
:10C9D00000000000F5FF37009E0337007460800000
:10C9E0004822DE006224E10094003A0001002000A9
:10C9F00001007800C0160200000000008100E8007D
:10CA00003322AF00FEFF3700A01188003000200065
:10CA10000008E600F6FF37000000200041408000DB
:10CA200052408000BC3502000000000029002000B8
:10CA3000743802000000000091002000010078001E
:10CA4000C0160200000000008100E8003322AF00A1
:10CA5000FEFF3700A0118800C00020000008E6009B
:10CA6000F6FF37003A6DEF003B6DEF00A6200200A5
:10CA7000000000006029EF004300A9004040800052
:10CA800051408000F226210033A82300F62E020038
:10CA90000000000080027800010378000000200000
:10CAA0008500780006017800BC3502000000000017
:10CAB00019002000A63A02000000000070C2B30076
:10CAC0003AEDB70020C0B3003BEDB700A62002004E
:10CAD000000000003A6DEF00CC20020000000000D2
:10CAE0003A6DEF00CC200200000000003A6DEF002C
:10CAF000CC20020000000000B0C3B3003AEDB70044
:10CB000020C0B3003BEDB700A620020000000000EB
:10CB100000CEB3003AEDB700CC20020000000000C8
:10CB200000CEB3003AEDB700CC20020000000000B8
:10CB300000CEB3003AEDB700CC20020000000000A8
:10CB400030C0B30030EDB7002E240200000000001A
:10CB50003A6DEF0030C0B3003BEDB700A6200200F5
:10CB60000000000006E8A90005002000050078008C
:10CB7000DA160200000000000040B3004220AF00BF
:10CB8000050037008502E80036EDB70024240200D6
:10CB900000000000F5FF370028C8BF0036EDB700E1
:10CBA000242402000000000027C8BF008002780093
:10CBB0000B60EF000600200005007800860078007A
:10CBC00004002000E22B02000000000000C2B300BD
:10CBD00036EDB700242402000000000000C2B300BC
:10CBE00036EDB700242402000000000010C4B3009A
:10CBF0003AEDB70030C0B3003BEDB700A62002000D
:10CC00000000000006E8A9000500200005007800EB
:10CC1000B0160200000000000040B3004220AF0048
:10CC2000050037008502E80036EDB7002424020035
:10CC300000000000F5FF3700060337007460800035
:10CC40004822DE006324E10099003A000100200040
:10CC500001007800EA160200000000008100E800F0
:10CC60003322AF00FEFF3700A011880040002000F3
:10CC70000008E600F6FF3700000020004140800079
:10CC800052408000BC350200000000002900200056
:10CC90007438020000000000A100200001007800AC
:10CCA000EA160200000000008100E8003322AF0015
:10CCB000FEFF3700A0118800D00020000008E60029
:10CCC000F6FF37003A6DEF003B6DEF00A620020043
:10CCD000000000006029EF004300A90040408000F0
:10CCE00051408000F226210033A82300F62E0200D6
:10CCF0000000000080027800010378000500780041
:10CD00008600780002002000031224008030020018
:10CD1000000000008003780001047800000020007B
:10CD20008700780008017800BC3502000000000090
:10CD300019002000A63A02000000000070C2B300F3
:10CD40003AEDB70020C0B3003BEDB700A6200200CB
:10CD5000000000003A6DEF00CC200200000000004F
:10CD60003A6DEF00CC200200000000003A6DEF00A9
:10CD7000CC20020000000000B0C3B3003AEDB700C1
:10CD800020C0B3003BEDB700A62002000000000069
:10CD90003A6DEF00CC200200000000003A6DEF0079
:10CDA000CC200200000000003A6DEF00CC20020011
:10CDB0000000000030C0B30030EDB7002E240200A8
:10CDC000000000003A6DEF0030C0B3003BEDB7004B
:10CDD000A62002000000000006E8A90005002000CF
:10CDE0000500780006170200000000000040B300B4
:10CDF0004220AF00050037008502E80036EDB7009D
:10CE00002424020000000000F5FF370028C8BF00FE
:10CE100036EDB700242402000000000027C8BF0040
:10CE2000800278000B60EF0006002000050078000B
:10CE30008600780004002000E22B020000000000C1
:10CE400000C2B30036EDB700242402000000000049
:10CE500000C2B30036EDB700242402000000000039
:10CE600010C4B3003AEDB70030C0B3003BEDB700DB
:10CE7000A62002000000000006E8A900050020002E
:10CE800005007800B0160200000000000040B3006A
:10CE90004220AF00050037008502E80036EDB700FC
:10CEA0002424020000000000F5FF3700690237006B
:10CEB000746080004822DE006424E10026013A000C
:10CEC0000100200001007800181702000000000097
:10CED0008100E8003322AF00FEFF3700A011880078
:10CEE000400020000008E600F6FF370000002000A8
:10CEF0004140800052408000BC350200000000002C
:10CF0000290020007438020000000000A100200069
:10CF10000100780018170200000000008100E800FE
:10CF20003322AF00FEFF3700A0118800D0002000A0
:10CF30000008E600F6FF37004040800051408000C6
:10CF400002002400C36124008E2E020000000000B5
:10CF50007B0039003A6DEF003B6DEF00A620020028
:10CF6000000000006029EF004300A900404080005D
:10CF700051408000F226210033A82300F62E020043
:10CF800000000000800278000103780005007800AE
:10CF90008600780002002000031224008030020086
:10CFA00000000000800378000104780000002000E9
:10CFB0008700780008017800BC35020000000000FE
:10CFC00019002000A63A02000000000070C2B30061
:10CFD0003AEDB70020C0B3003BEDB700A620020039
:10CFE000000000003A6DEF00CC20020000000000BD
:10CFF0003A6DEF00CC200200000000003A6DEF0017
:10D00000CC20020000000000B0C3B3003AEDB7002E
:10D0100020C0B3003BEDB700A620020000000000D6
:10D020003A6DEF00CC200200000000003A6DEF00E6
:10D03000CC200200000000003A6DEF00CC2002007E
:10D040000000000030C0B30030EDB7002E24020015
:10D05000000000003A6DEF0030C0B3003BEDB700B8
:10D06000A62002000000000006E8A900050020003C
:10D070000500780034170200000000000040B300F3
:10D080004220AF00050037008502E80036EDB7000A
:10D090002424020000000000F5FF370028C8BF006C
:10D0A00036EDB700242402000000000027C8BF00AE
:10D0B000800278000B60EF00060020000500780079
:10D0C0008600780004002000E22B0200000000002F
:10D0D00000C2B30036EDB7002424020000000000B7
:10D0E00000C2B30036EDB7002424020000000000A7
:10D0F00010C4B3003AEDB70030C0B3003BEDB70049
:10D10000A62002000000000006E8A900050020009B
:10D1100005007800B0160200000000000040B300D7
:10D120004220AF00050037008502E80036EDB70069
:10D130002424020000000000F5FF370085003700BE
:10D1400000002400C1612400424080005340800060
:10D150008E2E020000000000010031007D003A0028
:10D160003A6DEF003B6DEF00A620020000000000CA
:10D170006029EF004300A90040408000514080003A
:10D18000F226210033A82300F62E02000000000042
:10D19000800278000103780005007800860078009E
:10D1A00002002000A347240080300200000000009D
:10D1B00080037800010478000000200087007800D8
:10D1C00008017800BC3502000000000029002000A2
:10D1D000A63A02000000000070C2B3003AEDB700AA
:10D1E00020C0B3003BEDB700A62002000000000005
:10D1F00000CEB3003AEDB700CC20020000000000E2
:10D2000000CEB3003AEDB700CC20020000000000D1
:10D2100000CEB3003AEDB700CC20020000000000C1
:10D22000B0C3B3003AEDB70020C0B3003BEDB70088
:10D23000A6200200000000003A6DEF00CC200200A2
:10D24000000000003A6DEF00CC200200000000005A
:10D250003A6DEF00CC2002000000000030C0B300A7
:10D2600030EDB7002E240200000000003A6DEF0000
:10D2700030C0B3003BEDB700A62002000000000064
:10D2800006E8A90005002000050078003417020018
:10D29000000000000040B3004220AF00050037004E
:10D2A0008502E80036EDB7002424020000000000EB
:10D2B000F5FF370028C8BF0036EDB7002424020070
:10D2C0000000000027C8BF00800278000B60EF005C
:10D2D0000600200005007800860078000400200089
:10D2E000E22B02000000000000C2B30036EDB700E0
:10D2F000242402000000000000C2B30036EDB70095
:10D30000242402000000000010C4B3003AEDB7006E
:10D3100030C0B3003BEDB700A620020000000000C3
:10D3200006E8A90005002000050078004617020065
:10D33000000000000040B3004220AF0005003700AD
:10D340008502E80036EDB70024240200000000004A
:10D35000F5FF37003F013700746080004822DE008F
:10D360006524E1009C003A000100200001007800E3
:10D3700056170200000000008100E8003322AF00D1
:10D38000FEFF3700A0118800400020000008E600E2
:10D39000F6FF37000000200041408000524080002E
:10D3A000BC35020000000000290020007438020093
:10D3B00000000000A10020000100780056170200C4
:10D3C000000000008100E8003322AF00FEFF3700BC
:10D3D000A0118800D00020000008E600F6FF37000A
:10D3E0003A6DEF003B6DEF00A62002000000000048
:10D3F0006029EF004300A9004040800051408000B8
:10D40000F226210033A82300F62E020000000000BF
:10D41000800278000103780005007800860078001B
:10D4200002002000A347240080300200000000001A
:10D430008003780001047800000020008700780055
:10D4400008017800BC35020000000000290020001F
:10D45000A63A02000000000070C2B3003AEDB70027
:10D4600020C0B3003BEDB700A62002000000000082
:10D4700000CEB3003AEDB700CC200200000000005F
:10D4800000CEB3003AEDB700CC200200000000004F
:10D4900000CEB3003AEDB700CC200200000000003F
:10D4A000B0C3B3003AEDB70020C0B3003BEDB70006
:10D4B000A6200200000000003A6DEF00CC20020020
:10D4C000000000003A6DEF00CC20020000000000D8
:10D4D0003A6DEF00CC2002000000000030C0B30025
:10D4E00030EDB7002E240200000000003A6DEF007E
:10D4F00030C0B3003BEDB700A620020000000000E2
:10D5000006E8A90005002000050078007217020057
:10D51000000000000040B3004220AF0005003700CB
:10D520008502E80036EDB700242402000000000068
:10D53000F5FF370028C8BF0036EDB70024240200ED
:10D540000000000027C8BF00800278000B60EF00D9
:10D550000600200005007800860078000400200006
:10D56000E22B02000000000000C2B30036EDB7005D
:10D57000242402000000000000C2B30036EDB70012
:10D58000242402000000000010C4B3003AEDB700EC
:10D5900030C0B3003BEDB700A62002000000000041
:10D5A00006E8A900050020000500780046170200E3
:10D5B000000000000040B3004220AF00050037002B
:10D5C0008502E80036EDB7002424020000000000C8
:10D5D000F5FF37009F003700746080004822DE00AE
:10D5E0006624E1009B003A00010020000100780061
:10D5F00084170200000000008100E8003322AF0021
:10D60000FEFF3700A0118800400020000008E6005F
:10D61000F6FF3700000020004140800052408000AB
:10D62000BC35020000000000290020007438020010
:10D6300000000000A1002000010078008417020013
:10D64000000000008100E8003322AF00FEFF370039
:10D65000A0118800D00020000008E600F6FF370087
:10D660003A6DEF003B6DEF00A620020000000000C5
:10D670006029EF004300A900404080005140800035
:10D68000F226210033A82300F62E0200000000003D
:10D690008002780001037800050078008600780099
:10D6A00002002000A3472400803002000000000098
:10D6B00080037800010478000000200087007800D3
:10D6C00008017800BC35020000000000290020009D
:10D6D000A63A02000000000070C2B3003AEDB700A5
:10D6E00020C0B3003BEDB700A62002000000000000
:10D6F00000CEB3003AEDB700CC20020000000000DD
:10D7000000CEB3003AEDB700CC20020000000000CC
:10D7100000CEB3003AEDB700CC20020000000000BC
:10D72000B0C3B3003AEDB70020C0B3003BEDB70083
:10D73000A6200200000000003A6DEF00CC2002009D
:10D74000000000003A6DEF00CC2002000000000055
:10D750003A6DEF00CC2002000000000030C0B300A2
:10D7600030EDB7002E240200000000003A6DEF00FB
:10D7700030C0B3003BEDB700A6200200000000005F
:10D7800006E8A9000500200005007800A0170200A7
:10D79000000000000040B3004220AF000500370049
:10D7A0008502E80036EDB7002424020000000000E6
:10D7B000F5FF370028C8BF0036EDB700242402006B
:10D7C0000000000027C8BF00800278000B60EF0057
:10D7D0000600200005007800860078000400200084
:10D7E000E22B02000000000000C2B30036EDB700DB
:10D7F000242402000000000000C2B30036EDB70090
:10D80000242402000000000010C4B3003AEDB70069
:10D8100030C0B3003BEDB700A620020000000000BE
:10D8200006E8A90005002000050078004617020060
:10D83000000000000040B3004220AF0005003700A8
:10D840008502E80036EDB700242402000000000045
:10D85000F5FF3700CF02780000000600851F780032
:10D86000C500200003000900B51F78000202B800BF
:10D870000303B8004200A9008502430060844B0006
:10D88000020BB80085024B0008844B00030BB80064
:10D89000080443000780B000870178000801780081
:10D8A00085007800040078002501200003000900AD
:10D8B000CF127800CF02780000000600851F7800A4
:10D8C000C500200003000900B51F780000027800A1
:10D8D0008102780002037800830378000000EB00E7
:10D8E0008000EB000001EB008001EB000800A100CC
:10D8F00007F0A600050037000A00A0000402EA00B5
:10D900008582EA000683EA008783EA0085046A00CC
:10D9100002003A0087046B001500320039472000EE
:10D920000340A7000B0037004200A9000482D20088
:10D930008582D2000683D2008783D2000080D20085
:10D940008180D2000281D2008381D2008904E90063
:10D95000F3FF3A00C44CDD004200A90009F0A10029
:10D960000340A10083816C000A00A70003F0A0001F
:10D970002501200003000900CF127800CF027800B3
:10D98000000006005D4CE20020003A005E0CF8004A
:10D99000600CF900622CEF000063800011638000CE
:10D9A00002352C00030020002E6C02000000000055
:10D9B000006388001163880004638000034E240024
:10D9C000030052000063880014638000348AB100B1
:10D9D0001463880000638000116380007E5402009D
:10D9E00000000000C0608800D1608800C060800036
:10D9F000D160800002402200439724008030020062
:10DA000000000000E0608800F1608800E4628000AF
:10DA10004822DE006124E10004003200E46280005C
:10DA20004822DE006224E10020003A005E0CF8008B
:10DA3000600CF900622CEF0000638000116380002D
:10DA4000823E2000030020002E6C02000000000037
:10DA5000006388001163880004638000034E240083
:10DA6000030052000063880014638000348AB10010
:10DA70001463880000638000116380007E540200FC
:10DA800000000000C0608800D1608800C060800095
:10DA9000D160800002002000A347240080300200F3
:10DAA00000000000E0608800F1608800E46280000F
:10DAB0004822DE006324E10020003A005E0CF800FA
:10DAC000600CF900622CEF0000638000116380009D
:10DAD00012272000030020002E6C0200000000002E
:10DAE000006388001163880004638000034E2400F3
:10DAF000030052000063880014638000348AB10080
:10DB00001463880000638000116380007E5402006B
:10DB100000000000C0608800D1608800C060800004
:10DB2000D160800002002000A34724008030020062
:10DB300000000000E0608800F1608800E46280007E
:10DB40004822DE006424E10020003A005E0CF80068
:10DB5000600CF900622CEF0000638000116380000C
:10DB6000823E2000030020002E6C02000000000016
:10DB7000006388001163880004638000034E240062
:10DB8000030052000063880014638000348AB100EF
:10DB90001463880000638000116380007E540200DB
:10DBA00000000000C0608800D1608800C060800074
:10DBB000D160800002002000A347240080300200D2
:10DBC00000000000E0608800F1608800E4628000EE
:10DBD0004822DE006524E10020003A005E0CF800D7
:10DBE000600CF900622CEF0000638000116380007C
:10DBF000224E2000030020002E6C020000000000D6
:10DC0000006388001163880004638000034E2400D1
:10DC1000030052000063880014638000348AB1005E
:10DC20001463880000638000116380007E5402004A
:10DC300000000000C0608800D1608800C0608000E3
:10DC4000D160800002002000A34724008030020041
:10DC500000000000E0608800F1608800E46280005D
:10DC60004822DE006624E10028003A005E0CF8003D
:10DC7000600CF900622CEF000063800011638000EB
:10DC800002002000030020005E6C02000000000083
:10DC900054752E00C5AA2A00A6AA2000A7092400B0
:10DCA000F8350200000000008A3702000000000082
:10DCB000006388001163880004638000034E240021
:10DCC000030052000063880014638000348AB100AE
:10DCD0001463880000638000116380007E5402009A
:10DCE00000000000C0608800D1608800C060800033
:10DCF000D160800002002000A34724008030020091
:10DD000000000000E0608800F16088005DCCBF008A
:10DD100030EDB7005E0CF800320DF90076310200EC
:10DD2000000000005DCCBF000FECB7001C0CF80039
:10DD30000808F9001E0CF8000A08F9005E0CF8004B
:10DD4000100CF9000F4CE20002003A00A834020067
:10DD5000000000000F4CE200CD003A004300A90093
:10DD60004040800051408000F226210033B0230063
:10DD7000F62E020000000000800278000103780007
:10DD800001002000010078005A1602000000000087
:10DD90008100E8003322AF00FEFF3700A0118800A9
:10DDA000500020000008E600F6FF370000002000C9
:10DDB0008500780006017800BC35020000000000F4
:10DDC000290020007438020000000000B10020008B
:10DDD000010078005A160200000000008100E800EF
:10DDE0003322AF00FEFF3700A0118800E0002000C2
:10DDF0000008E600F6FF37003A6DEF003B6DEF00DC
:10DE0000A6200200000000006029EF004300A900E6
:10DE10004040800051408000F226210033A82300BA
:10DE2000F62E020000000000800278000103780056
:10DE3000050078008600780002002000832C240072
:10DE40008E2E020000000000330039004300A900BC
:10DE50004040800051408000F226210033B0230072
:10DE6000F62E020000000000800278000103780016
:10DE7000000020008500780006017800BC35020013
:10DE80000000000029002000A63A02000000000067
:10DE900070C2B3003AEDB70020C0B3003BEDB7004D
:10DEA000A62002000000000000CEB3003AEDB7004B
:10DEB000CC2002000000000000CEB3003AEDB70015
:10DEC000CC2002000000000000CEB3003AEDB70005
:10DED000CC20020000000000B0C3B3003AEDB70050
:10DEE00020C0B3003BEDB700A620020000000000F8
:10DEF0003A6DEF00CC200200000000003A6DEF0008
:10DF0000CC200200000000003A6DEF00CC2002009F
:10DF100000000000320037004300A90040408000AC
:10DF200051408000F226210033B02300F62E02007B
:10DF3000000000008002780001037800000020004B
:10DF40008500780006017800BC3502000000000062
:10DF500019002000A63A02000000000070C2B300C1
:10DF60003AEDB70020C0B3003BEDB700A620020099
:10DF7000000000003A6DEF00CC200200000000001D
:10DF80003A6DEF00CC200200000000003A6DEF0077
:10DF9000CC20020000000000B0C3B3003AEDB7008F
:10DFA00020C0B3003BEDB700A62002000000000037
:10DFB00000CEB3003AEDB700CC2002000000000014
:10DFC00000CEB3003AEDB700CC2002000000000004
:10DFD00000CEB3003AEDB700CC20020000000000F4
:10DFE00030C0B30030EDB7002E2402000000000066
:10DFF0003A6DEF0030C0B3003BEDB700A620020041
:10E000000000000006E8A9000500200005007800D7
:10E0100076160200000000000040B3004220AF006E
:10E02000050037008502E80036EDB7002424020021
:10E0300000000000F5FF370028C8BF0036EDB7002C
:10E04000242402000000000027C8BF0080027800DE
:10E050000B60EF00060020000500780086007800C5
:10E0600004002000E22B02000000000000C2B30008
:10E0700036EDB700242402000000000000C2B30007
:10E0800036EDB700242402000000000036043700FB
:10E09000746080004822DE006124E10094003A00B0
:10E0A0000100200001007800861602000000000038
:10E0B0008100E8003322AF00FEFF3700A011880086
:10E0C000300020000008E600F6FF370000002000C6
:10E0D0004140800052408000BC350200000000003A
:10E0E0002900200074380200000000009100200088
:10E0F0000100780086160200000000008100E800A0
:10E100003322AF00FEFF3700A0118800C0002000BE
:10E110000008E600F6FF37003A6DEF003B6DEF00B8
:10E12000A6200200000000006029EF004300A900C3
:10E130004040800051408000F226210033A8230097
:10E14000F62E020000000000800278000103780033
:10E15000000020008500780006017800BC35020030
:10E160000000000019002000A63A02000000000094
:10E1700070C2B3003AEDB70020C0B3003BEDB7006A
:10E18000A6200200000000003A6DEF00CC20020043
:10E19000000000003A6DEF00CC20020000000000FB
:10E1A0003A6DEF00CC20020000000000B0C3B300C5
:10E1B0003AEDB70020C0B3003BEDB700A620020047
:10E1C0000000000000CEB3003AEDB700CC20020002
:10E1D0000000000000CEB3003AEDB700CC200200F2
:10E1E0000000000000CEB3003AEDB700CC200200E2
:10E1F0000000000030C0B30030EDB7002E24020054
:10E20000000000003A6DEF0030C0B3003BEDB700F6
:10E21000A62002000000000006E8A900050020007A
:10E2200005007800A0160200000000000040B300C6
:10E230004220AF00050037008502E80036EDB70048
:10E240002424020000000000F5FF370028C8BF00AA
:10E2500036EDB700242402000000000027C8BF00EC
:10E26000800278000B60EF000600200005007800B7
:10E270008600780004002000E22B0200000000006D
:10E2800000C2B30036EDB7002424020000000000F5
:10E2900000C2B30036EDB7002424020000000000E5
:10E2A00010C4B3003AEDB70030C0B3003BEDB70087
:10E2B000A62002000000000006E8A90005002000DA
:10E2C00005007800B0160200000000000040B30016
:10E2D0004220AF00050037008502E80036EDB700A8
:10E2E0002424020000000000F5FF37009E033700E1
:10E2F000746080004822DE006224E10094003A004D
:10E300000100200001007800C0160200000000009B
:10E310008100E8003322AF00FEFF3700A011880023
:10E32000300020000008E600F6FF37000000200063
:10E330004140800052408000BC35020000000000D7
:10E340002900200074380200000000009100200025
:10E3500001007800C0160200000000008100E80003
:10E360003322AF00FEFF3700A0118800C00020005C
:10E370000008E600F6FF37003A6DEF003B6DEF0056
:10E38000A6200200000000006029EF004300A90061
:10E390004040800051408000F226210033A8230035
:10E3A000F62E0200000000008002780001037800D1
:10E3B000000020008500780006017800BC350200CE
:10E3C0000000000019002000A63A02000000000032
:10E3D00070C2B3003AEDB70020C0B3003BEDB70008
:10E3E000A6200200000000003A6DEF00CC200200E1
:10E3F000000000003A6DEF00CC2002000000000099
:10E400003A6DEF00CC20020000000000B0C3B30062
:10E410003AEDB70020C0B3003BEDB700A6200200E4
:10E420000000000000CEB3003AEDB700CC2002009F
:10E430000000000000CEB3003AEDB700CC2002008F
:10E440000000000000CEB3003AEDB700CC2002007F
:10E450000000000030C0B30030EDB7002E240200F1
:10E46000000000003A6DEF0030C0B3003BEDB70094
:10E47000A62002000000000006E8A9000500200018
:10E4800005007800DA160200000000000040B3002A
:10E490004220AF00050037008502E80036EDB700E6
:10E4A0002424020000000000F5FF370028C8BF0048
:10E4B00036EDB700242402000000000027C8BF008A
:10E4C000800278000B60EF00060020000500780055
:10E4D0008600780004002000E22B0200000000000B
:10E4E00000C2B30036EDB700242402000000000093
:10E4F00000C2B30036EDB700242402000000000083
:10E5000010C4B3003AEDB70030C0B3003BEDB70024
:10E51000A62002000000000006E8A9000500200077
:10E5200005007800B0160200000000000040B300B3
:10E530004220AF00050037008502E80036EDB70045
:10E540002424020000000000F5FF37000603370016
:10E55000746080004822DE006324E10099003A00E4
:10E560000100200001007800EA160200000000000F
:10E570008100E8003322AF00FEFF3700A0118800C1
:10E58000400020000008E600F6FF370000002000F1
:10E590004140800052408000BC3502000000000075
:10E5A000290020007438020000000000A1002000B3
:10E5B00001007800EA160200000000008100E80077
:10E5C0003322AF00FEFF3700A0118800D0002000EA
:10E5D0000008E600F6FF37003A6DEF003B6DEF00F4
:10E5E000A6200200000000006029EF004300A900FF
:10E5F0004040800051408000F226210033A82300D3
:10E60000F62E02000000000080027800010378006E
:10E610000500780086007800020020000312240024
:10E6200080300200000000008003780001047800C0
:10E63000000020008700780008017800BC35020047
:10E640000000000019002000A63A020000000000AF
:10E6500070C2B3003AEDB70020C0B3003BEDB70085
:10E66000A6200200000000003A6DEF00CC2002005E
:10E67000000000003A6DEF00CC2002000000000016
:10E680003A6DEF00CC20020000000000B0C3B300E0
:10E690003AEDB70020C0B3003BEDB700A620020062
:10E6A000000000003A6DEF00CC20020000000000E6
:10E6B0003A6DEF00CC200200000000003A6DEF0040
:10E6C000CC2002000000000030C0B30030EDB700E5
:10E6D0002E240200000000003A6DEF0030C0B300AD
:10E6E0003BEDB700A62002000000000006E8A900EC
:10E6F0000500200005007800061702000000000059
:10E700000040B3004220AF00050037008502E8005A
:10E7100036EDB7002424020000000000F5FF3700AA
:10E7200028C8BF0036EDB700242402000000000016
:10E7300027C8BF00800278000B60EF0006002000B1
:10E74000050078008600780004002000E22B02001B
:10E750000000000000C2B30036EDB7002424020020
:10E760000000000000C2B30036EDB7002424020010
:10E770000000000010C4B3003AEDB70030C0B30091
:10E780003BEDB700A62002000000000006E8A9004B
:10E790000500200005007800B0160200000000000F
:10E7A0000040B3004220AF00050037008502E800BA
:10E7B00036EDB7002424020000000000F5FF37000A
:10E7C00069023700746080004822DE006424E100A2
:10E7D00026013A000100200001007800181702000D
:10E7E000000000008100E8003322AF00FEFF370088
:10E7F000A0118800400020000008E600F6FF370066
:10E80000000020004140800052408000BC350200E2
:10E810000000000029002000743802000000000001
:10E82000A10020000100780018170200000000007D
:10E830008100E8003322AF00FEFF3700A0118800FE
:10E84000D00020000008E600F6FF370040408000BE
:10E850005140800002002400C36124008E2E02007B
:10E86000000000007B0039003A6DEF003B6DEF00C7
:10E87000A6200200000000006029EF004300A9006C
:10E880004040800051408000F226210033A8230040
:10E89000F62E0200000000008002780001037800DC
:10E8A0000500780086007800020020000312240092
:10E8B000803002000000000080037800010478002E
:10E8C000000020008700780008017800BC350200B5
:10E8D0000000000019002000A63A0200000000001D
:10E8E00070C2B3003AEDB70020C0B3003BEDB700F3
:10E8F000A6200200000000003A6DEF00CC200200CC
:10E90000000000003A6DEF00CC2002000000000083
:10E910003A6DEF00CC20020000000000B0C3B3004D
:10E920003AEDB70020C0B3003BEDB700A6200200CF
:10E93000000000003A6DEF00CC2002000000000053
:10E940003A6DEF00CC200200000000003A6DEF00AD
:10E95000CC2002000000000030C0B30030EDB70052
:10E960002E240200000000003A6DEF0030C0B3001A
:10E970003BEDB700A62002000000000006E8A90059
:10E980000500200005007800341702000000000098
:10E990000040B3004220AF00050037008502E800C8
:10E9A00036EDB7002424020000000000F5FF370018
:10E9B00028C8BF0036EDB700242402000000000084
:10E9C00027C8BF00800278000B60EF00060020001F
:10E9D000050078008600780004002000E22B020089
:10E9E0000000000000C2B30036EDB700242402008E
:10E9F0000000000000C2B30036EDB700242402007E
:10EA00000000000010C4B3003AEDB70030C0B300FE
:10EA10003BEDB700A62002000000000006E8A900B8
:10EA20000500200005007800B0160200000000007C
:10EA30000040B3004220AF00050037008502E80027
:10EA400036EDB7002424020000000000F5FF370077
:10EA50008500370000002400C1612400424080008E
:10EA6000534080008E2E02000000000001003100A3
:10EA70007D003A003A6DEF003B6DEF00A6200200EA
:10EA8000000000006029EF004300A9004040800022
:10EA900051408000F226210033A82300F62E020008
:10EAA0000000000080027800010378000500780073
:10EAB0008600780002002000A34724008030020076
:10EAC00000000000800378000104780000002000AE
:10EAD0008700780008017800BC35020000000000C3
:10EAE00029002000A63A02000000000070C2B30016
:10EAF0003AEDB70020C0B3003BEDB700A6200200FE
:10EB00000000000000CEB3003AEDB700CC200200B8
:10EB10000000000000CEB3003AEDB700CC200200A8
:10EB20000000000000CEB3003AEDB700CC20020098
:10EB300000000000B0C3B3003AEDB70020C0B3003E
:10EB40003BEDB700A6200200000000003A6DEF0088
:10EB5000CC200200000000003A6DEF00CC20020043
:10EB6000000000003A6DEF00CC2002000000000021
:10EB700030C0B30030EDB7002E24020000000000CA
:10EB80003A6DEF0030C0B3003BEDB700A6200200A5
:10EB90000000000006E8A90005002000050078003C
:10EBA00034170200000000000040B3004220AF0014
:10EBB000050037008502E80036EDB7002424020086
:10EBC00000000000F5FF370028C8BF0036EDB70091
:10EBD000242402000000000027C8BF008002780043
:10EBE0000B60EF000600200005007800860078002A
:10EBF00004002000E22B02000000000000C2B3006D
:10EC000036EDB700242402000000000000C2B3006B
:10EC100036EDB700242402000000000010C4B30049
:10EC20003AEDB70030C0B3003BEDB700A6200200BC
:10EC30000000000006E8A90005002000050078009B
:10EC400046170200000000000040B3004220AF0061
:10EC5000050037008502E80036EDB70024240200E5
:10EC600000000000F5FF37003F01370074608000AE
:10EC70004822DE006524E1009C003A0001002000EB
:10EC80000100780056170200000000008100E80033
:10EC90003322AF00FEFF3700A011880040002000A3
:10ECA0000008E600F6FF3700000020004140800029
:10ECB00052408000BC350200000000002900200006
:10ECC0007438020000000000A1002000010078005C
:10ECD00056170200000000008100E8003322AF0058
:10ECE000FEFF3700A0118800D00020000008E600D9
:10ECF000F6FF37003A6DEF003B6DEF00A6200200F3
:10ED0000000000006029EF004300A900404080009F
:10ED100051408000F226210033A82300F62E020085
:10ED200000000000800278000103780005007800F0
:10ED30008600780002002000A347240080300200F3
:10ED4000000000008003780001047800000020002B
:10ED50008700780008017800BC3502000000000040
:10ED600029002000A63A02000000000070C2B30093
:10ED70003AEDB70020C0B3003BEDB700A62002007B
:10ED80000000000000CEB3003AEDB700CC20020036
:10ED90000000000000CEB3003AEDB700CC20020026
:10EDA0000000000000CEB3003AEDB700CC20020016
:10EDB00000000000B0C3B3003AEDB70020C0B300BC
:10EDC0003BEDB700A6200200000000003A6DEF0006
:10EDD000CC200200000000003A6DEF00CC200200C1
:10EDE000000000003A6DEF00CC200200000000009F
:10EDF00030C0B30030EDB7002E2402000000000048
:10EE00003A6DEF0030C0B3003BEDB700A620020022
:10EE10000000000006E8A9000500200005007800B9
:10EE200072170200000000000040B3004220AF0053
:10EE3000050037008502E80036EDB7002424020003
:10EE400000000000F5FF370028C8BF0036EDB7000E
:10EE5000242402000000000027C8BF0080027800C0
:10EE60000B60EF00060020000500780086007800A7
:10EE700004002000E22B02000000000000C2B300EA
:10EE800036EDB700242402000000000000C2B300E9
:10EE900036EDB700242402000000000010C4B300C7
:10EEA0003AEDB70030C0B3003BEDB700A62002003A
:10EEB0000000000006E8A900050020000500780019
:10EEC00046170200000000000040B3004220AF00DF
:10EED000050037008502E80036EDB7002424020063
:10EEE00000000000F5FF37009F00370074608000CD
:10EEF0004822DE006624E1009B003A000100200069
:10EF00000100780084170200000000008100E80082
:10EF10003322AF00FEFF3700A01188004000200020
:10EF20000008E600F6FF37000000200041408000A6
:10EF300052408000BC350200000000002900200083
:10EF40007438020000000000A100200001007800D9
:10EF500084170200000000008100E8003322AF00A7
:10EF6000FEFF3700A0118800D00020000008E60056
:10EF7000F6FF37003A6DEF003B6DEF00A620020070
:10EF8000000000006029EF004300A900404080001D
:10EF900051408000F226210033A82300F62E020003
:10EFA000000000008002780001037800050078006E
:10EFB0008600780002002000A34724008030020071
:10EFC00000000000800378000104780000002000A9
:10EFD0008700780008017800BC35020000000000BE
:10EFE00029002000A63A02000000000070C2B30011
:10EFF0003AEDB70020C0B3003BEDB700A6200200F9
:10F000000000000000CEB3003AEDB700CC200200B3
:10F010000000000000CEB3003AEDB700CC200200A3
:10F020000000000000CEB3003AEDB700CC20020093
:10F0300000000000B0C3B3003AEDB70020C0B30039
:10F040003BEDB700A6200200000000003A6DEF0083
:10F05000CC200200000000003A6DEF00CC2002003E
:10F06000000000003A6DEF00CC200200000000001C
:10F0700030C0B30030EDB7002E24020000000000C5
:10F080003A6DEF0030C0B3003BEDB700A6200200A0
:10F090000000000006E8A900050020000500780037
:10F0A000A0170200000000000040B3004220AF00A3
:10F0B000050037008502E80036EDB7002424020081
:10F0C00000000000F5FF370028C8BF0036EDB7008C
:10F0D000242402000000000027C8BF00800278003E
:10F0E0000B60EF0006002000050078008600780025
:10F0F00004002000E22B02000000000000C2B30068
:10F1000036EDB700242402000000000000C2B30066
:10F1100036EDB700242402000000000010C4B30044
:10F120003AEDB70030C0B3003BEDB700A6200200B7
:10F130000000000006E8A900050020000500780096
:10F1400046170200000000000040B3004220AF005C
:10F15000050037008502E80036EDB70024240200E0
:10F1600000000000F5FF370040C0B30030EDB700ED
:10F170002E2402000000000050C0B30030EDB700A4
:10F180002E2402000000000010C0B30030EDB700D4
:10F19000E03B0200000000000060EF0000000600FD
:10F1A000851F7800E46280006124E10007003A00D6
:10F1B0002768EC00344180004822DE006F24E10023
:10F1C000010039002768EF000D0037005C4CE200B9
:10F1D00008003A002768ED00344180004822DE0034
:10F1E000F4CFB20002003A00F0C0B30027E8B70045
:10F1F00003003700E46280006224E10000003A006E
:10F200000100200001007800C21D02000000000083
:10F210008100E8003322AF00FEFF3700A011880014
:10F22000F00020000008E600F6FF370027C8BF0006
:10F230000160EF0004002000C8240200000000006C
:10F240002101200001007800C21D02000000000022
:10F250008100E8003322AF00FEFF3700A0118800D4
:10F26000500120000008E600F6FF370027C8BF0065
:10F270000160EF004400DD002CE8B7002CC8BF009F
:10F2800060ECB700616CEF00BE27020000000000D8
:10F290002EE8B700644180006142420004407800DB
:10F2A0000AE0B7000540780060ECB700616CEF0041
:10F2B000BE270200000000002FE8B7002EC8BF00E4
:10F2C00030E8B7003168EF0030C8BF0031E8B70060
:10F2D0003068EF00744180004822DE0083418000E6
:10F2E000048041008041880084418000F33F200079
:10F2F0000418E10001003900040037008441800057
:10F30000030028000418E10004003E00D0C2B3004E
:10F3100028E8B700260037000200370000C5B30018
:10F3200028E8B7000100200001007800E61D020077
:10F33000000000008100E8003322AF00FEFF37002C
:10F34000A0118800600020000008E600F6FF3700EA
:10F350008041800004002000C8240200000000005A
:10F360003322AF00FEFF370004022000A411880002
:10F37000644180006A424200044078000AE0B7001D
:10F380000540780060ECB700616CEF00BE2702001A
:10F390000000000012ECB70012CCBF005DECB7001B
:10F3A0003008F8005E0CF900C26C0200000000009A
:10F3B000CF02780000000600851F7800861F7800C5
:10F3C000871F7800586CEF00D222EF0004802000E5
:10F3D000B41688000000000000000000F43F200088
:10F3E00094168800D742A800D342A900000000006C
:10F3F00000000000562402000000000010C0B3000E
:10F400003AEDB70010C0B3003BEDB700A6200200F4
:10F41000000000000500200005007800941A02009A
:10F42000000000000040B3004220AF00050037009C
:10F430008502E80036EDB700242402000000000039
:10F44000F5FF370010C0B3003AEDB70030C0B3008D
:10F450003BEDB700A62002000000000005002000E0
:10F4600005007800D2180200000000000040B30040
:10F470004220AF00050037008502E80036EDB700F6
:10F480002424020000000000F5FF370010C0B30084
:10F490003AEDB70040C0B3003BEDB700A620020034
:10F4A000000000000500200005007800AE1A0200F0
:10F4B000000000000040B3004220AF00050037000C
:10F4C0008502E80036EDB7002424020000000000A9
:10F4D000F5FF37000500200005007800C81A02007B
:10F4E000000000000040B3004220AF0006003700DB
:10F4F0008502E8003322AF00FEFF370034E2B70098
:10F500003562EF00F4FF37000500200005007800A9
:10F51000E81A0200000000000040B3004220AF00E3
:10F52000060037008502E8003322AF00FEFF3700F7
:10F5300034E2B7003562EF00F4FF37000500200029
:10F54000050078000C1B0200000000000040B30022
:10F550004220AF00060037008502E8003322AF00EA
:10F56000FEFF370034E2B7003562EF00F4FF3700EA
:10F57000D262A800D462AF0007003700D242A800D0
:10F58000D442AF0004003700D282A800D482AF007A
:10F5900001003700F6FF3700D282A800D482AE0007
:10F5A000C30037005624020000000000542CEF0076
:10F5B000F42A2400B4628800596CEF00C462800011
:10F5C0004822DE006F24E100B80032008529A8003F
:10F5D00059CCBF0027E8B700216DEF00540CF800AC
:10F5E000220DF900560CF800240DF900EC3C020045
:10F5F000000000008529AE00AA003700A00020000E
:10F60000641F02000000000010C0B30030EDB7001E
:10F61000E03B02000000000090C0B3003AEDB700EC
:10F6200060C0B3003BEDB700A62002000000000060
:10F6300005002000050078002E1B020000000000DD
:10F640000040B3004220AF00050037008502E8000B
:10F6500036EDB7002424020000000000F5FF37005B
:10F66000646180004822DE00A3052000041CE10044
:10F6700075003E002DCCBF005AECB7004300A90036
:10F68000A0628000B1628000D2CC2C00C3D42300E1
:10F69000F62E020000000000A0628800B16288001F
:10F6A00010C0B3005CECB700825202000000000002
:10F6B00020032000641F02000000000010C0B300FF
:10F6C00030EDB700E03B0200000000002DCCBF0091
:10F6D0005BECB7005ACCBF00D46280004822DE0049
:10F6E0000024E100010039000C0037004300A800AD
:10F6F000A0628000B1628000D2CC2C00C3D4230071
:10F70000F62E020000000000A0628800B1628800AE
:10F710005C6CEF008252020000000000522CEF00EF
:10F720009462800083BB20000418E1000A003900C5
:10F73000B05F0200000000008509AE000400370041
:10F7400024032000936280000480410090628800BE
:10F75000522CEC00F2FF3700844B80006224E10061
:10F7600022003900522CEF009462800003712200C5
:10F770000418E1000A003900B05F02000000000038
:10F780008509AE0004003700240320009362800046
:10F790000480410090628800522CEC00F2FF370098
:10F7A0003C6102000000000056240200000000003E
:10F7B0008529A9004300A900A0628000B1628000F1
:10F7C000D2CC2C00C3DC2300F62E02000000000087
:10F7D000A0628800B162880010C0B3005CECB70082
:10F7E00082520200000000000D0037004300A90013
:10F7F000A0628000B1628000D2CC2C00C3D4230070
:10F80000F62E020000000000A0628800B1628800AD
:10F8100010C0B3005CECB700825202000000000090
:10F8200000002000812D24004240800053408000D1
:10F830008E2E0200000000000100310001003A009D
:10F84000180037000D0037004300A900A0628000B7
:10F85000B1628000D2CC2C00C3D42300F62E02006B
:10F8600000000000A0628800B162880010C0B300F0
:10F870005CECB70082520200000000000000200093
:10F88000812D240042408000534080008E2E0200D3
:10F89000000000000100310001003A0001003700C3
:10F8A00054FF3700596CEC0044FF37008529A9004C
:10F8B0007A2502000000000056240200000000002B
:10F8C0002768EF0020C0B3005CECB700D0780200DE
:10F8D00000000000CF0378004F037800CF027800CB
:10F8E00000000600E41F200004638800BE27020019
:10F8F0000000000029ECB700446180004822DE00CF
:10F90000F4CFB20002003A0080C0B30029ECB70087
:10F91000D41F200004638800BE27020000000000FE
:10F920002AECB70054618000F4CFB20002003A0024
:10F9300000C2B3002AECB700F41F20000463880063
:10F94000BE270200000000002CECB70064618000BC
:10F95000F4CFB20002003A00E0C1B3002CECB700D3
:10F9600000C2B3001CEDB700E0CFB3001DEDB7003F
:10F97000B42802000000000010C2B3001CEDB70064
:10F9800080C0B3001DEDB700B428020000000000E5
:10F9900020C2B3001CEDB700E0C5B3001DEDB700F9
:10F9A000B42802000000000030C2B3001CEDB70014
:10F9B00000C6B3001DEDB700B4280200000000002F
:10F9C00040C2B3001CEDB700C0C0B3001DEDB700CE
:10F9D000B42802000000000050C2B3001CEDB700C4
:10F9E00000C2B3001DEDB700B42802000000000003
:10F9F00060C2B3001CEDB70040C8B3001DEDB700F6
:10FA0000B42802000000000070C2B3001CEDB70073
:10FA10002ACCBF001DEDB700B42802000000000092
:10FA200080C2B3001CEDB70029CCBF001DEDB700AC
:10FA3000B42802000000000090C2B3001CEDB70023
:10FA4000A0C4B3001DEDB700B42802000000000000
:10FA5000A0C2B3001CEDB70050C8B3001DEDB70045
:10FA6000B428020000000000B0C2B3001CEDB700D3
:10FA700060C6B3001DEDB700B4280200000000000E
:10FA8000C0C2B3001CEDB700C0C7B3001DEDB70086
:10FA9000B428020000000000D0C2B3001CEDB70083
:10FAA000F0C6B3001DEDB700B4280200000000004E
:10FAB000E0C2B3001CEDB700A0C6B3001DEDB70057
:10FAC000B428020000000000F0C2B3001CEDB70033
:10FAD00090C1B3001DEDB700B42802000000000083
:10FAE00000C3B3001CEDB700A0C0B3001DEDB7000C
:10FAF000B42802000000000010C3B3001CEDB700E2
:10FB00002CCCBF001DEDB700B4280200000000009F
:10FB100020C3B3001CEDB700C0C0B3001DEDB7009B
:10FB2000B42802000000000030C3B3001CEDB70091
:10FB3000C0C0B3001DEDB700B428020000000000F3
:10FB400040C3B3001CEDB7001D6DEF00B4280200E8
:10FB50000000000050C3B3001CEDB70030C0B3007C
:10FB60001DEDB700B42802000000000060C3B30020
:10FB70001CEDB70000C8B3001DEDB700B4280200AB
:10FB80000000000070C3B3001CEDB700C0C1B3009B
:10FB90001DEDB700B42802000000000080C3B300D0
:10FBA0001CEDB70060C0B3001DEDB700B428020023
:10FBB0000000000090C3B3001CEDB7001D6DEF0006
:10FBC000B428020000000000A0C3B3001CEDB70081
:10FBD0001D6DEF00B428020000000000B0C3B300A8
:10FBE0001CEDB7001D6DEF00B428020000000000FE
:10FBF000C0C3B3001CEDB7001D6DEF00B4280200B8
:10FC000000000000D0C3B3001CEDB7001D6DEF0075
:10FC1000B428020000000000E0C3B3001CEDB700F0
:10FC20001D6DEF00B428020000000000F0C3B30017
:10FC30001CEDB7001D6DEF00B428020000000000AD
:10FC4000E262A800DE62A900C41F200004638800ED
:10FC5000BE270200000000002BECB70054618000BA
:10FC60004822DE00F4CFB20006003A00304A02001B
:10FC7000000000006452020000000000DC79020075
:10FC8000000000000060EF0000000600851F780003
:10FC900054C8BF005548E300FDFF3200A442800075
:10FCA0004822DE0043832000030042001040780019
:10FCB00057E8B700A44280004822DE0061424200BB
:10FCC0000440780000E0B7007F40600055E8B700CE
:10FCD00057C8BF0000E0B700CF0278000000060060
:10FCE000851F7800520CF800540CF900A0628000C7
:10FCF0001004E00002003200542CEC00FBFF37003F
:10FD0000A4628000936280000300520000E0B7000C
:10FD1000CF02780000000600851F7800564CE200F4
:10FD20001D0032009062800090427800A062800046
:10FD300010407800002CE1000C003200906280003E
:10FD400090427800A062800010407800002CE10012
:10FD50000200310000C0EB000100370010C0B3000A
:10FD600000E0B7000D00370005003700906280000A
:10FD70001004E00002003A000060EF0007003700C6
:10FD800090628000522CEC00A0628000542CEC00A9
:10FD9000566CED00E1FF37000060EF00CF02780005
:10FDA00000000600851F7800467E0200000000006B
:10FDB0002EECB700746180006D24E10006003A006B
:10FDC000C44280000960EF00A38520008302420046
:10FDD000804AEB000E003700C44280000960EF004B
:10FDE000A3852000830242002ECCBF0080429800F1
:10FDF000C442800023022000041CE10002003E00F7
:10FE00005868EF00010037005868EC0048063700DA
:10FE10000200200001C3200002007800561E0200EC
:10FE200000000000805878000201E8000004E000B3
:10FE30004220AE00F8FF37000200200061C320001E
:10FE400002007800661E0200000000008058780062
:10FE50000201E8000004E0004220AE00F8FF370095
:10FE600002002000A1C3200002007800761E0200DC
:10FE700000000000805878000201E8000004E00063
:10FE80004220AE00F8FF37000200200001C420002D
:10FE900002007800861E02000000000080587800F2
:10FEA0000201E8000004E0004220AE00F8FF370045
:10FEB0000200200041C4200002007800961E0200CB
:10FEC00000000000805878000201E8000004E00013
:10FED0004220AE00F8FF370002002000A1C420003D
:10FEE00002007800A61E0200000000008058780082
:10FEF0000201E8000004E0004220AE00F8FF3700F5
:10FF000002002000E1C4200002007800B61E0200BA
:10FF100000000000805878000201E8000004E000C2
:10FF20004220AE00F8FF3700A485200094628800CC
:10FF3000707E0200000000006304E100F10539005A
:10FF400030C0B30056ECB700A4852000946288004E
:10FF500004C32000A46288008C7E02000000000020
:10FF60002FECB70030C0B30056ECB700A4852000DA
:10FF70009462880064C32000A46288008C7E020022
:10FF80000000000034ECB70030C0B30056ECB700FE
:10FF9000A485200094628800A4C32000A462880085
:10FFA0008C7E02000000000035ECB70030C0B300CA
:10FFB00056ECB700A48520009462880004C4200099
:10FFC000A46288008C7E0200000000003EECB700B6
:10FFD00030C0B30056ECB700A485200094628800BE
:10FFE00044C42000A46288008C7E0200000000004F
:10FFF0003FECB70030C0B30056ECB700A48520003A
:020000040001F9
:1000000094628800A4C42000A46288008C7E020050
:100010000000000048ECB70030C0B30056ECB70059
:10002000A485200094628800E4C42000A4628800B3
:100030008C7E02000000000049ECB7002F4CE2006B
:100040001A003A000500200005007800C61E0200D4
:10005000000000000040B3004220AF00060037005F
:100060008502E8003322AF00FEFF370034E2B7001C
:100070003562EF00F4FF37003322AF00FEFF370098
:1000800004022000A41188005C6CEF008252020080
:100090000000000010C0B30030EDB700E03B0200EC
:1000A000000000008560A90096053700344CE2008E
:1000B0001B003A000500200005007800DE1E02004B
:1000C000000000000040B3004220AF0006003700EF
:1000D0008502E8003322AF00FEFF370034E2B700AC
:1000E0003562EF00F4FF37003322AF00FEFF370028
:1000F00004022000A411880010C0B3005CECB7001B
:10010000825202000000000010C0B30030EDB700C2
:10011000E03B0200000000008560A900790537007F
:10012000354CE20018053A00050020000500780073
:10013000F61E0200000000000040B3004220AF00A5
:10014000060037008502E8003322AF00FEFF3700CB
:1001500034E2B7003562EF00F4FF37003322AF001E
:10016000FEFF370004022000A41188000F4CE200BB
:10017000CD003A004300A90040408000514080007B
:10018000F226210033B02300F62E0200000000000A
:10019000800278000103780001002000010078004F
:1001A0005A160200000000008100E8003322AF0070
:1001B000FEFF3700A0118800500020000008E60074
:1001C000F6FF370000002000850078000601780067
:1001D000BC35020000000000290020007438020035
:1001E00000000000B1002000010078005A16020053
:1001F000000000008100E8003322AF00FEFF37005E
:10020000A0118800E00020000008E600F6FF37009B
:100210003A6DEF003B6DEF00A620020000000000E9
:100220006029EF004300A900404080005140800059
:10023000F226210033A82300F62E02000000000061
:1002400080027800010378000500780086007800BD
:1002500002002000832C24008E2E020000000000EB
:10026000330039004300A900404080005140800025
:10027000F226210033B02300F62E02000000000019
:1002800080027800010378000000200085007800DB
:1002900006017800BC3502000000000029002000A3
:1002A000A63A02000000000070C2B3003AEDB700A9
:1002B00020C0B3003BEDB700A62002000000000004
:1002C00000CEB3003AEDB700CC20020000000000E1
:1002D00000CEB3003AEDB700CC20020000000000D1
:1002E00000CEB3003AEDB700CC20020000000000C1
:1002F000B0C3B3003AEDB70020C0B3003BEDB70088
:10030000A6200200000000003A6DEF00CC200200A1
:10031000000000003A6DEF00CC2002000000000059
:100320003A6DEF00CC2002000000000032003700E0
:100330004300A9004040800051408000F226210087
:1003400033B02300F62E0200000000008002780087
:100350000103780000002000850078000601780085
:10036000BC3502000000000019002000A63A02007F
:100370000000000070C2B3003AEDB70020C0B30027
:100380003BEDB700A6200200000000003A6DEF0030
:10039000CC200200000000003A6DEF00CC200200EB
:1003A000000000003A6DEF00CC20020000000000C9
:1003B000B0C3B3003AEDB70020C0B3003BEDB700C7
:1003C000A62002000000000000CEB3003AEDB70006
:1003D000CC2002000000000000CEB3003AEDB700D0
:1003E000CC2002000000000000CEB3003AEDB700C0
:1003F000CC2002000000000030C0B30030EDB70098
:100400002E240200000000003A6DEF0030C0B3005F
:100410003BEDB700A62002000000000006E8A9009E
:10042000050020000500780076160200000000009C
:100430000040B3004220AF00050037008502E8000D
:1004400036EDB7002424020000000000F5FF37005D
:1004500028C8BF0036EDB7002424020000000000C9
:1004600027C8BF00800278000B60EF000600200064
:10047000050078008600780004002000E22B0200CE
:100480000000000000C2B30036EDB70024240200D3
:100490000000000000C2B30036EDB70024240200C3
:1004A0000000000036043700746080004822DE003F
:1004B0006124E10094003A0001002000010078006E
:1004C00086160200000000008100E8003322AF0021
:1004D000FEFF3700A0118800300020000008E60071
:1004E000F6FF3700000020004140800052408000AD
:1004F000BC35020000000000290020007438020012
:100500000000000091002000010078008616020023
:10051000000000008100E8003322AF00FEFF37003A
:10052000A0118800C00020000008E600F6FF370098
:100530003A6DEF003B6DEF00A620020000000000C6
:100540006029EF004300A900404080005140800036
:10055000F226210033A82300F62E0200000000003E
:1005600080027800010378000000200085007800F8
:1005700006017800BC3502000000000019002000D0
:10058000A63A02000000000070C2B3003AEDB700C6
:1005900020C0B3003BEDB700A62002000000000021
:1005A0003A6DEF00CC200200000000003A6DEF0031
:1005B000CC200200000000003A6DEF00CC200200C9
:1005C00000000000B0C3B3003AEDB70020C0B30094
:1005D0003BEDB700A62002000000000000CEB300F3
:1005E0003AEDB700CC2002000000000000CEB300BE
:1005F0003AEDB700CC2002000000000000CEB300AE
:100600003AEDB700CC2002000000000030C0B3007B
:1006100030EDB7002E240200000000003A6DEF001C
:1006200030C0B3003BEDB700A62002000000000080
:1006300006E8A9000500200005007800A0160200C9
:10064000000000000040B3004220AF00050037006A
:100650008502E80036EDB700242402000000000007
:10066000F5FF370028C8BF0036EDB700242402008C
:100670000000000027C8BF00800278000B60EF0078
:1006800006002000050078008600780004002000A5
:10069000E22B02000000000000C2B30036EDB700FC
:1006A000242402000000000000C2B30036EDB700B1
:1006B000242402000000000010C4B3003AEDB7008B
:1006C00030C0B3003BEDB700A620020000000000E0
:1006D00006E8A9000500200005007800B016020019
:1006E000000000000040B3004220AF0005003700CA
:1006F0008502E80036EDB700242402000000000067
:10070000F5FF37009E033700746080004822DE004A
:100710006224E10094003A0001002000010078000A
:10072000C0160200000000008100E8003322AF0084
:10073000FEFF3700A0118800300020000008E6000E
:10074000F6FF37000000200041408000524080004A
:10075000BC350200000000002900200074380200AF
:10076000000000009100200001007800C016020087
:10077000000000008100E8003322AF00FEFF3700D8
:10078000A0118800C00020000008E600F6FF370036
:100790003A6DEF003B6DEF00A62002000000000064
:1007A0006029EF004300A9004040800051408000D4
:1007B000F226210033A82300F62E020000000000DC
:1007C0008002780001037800000020008500780096
:1007D00006017800BC35020000000000190020006E
:1007E000A63A02000000000070C2B3003AEDB70064
:1007F00020C0B3003BEDB700A620020000000000BF
:100800003A6DEF00CC200200000000003A6DEF00CE
:10081000CC200200000000003A6DEF00CC20020066
:1008200000000000B0C3B3003AEDB70020C0B30031
:100830003BEDB700A62002000000000000CEB30090
:100840003AEDB700CC2002000000000000CEB3005B
:100850003AEDB700CC2002000000000000CEB3004B
:100860003AEDB700CC2002000000000030C0B30019
:1008700030EDB7002E240200000000003A6DEF00BA
:1008800030C0B3003BEDB700A6200200000000001E
:1008900006E8A9000500200005007800DA1602002D
:1008A000000000000040B3004220AF000500370008
:1008B0008502E80036EDB7002424020000000000A5
:1008C000F5FF370028C8BF0036EDB700242402002A
:1008D0000000000027C8BF00800278000B60EF0016
:1008E0000600200005007800860078000400200043
:1008F000E22B02000000000000C2B30036EDB7009A
:10090000242402000000000000C2B30036EDB7004E
:10091000242402000000000010C4B3003AEDB70028
:1009200030C0B3003BEDB700A6200200000000007D
:1009300006E8A9000500200005007800B0160200B6
:10094000000000000040B3004220AF000500370067
:100950008502E80036EDB700242402000000000004
:10096000F5FF370006033700746080004822DE0080
:100970006324E10099003A000100200001007800A2
:10098000EA160200000000008100E8003322AF00F8
:10099000FEFF3700A0118800400020000008E6009C
:1009A000F6FF3700000020004140800052408000E8
:1009B000BC3502000000000029002000743802004D
:1009C00000000000A100200001007800EA160200EB
:1009D000000000008100E8003322AF00FEFF370076
:1009E000A0118800D00020000008E600F6FF3700C4
:1009F0003A6DEF003B6DEF00A62002000000000002
:100A00006029EF004300A900404080005140800071
:100A1000F226210033A82300F62E02000000000079
:100A200080027800010378000500780086007800D5
:100A300002002000031224008030020000000000A9
:100A4000800378000104780000002000870078000F
:100A500008017800BC3502000000000019002000E9
:100A6000A63A02000000000070C2B3003AEDB700E1
:100A700020C0B3003BEDB700A6200200000000003C
:100A80003A6DEF00CC200200000000003A6DEF004C
:100A9000CC200200000000003A6DEF00CC200200E4
:100AA00000000000B0C3B3003AEDB70020C0B300AF
:100AB0003BEDB700A6200200000000003A6DEF00F9
:100AC000CC200200000000003A6DEF00CC200200B4
:100AD000000000003A6DEF00CC2002000000000092
:100AE00030C0B30030EDB7002E240200000000003B
:100AF0003A6DEF0030C0B3003BEDB700A620020016
:100B00000000000006E8A9000500200005007800AC
:100B100006170200000000000040B3004220AF00B2
:100B2000050037008502E80036EDB70024240200F6
:100B300000000000F5FF370028C8BF0036EDB70001
:100B4000242402000000000027C8BF0080027800B3
:100B50000B60EF000600200005007800860078009A
:100B600004002000E22B02000000000000C2B300DD
:100B700036EDB700242402000000000000C2B300DC
:100B800036EDB700242402000000000010C4B300BA
:100B90003AEDB70030C0B3003BEDB700A62002002D
:100BA0000000000006E8A90005002000050078000C
:100BB000B0160200000000000040B3004220AF0069
:100BC000050037008502E80036EDB7002424020056
:100BD00000000000F5FF37006902370074608000F4
:100BE0004822DE006424E10026013A0001002000D2
:100BF0000100780018170200000000008100E800E2
:100C00003322AF00FEFF3700A01188004000200013
:100C10000008E600F6FF3700000020004140800099
:100C200052408000BC350200000000002900200076
:100C30007438020000000000A100200001007800CC
:100C400018170200000000008100E8003322AF0006
:100C5000FEFF3700A0118800D00020000008E60049
:100C6000F6FF370040408000514080000200240021
:100C7000C36124008E2E0200000000007B003900BA
:100C80003A6DEF003B6DEF00A6200200000000006F
:100C90006029EF004300A9004040800051408000DF
:100CA000F226210033A82300F62E020000000000E7
:100CB0008002780001037800050078008600780043
:100CC0000200200003122400803002000000000017
:100CD000800378000104780000002000870078007D
:100CE00008017800BC350200000000001900200057
:100CF000A63A02000000000070C2B3003AEDB7004F
:100D000020C0B3003BEDB700A620020000000000A9
:100D10003A6DEF00CC200200000000003A6DEF00B9
:100D2000CC200200000000003A6DEF00CC20020051
:100D300000000000B0C3B3003AEDB70020C0B3001C
:100D40003BEDB700A6200200000000003A6DEF0066
:100D5000CC200200000000003A6DEF00CC20020021
:100D6000000000003A6DEF00CC20020000000000FF
:100D700030C0B30030EDB7002E24020000000000A8
:100D80003A6DEF0030C0B3003BEDB700A620020083
:100D90000000000006E8A90005002000050078001A
:100DA00034170200000000000040B3004220AF00F2
:100DB000050037008502E80036EDB7002424020064
:100DC00000000000F5FF370028C8BF0036EDB7006F
:100DD000242402000000000027C8BF008002780021
:100DE0000B60EF0006002000050078008600780008
:100DF00004002000E22B02000000000000C2B3004B
:100E000036EDB700242402000000000000C2B30049
:100E100036EDB700242402000000000010C4B30027
:100E20003AEDB70030C0B3003BEDB700A62002009A
:100E30000000000006E8A900050020000500780079
:100E4000B0160200000000000040B3004220AF00D6
:100E5000050037008502E80036EDB70024240200C3
:100E600000000000F5FF3700850037000000240077
:100E7000C161240042408000534080008E2E020059
:100E800000000000010031007D003A003A6DEF00E3
:100E90003B6DEF00A6200200000000006029EF007B
:100EA0004300A9004040800051408000F22621000C
:100EB00033A82300F62E0200000000008002780014
:100EC0000103780005007800860078000200200009
:100ED000A347240080300200000000008003780057
:100EE00001047800000020008700780008017800E5
:100EF000BC3502000000000029002000A63A0200D4
:100F00000000000070C2B3003AEDB70020C0B3008B
:100F10003BEDB700A62002000000000000CEB300A9
:100F20003AEDB700CC2002000000000000CEB30074
:100F30003AEDB700CC2002000000000000CEB30064
:100F40003AEDB700CC20020000000000B0C3B300AF
:100F50003AEDB70020C0B3003BEDB700A620020079
:100F6000000000003A6DEF00CC20020000000000FD
:100F70003A6DEF00CC200200000000003A6DEF0057
:100F8000CC2002000000000030C0B30030EDB700FC
:100F90002E240200000000003A6DEF0030C0B300C4
:100FA0003BEDB700A62002000000000006E8A90003
:100FB0000500200005007800341702000000000042
:100FC0000040B3004220AF00050037008502E80072
:100FD00036EDB7002424020000000000F5FF3700C2
:100FE00028C8BF0036EDB70024240200000000002E
:100FF00027C8BF00800278000B60EF0006002000C9
:10100000050078008600780004002000E22B020032
:101010000000000000C2B30036EDB7002424020037
:101020000000000000C2B30036EDB7002424020027
:101030000000000010C4B3003AEDB70030C0B300A8
:101040003BEDB700A62002000000000006E8A90062
:10105000050020000500780046170200000000008F
:101060000040B3004220AF00050037008502E800D1
:1010700036EDB7002424020000000000F5FF370021
:101080003F013700746080004822DE006524E100E3
:101090009C003A0001002000010078005617020071
:1010A000000000008100E8003322AF00FEFF37009F
:1010B000A0118800400020000008E600F6FF37007D
:1010C000000020004140800052408000BC350200FA
:1010D0000000000029002000743802000000000019
:1010E000A100200001007800561702000000000057
:1010F0008100E8003322AF00FEFF3700A011880016
:10110000D00020000008E600F6FF37003A6DEF003F
:101110003B6DEF00A6200200000000006029EF00F8
:101120004300A9004040800051408000F226210089
:1011300033A82300F62E0200000000008002780091
:101140000103780005007800860078000200200086
:10115000A3472400803002000000000080037800D4
:101160000104780000002000870078000801780062
:10117000BC3502000000000029002000A63A020051
:101180000000000070C2B3003AEDB70020C0B30009
:101190003BEDB700A62002000000000000CEB30027
:1011A0003AEDB700CC2002000000000000CEB300F2
:1011B0003AEDB700CC2002000000000000CEB300E2
:1011C0003AEDB700CC20020000000000B0C3B3002D
:1011D0003AEDB70020C0B3003BEDB700A6200200F7
:1011E000000000003A6DEF00CC200200000000007B
:1011F0003A6DEF00CC200200000000003A6DEF00D5
:10120000CC2002000000000030C0B30030EDB70079
:101210002E240200000000003A6DEF0030C0B30041
:101220003BEDB700A62002000000000006E8A90080
:101230000500200005007800721702000000000081
:101240000040B3004220AF00050037008502E800EF
:1012500036EDB7002424020000000000F5FF37003F
:1012600028C8BF0036EDB7002424020000000000AB
:1012700027C8BF00800278000B60EF000600200046
:10128000050078008600780004002000E22B0200B0
:101290000000000000C2B30036EDB70024240200B5
:1012A0000000000000C2B30036EDB70024240200A5
:1012B0000000000010C4B3003AEDB70030C0B30026
:1012C0003BEDB700A62002000000000006E8A900E0
:1012D000050020000500780046170200000000000D
:1012E0000040B3004220AF00050037008502E8004F
:1012F00036EDB7002424020000000000F5FF37009F
:101300009F003700746080004822DE006624E10000
:101310009B003A00010020000100780084170200C1
:10132000000000008100E8003322AF00FEFF37001C
:10133000A0118800400020000008E600F6FF3700FA
:10134000000020004140800052408000BC35020077
:101350000000000029002000743802000000000096
:10136000A1002000010078008417020000000000A6
:101370008100E8003322AF00FEFF3700A011880093
:10138000D00020000008E600F6FF37003A6DEF00BD
:101390003B6DEF00A6200200000000006029EF0076
:1013A0004300A9004040800051408000F226210007
:1013B00033A82300F62E020000000000800278000F
:1013C0000103780005007800860078000200200004
:1013D000A347240080300200000000008003780052
:1013E00001047800000020008700780008017800E0
:1013F000BC3502000000000029002000A63A0200CF
:101400000000000070C2B3003AEDB70020C0B30086
:101410003BEDB700A62002000000000000CEB300A4
:101420003AEDB700CC2002000000000000CEB3006F
:101430003AEDB700CC2002000000000000CEB3005F
:101440003AEDB700CC20020000000000B0C3B300AA
:101450003AEDB70020C0B3003BEDB700A620020074
:10146000000000003A6DEF00CC20020000000000F8
:101470003A6DEF00CC200200000000003A6DEF0052
:10148000CC2002000000000030C0B30030EDB700F7
:101490002E240200000000003A6DEF0030C0B300BF
:1014A0003BEDB700A62002000000000006E8A900FE
:1014B0000500200005007800A017020000000000D1
:1014C0000040B3004220AF00050037008502E8006D
:1014D00036EDB7002424020000000000F5FF3700BD
:1014E00028C8BF0036EDB700242402000000000029
:1014F00027C8BF00800278000B60EF0006002000C4
:10150000050078008600780004002000E22B02002D
:101510000000000000C2B30036EDB7002424020032
:101520000000000000C2B30036EDB7002424020022
:101530000000000010C4B3003AEDB70030C0B300A3
:101540003BEDB700A62002000000000006E8A9005D
:10155000050020000500780046170200000000008A
:101560000040B3004220AF00050037008502E800CC
:1015700036EDB7002424020000000000F5FF37001C
:101580008560A9005F0037003E4CE20015003A007C
:1015900005002000050078000E1F0200000000007A
:1015A0000040B3004220AF00060037008502E8008B
:1015B0003322AF00FEFF370034E2B7003562EF00A0
:1015C000F4FF37003322AF00FEFF37000402200093
:1015D000A41188003C610200000000008560A900A1
:1015E000480037003F4CE20015003A00050020009B
:1015F00005007800261F0200000000000040B30034
:101600004220AF00060037008502E8003322AF0019
:10161000FEFF370034E2B7003562EF00F4FF370019
:101620003322AF00FEFF370004022000A41188001F
:10163000BC2C0200000000008560A90031003700CA
:10164000484CE20015003A00050020000500780033
:101650003E1F0200000000000040B3004220AF0027
:10166000060037008502E8003322AF00FEFF370096
:1016700034E2B7003562EF00F4FF37003322AF00E9
:10168000FEFF370004022000A4118800244E02004F
:10169000000000008560A9001A003700494CE200F4
:1016A00018003A000500200005007800261C020002
:1016B000000000000040B3004220AF0006003700E9
:1016C0008502E8003322AF00FEFF370034E2B700A6
:1016D0003562EF00F4FF37003322AF00FEFF370022
:1016E00004022000A4118800304A0200000000001B
:1016F0006452020000000000DC79020000000000DB
:101700008560A90002002000A18520000200780069
:10171000561F020000000000805878000201E80017
:101720000004E0004220AE00F8FF37005868EF00E8
:10173000CF02780000000600851F7800861F780021
:1017400001002000010078003216020000000000B5
:101750008100E8003322AF00FEFF3700A0118800AF
:10176000400120000008E600F6FF37000FCCBF0064
:101770000160EF0004002000C82402000000000007
:101780007101200001007800321602000000000004
:101790008100E8003322AF00FEFF3700A01188006F
:1017A000A00120000008E600F6FF3700A0C2B30049
:1017B00028E8B7000F4CE20009003A0005002000BD
:1017C0002642240010C0B30021EDB700156988003F
:1017D00026698800EC3C0200000000004C00370045
:1017E000746080004822DE006124E10009003A00B4
:1017F00005002000B636240020C0B30021EDB7005C
:101800001569880026698800EC3C02000000000091
:101810003F003700746080004822DE006224E1004F
:1018200009003A0005002C00F650240030C0B30037
:1018300021EDB7001569880026698800EC3C02009C
:101840000000000032003700746080004822DE0093
:101850006324E10009003A0005002400665F2400CB
:1018600040C0B30021EDB7001569880026698800E3
:10187000EC3C02000000000025003700746080008E
:101880004822DE006424E10009003A0005002B0034
:101890003663240050C0B30021EDB70015698800FD
:1018A00026698800EC3C02000000000018003700A8
:1018B000746080004822DE006524E10009003A00DF
:1018C00005002200B66C240060C0B30021EDB70013
:1018D0001569880026698800EC3C020000000000C1
:1018E0000B003700746080004822DE006624E100AF
:1018F00007003A0005002000862B2400216DEF0030
:101900001569880026698800EC3C02000000000090
:101910004F037800CF02780000000600851F780092
:10192000D222EF0004802000B416880000000000DE
:1019300000000000F43F200094168800D742A80061
:10194000D342A9000000000000000000D282A800DD
:10195000D482AE002B0037002F6CEF000500200072
:10196000050078003E1C0200000000000040B300AB
:101970004220AF00060037008502E8003322AF00A6
:10198000FEFF370034E2B7003562EF00F4FF3700A6
:10199000D282A800D482AE000B0037002F6CEC007E
:1019A00050002000641F02000000000074618000ED
:1019B0004822DE00A30F2000041CE10001003E00CD
:1019C00001003700F2FF3700746180004822DE001A
:1019D000A30F2000041CE10003003E009C8B0200CA
:1019E0000000000006003700746180004822DE001D
:1019F0006124E100020039003C61020000000000A7
:101A0000D1003700D262A800D462AE002D003700AA
:101A10002968EF000100200001007800561C020038
:101A2000000000008100E8003322AF00FEFF370015
:101A3000A0118800900020000008E600F6FF3700A3
:101A4000D262A800D462AE000B0037002968EC0017
:101A500050002000641F020000000000444180008C
:101A60004822DE00A30F2000041CE10001003E001C
:101A700001003700F2FF3700444180004822DE00B9
:101A8000A30F2000041CE10004003E005C6CEF008A
:101A9000D0780200000000000900370044418000B7
:101AA0004822DE006124E10005003900A0C2B30035
:101AB00028E8B7005C6CEF008252020000000000D2
:101AC000A1003700D242A800D442AE002C0037005B
:101AD0002A68EF0001002000010078006E1C02005F
:101AE000000000008100E8003322AF00FEFF370055
:101AF000A0118800A00020000008E600F6FF3700D3
:101B0000D242A800D442AE000A0037002A68EC0096
:101B100050002000641F02000000000054418000BB
:101B2000A30F2000041CE10001003E00010037006B
:101B3000F3FF370054418000A30F2000041CE10094
:101B400005003E0010C0B3005CECB700D078020086
:101B50000000000009003700544180006124E100CA
:101B600006003900A0C2B30028E8B70010C0B300D7
:101B70005CECB700825202000000000072003700E7
:101B8000D202A800D402AE003500370001002000C8
:101B900001007800861C0200000000008100E800BF
:101BA0003322AF00FEFF3700A01188007000200034
:101BB0000008E600F6FF3700F41F200004638800E9
:101BC000BE270200000000002CECB700010020003E
:101BD000010078009C1C0200000000008100E80069
:101BE0003322AF00FEFF3700A011880070002000F4
:101BF0000008E600F6FF37002CCCBF000160EF00C4
:101C000004002000C8240200000000003322AF00BE
:101C1000FEFF370004022000A41188002C6CED00A8
:101C20002C4CE20001003A002C6CEF0010C3B30012
:101C30001CEDB7002CCCBF001DEDB700B42802008E
:101C4000000000002CCCBF001EEDB700F41F2000E8
:101C5000E4688800362B0200000000003A003700DC
:101C6000D222A800D422AE003700370001002000A5
:101C700001007800B41C0200000000008100E800B0
:101C80003322AF00FEFF3700A01188009000200033
:101C90000008E600F6FF3700F41F20000463880008
:101CA000BE270200000000002CECB700010020005D
:101CB000010078009C1C0200000000008100E80088
:101CC0003322AF00FEFF3700A01188007000200013
:101CD0000008E600F6FF37002CCCBF000160EF00E3
:101CE00004002000C8240200000000003322AF00DE
:101CF000FEFF370004022000A41188002C6CEC00C9
:101D000064618000F3072000041CE1000200310040
:101D1000F0C7B3002CECB70010C3B3001CEDB70044
:101D20002CCCBF001DEDB700B4280200000000005D
:101D30002CCCBF001EEDB700F41F2000E468880023
:101D4000362B020000000000D282A800D482AE0030
:101D500004003700A0002000641F02000000000003
:101D6000F9FF3700D262A800D462AE000400370049
:101D7000A0002000641F020000000000F9FF3700EF
:101D8000D242A800D442AE0004003700A0002000D8
:101D9000641F020000000000F9FF3700D202A80013
:101DA000D402AE0004003700A0002000641F02002F
:101DB00000000000F9FF3700D222A800D422AE00B4
:101DC00004003700A0002000641F02000000000093
:101DD000F9FF37007A25020000000000CF027800EA
:101DE00000000600851F7800861F78000001EB00C8
:101DF0000103780064C110004211DD000200DD0023
:101E0000800278000C60EC000C60ED000D003200E8
:101E100005007800C42ADD004C00DE00F000B200AE
:101E20000003B000A20320000200E100010039001D
:101E30000D40B40036EDB70024240200000000007D
:101E4000F1FF37004F037800CF0278000000060052
:101E5000851F7800C500200003000900B51F780029
:101E600000037800810378000406780004F0A100E4
:101E70000400E00006003A0009F0A7000200370065
:101E80000500200013003700050020001100370076
:101E9000EB4252000E0039000003200009F0A600BA
:101EA000000220003322AF00FEFF3700A01188009F
:101EB00041E0AF00FBFF3700801088001162EF00A7
:101EC0008502E900F7FF3B005500200001003700C4
:101ED00084027800E8002000090020001000FA00C9
:101EE0000C377C000884E900FDFF3B00A4002000C3
:101EF00005E0A0000CF0A70005F0A000040F78009A
:101F000015079800060078008700780002A02C00D2
:101F1000A3B92300087122000DF0A1000DF0A2006A
:101F20009E2B0200000000000DF0A7000700370004
:101F3000400798005107980000017800810178005F
:101F40002E009000BE009000F4FF3700420798007A
:101F50005307980024079800350798001E02780060
:101F60009E029000060320000000E00012003A00EC
:101F700005E0A600120037000402E900040F780013
:101F80000400E0000E0032000524E10002003200EF
:101F90004200AF000E003700060320000000E00002
:101FA00005003A0005E0A6000500370005F0A60090
:101FB000060220000200370005E0A1001507980086
:101FC000004043003322AF00FEFF3700A01188001D
:101FD0004E009000DE009000A20020008001EB0087
:101FE0006100E10001003200CCFF37000080FA0000
:101FF0002501200003000900CF127800CF027800ED
:1020000000000600851F7800861F78000E28EC006F
:102010004220AF001028EC001228EC004220AF0054
:102020001428EC00844080006020E1003107390072
:1020300004003E0074408000830C20000418E1007E
:102040002C073E000E28EF001028EF000F4CE20096
:102050000100320026073700844B80006424E10031
:1020600001003E00220737000F4CE200CD003A008D
:102070004300A9004040800051408000F22621002A
:1020800033B02300F62E020000000000800278002A
:102090000103780001002000010078005A160200B8
:1020A000000000008100E8003322AF00FEFF37008F
:1020B000A0118800500020000008E600F6FF37005D
:1020C000000020008500780006017800BC35020081
:1020D0000000000029002000743802000000000009
:1020E000B1002000010078005A1602000000000034
:1020F0008100E8003322AF00FEFF3700A011880006
:10210000E00020000008E600F6FF37003A6DEF001F
:102110003B6DEF00A6200200000000006029EF00E8
:102120004300A9004040800051408000F226210079
:1021300033A82300F62E0200000000008002780081
:102140000103780005007800860078000200200076
:10215000832C24008E2E0200000000003300390082
:102160004300A9004040800051408000F226210039
:1021700033B02300F62E0200000000008002780039
:102180000103780000002000850078000601780037
:10219000BC3502000000000029002000A63A020021
:1021A0000000000070C2B3003AEDB70020C0B300D9
:1021B0003BEDB700A62002000000000000CEB300F7
:1021C0003AEDB700CC2002000000000000CEB300C2
:1021D0003AEDB700CC2002000000000000CEB300B2
:1021E0003AEDB700CC20020000000000B0C3B300FD
:1021F0003AEDB70020C0B3003BEDB700A6200200C7
:10220000000000003A6DEF00CC200200000000004A
:102210003A6DEF00CC200200000000003A6DEF00A4
:10222000CC20020000000000320037004300A9006B
:102230004040800051408000F226210033B023004E
:10224000F62E0200000000008002780001037800F2
:10225000000020008500780006017800BC350200EF
:102260000000000019002000A63A02000000000053
:1022700070C2B3003AEDB70020C0B3003BEDB70029
:10228000A6200200000000003A6DEF00CC20020002
:10229000000000003A6DEF00CC20020000000000BA
:1022A0003A6DEF00CC20020000000000B0C3B30084
:1022B0003AEDB70020C0B3003BEDB700A620020006
:1022C0000000000000CEB3003AEDB700CC200200C1
:1022D0000000000000CEB3003AEDB700CC200200B1
:1022E0000000000000CEB3003AEDB700CC200200A1
:1022F0000000000030C0B30030EDB7002E24020013
:10230000000000003A6DEF0030C0B3003BEDB700B5
:10231000A62002000000000006E8A9000500200039
:102320000500780076160200000000000040B300AF
:102330004220AF00050037008502E80036EDB70007
:102340002424020000000000F5FF370028C8BF0069
:1023500036EDB700242402000000000027C8BF00AB
:10236000800278000B60EF00060020000500780076
:102370008600780004002000E22B0200000000002C
:1023800000C2B30036EDB7002424020000000000B4
:1023900000C2B30036EDB7002424020000000000A4
:1023A00036043700746080004822DE006124E100BA
:1023B00094003A0001002000010078008616020017
:1023C000000000008100E8003322AF00FEFF37006C
:1023D000A0118800300020000008E600F6FF37005A
:1023E000000020004140800052408000BC350200C7
:1023F00000000000290020007438020000000000E6
:102400009100200001007800861602000000000004
:102410008100E8003322AF00FEFF3700A0118800E2
:10242000C00020000008E600F6FF37003A6DEF001C
:102430003B6DEF00A6200200000000006029EF00C5
:102440004300A9004040800051408000F226210056
:1024500033A82300F62E020000000000800278005E
:102460000103780000002000850078000601780054
:10247000BC3502000000000019002000A63A02004E
:102480000000000070C2B3003AEDB70020C0B300F6
:102490003BEDB700A6200200000000003A6DEF00FF
:1024A000CC200200000000003A6DEF00CC200200BA
:1024B000000000003A6DEF00CC2002000000000098
:1024C000B0C3B3003AEDB70020C0B3003BEDB70096
:1024D000A62002000000000000CEB3003AEDB700D5
:1024E000CC2002000000000000CEB3003AEDB7009F
:1024F000CC2002000000000000CEB3003AEDB7008F
:10250000CC2002000000000030C0B30030EDB70066
:102510002E240200000000003A6DEF0030C0B3002E
:102520003BEDB700A62002000000000006E8A9006D
:102530000500200005007800A01602000000000041
:102540000040B3004220AF00050037008502E800DC
:1025500036EDB7002424020000000000F5FF37002C
:1025600028C8BF0036EDB700242402000000000098
:1025700027C8BF00800278000B60EF000600200033
:10258000050078008600780004002000E22B02009D
:102590000000000000C2B30036EDB70024240200A2
:1025A0000000000000C2B30036EDB7002424020092
:1025B0000000000010C4B3003AEDB70030C0B30013
:1025C0003BEDB700A62002000000000006E8A900CD
:1025D0000500200005007800B01602000000000091
:1025E0000040B3004220AF00050037008502E8003C
:1025F00036EDB7002424020000000000F5FF37008C
:102600009E033700746080004822DE006224E100EF
:1026100094003A000100200001007800C01602007A
:10262000000000008100E8003322AF00FEFF370009
:10263000A0118800300020000008E600F6FF3700F7
:10264000000020004140800052408000BC35020064
:102650000000000029002000743802000000000083
:102660009100200001007800C01602000000000068
:102670008100E8003322AF00FEFF3700A011880080
:10268000C00020000008E600F6FF37003A6DEF00BA
:102690003B6DEF00A6200200000000006029EF0063
:1026A0004300A9004040800051408000F2262100F4
:1026B00033A82300F62E02000000000080027800FC
:1026C00001037800000020008500780006017800F2
:1026D000BC3502000000000019002000A63A0200EC
:1026E0000000000070C2B3003AEDB70020C0B30094
:1026F0003BEDB700A6200200000000003A6DEF009D
:10270000CC200200000000003A6DEF00CC20020057
:10271000000000003A6DEF00CC2002000000000035
:10272000B0C3B3003AEDB70020C0B3003BEDB70033
:10273000A62002000000000000CEB3003AEDB70072
:10274000CC2002000000000000CEB3003AEDB7003C
:10275000CC2002000000000000CEB3003AEDB7002C
:10276000CC2002000000000030C0B30030EDB70004
:102770002E240200000000003A6DEF0030C0B300CC
:102780003BEDB700A62002000000000006E8A9000B
:102790000500200005007800DA16020000000000A5
:1027A0000040B3004220AF00050037008502E8007A
:1027B00036EDB7002424020000000000F5FF3700CA
:1027C00028C8BF0036EDB700242402000000000036
:1027D00027C8BF00800278000B60EF0006002000D1
:1027E000050078008600780004002000E22B02003B
:1027F0000000000000C2B30036EDB7002424020040
:102800000000000000C2B30036EDB700242402002F
:102810000000000010C4B3003AEDB70030C0B300B0
:102820003BEDB700A62002000000000006E8A9006A
:102830000500200005007800B0160200000000002E
:102840000040B3004220AF00050037008502E800D9
:1028500036EDB7002424020000000000F5FF370029
:1028600006033700746080004822DE006324E10024
:1028700099003A000100200001007800EA160200E9
:10288000000000008100E8003322AF00FEFF3700A7
:10289000A0118800400020000008E600F6FF370085
:1028A000000020004140800052408000BC35020002
:1028B0000000000029002000743802000000000021
:1028C000A100200001007800EA16020000000000CC
:1028D0008100E8003322AF00FEFF3700A01188001E
:1028E000D00020000008E600F6FF37003A6DEF0048
:1028F0003B6DEF00A6200200000000006029EF0001
:102900004300A9004040800051408000F226210091
:1029100033A82300F62E0200000000008002780099
:10292000010378000500780086007800020020008E
:1029300003122400803002000000000080037800B1
:10294000010478000000200087007800080178006A
:10295000BC3502000000000019002000A63A020069
:102960000000000070C2B3003AEDB70020C0B30011
:102970003BEDB700A6200200000000003A6DEF001A
:10298000CC200200000000003A6DEF00CC200200D5
:10299000000000003A6DEF00CC20020000000000B3
:1029A000B0C3B3003AEDB70020C0B3003BEDB700B1
:1029B000A6200200000000003A6DEF00CC200200CB
:1029C000000000003A6DEF00CC2002000000000083
:1029D0003A6DEF00CC2002000000000030C0B300D0
:1029E00030EDB7002E240200000000003A6DEF0029
:1029F00030C0B3003BEDB700A6200200000000008D
:102A000006E8A9000500200005007800061702006E
:102A1000000000000040B3004220AF000500370076
:102A20008502E80036EDB700242402000000000013
:102A3000F5FF370028C8BF0036EDB7002424020098
:102A40000000000027C8BF00800278000B60EF0084
:102A500006002000050078008600780004002000B1
:102A6000E22B02000000000000C2B30036EDB70008
:102A7000242402000000000000C2B30036EDB700BD
:102A8000242402000000000010C4B3003AEDB70097
:102A900030C0B3003BEDB700A620020000000000EC
:102AA00006E8A9000500200005007800B016020025
:102AB000000000000040B3004220AF0005003700D6
:102AC0008502E80036EDB700242402000000000073
:102AD000F5FF370069023700746080004822DE008D
:102AE0006424E10026013A00010020000100780082
:102AF00018170200000000008100E8003322AF0038
:102B0000FEFF3700A0118800400020000008E6000A
:102B1000F6FF370000002000414080005240800056
:102B2000BC350200000000002900200074380200BB
:102B300000000000A100200001007800181702002A
:102B4000000000008100E8003322AF00FEFF3700E4
:102B5000A0118800D00020000008E600F6FF370032
:102B6000404080005140800002002400C3612400E6
:102B70008E2E0200000000007B0039003A6DEF004D
:102B80003B6DEF00A6200200000000006029EF006E
:102B90004300A9004040800051408000F2262100FF
:102BA00033A82300F62E0200000000008002780007
:102BB00001037800050078008600780002002000FC
:102BC000031224008030020000000000800378001F
:102BD00001047800000020008700780008017800D8
:102BE000BC3502000000000019002000A63A0200D7
:102BF0000000000070C2B3003AEDB70020C0B3007F
:102C00003BEDB700A6200200000000003A6DEF0087
:102C1000CC200200000000003A6DEF00CC20020042
:102C2000000000003A6DEF00CC2002000000000020
:102C3000B0C3B3003AEDB70020C0B3003BEDB7001E
:102C4000A6200200000000003A6DEF00CC20020038
:102C5000000000003A6DEF00CC20020000000000F0
:102C60003A6DEF00CC2002000000000030C0B3003D
:102C700030EDB7002E240200000000003A6DEF0096
:102C800030C0B3003BEDB700A620020000000000FA
:102C900006E8A900050020000500780034170200AE
:102CA000000000000040B3004220AF0005003700E4
:102CB0008502E80036EDB700242402000000000081
:102CC000F5FF370028C8BF0036EDB7002424020006
:102CD0000000000027C8BF00800278000B60EF00F2
:102CE000060020000500780086007800040020001F
:102CF000E22B02000000000000C2B30036EDB70076
:102D0000242402000000000000C2B30036EDB7002A
:102D1000242402000000000010C4B3003AEDB70004
:102D200030C0B3003BEDB700A62002000000000059
:102D300006E8A9000500200005007800B016020092
:102D4000000000000040B3004220AF000500370043
:102D50008502E80036EDB7002424020000000000E0
:102D6000F5FF37008500370000002400C161240012
:102D700042408000534080008E2E02000000000080
:102D8000010031007D003A003A6DEF003B6DEF002D
:102D9000A6200200000000006029EF004300A90007
:102DA0004040800051408000F226210033A82300DB
:102DB000F62E020000000000800278000103780077
:102DC000050078008600780002002000A347240058
:102DD00080300200000000008003780001047800C9
:102DE000000020008700780008017800BC35020050
:102DF0000000000029002000A63A020000000000A8
:102E000070C2B3003AEDB70020C0B3003BEDB7008D
:102E1000A62002000000000000CEB3003AEDB7008B
:102E2000CC2002000000000000CEB3003AEDB70055
:102E3000CC2002000000000000CEB3003AEDB70045
:102E4000CC20020000000000B0C3B3003AEDB70090
:102E500020C0B3003BEDB700A62002000000000038
:102E60003A6DEF00CC200200000000003A6DEF0048
:102E7000CC200200000000003A6DEF00CC200200E0
:102E80000000000030C0B30030EDB7002E24020077
:102E9000000000003A6DEF0030C0B3003BEDB7001A
:102EA000A62002000000000006E8A900050020009E
:102EB0000500780034170200000000000040B30055
:102EC0004220AF00050037008502E80036EDB7006C
:102ED0002424020000000000F5FF370028C8BF00CE
:102EE00036EDB700242402000000000027C8BF0010
:102EF000800278000B60EF000600200005007800DB
:102F00008600780004002000E22B02000000000090
:102F100000C2B30036EDB700242402000000000018
:102F200000C2B30036EDB700242402000000000008
:102F300010C4B3003AEDB70030C0B3003BEDB700AA
:102F4000A62002000000000006E8A90005002000FD
:102F50000500780046170200000000000040B300A2
:102F60004220AF00050037008502E80036EDB700CB
:102F70002424020000000000F5FF37003F01370065
:102F8000746080004822DE006524E1009C003A0065
:102F90000100200001007800561702000000000028
:102FA0008100E8003322AF00FEFF3700A011880047
:102FB000400020000008E600F6FF37000000200077
:102FC0004140800052408000BC35020000000000FB
:102FD000290020007438020000000000A100200039
:102FE0000100780056170200000000008100E80090
:102FF0003322AF00FEFF3700A0118800D000200070
:103000000008E600F6FF37003A6DEF003B6DEF0079
:10301000A6200200000000006029EF004300A90084
:103020004040800051408000F226210033A8230058
:10303000F62E0200000000008002780001037800F4
:10304000050078008600780002002000A3472400D5
:103050008030020000000000800378000104780046
:10306000000020008700780008017800BC350200CD
:103070000000000029002000A63A02000000000025
:1030800070C2B3003AEDB70020C0B3003BEDB7000B
:10309000A62002000000000000CEB3003AEDB70009
:1030A000CC2002000000000000CEB3003AEDB700D3
:1030B000CC2002000000000000CEB3003AEDB700C3
:1030C000CC20020000000000B0C3B3003AEDB7000E
:1030D00020C0B3003BEDB700A620020000000000B6
:1030E0003A6DEF00CC200200000000003A6DEF00C6
:1030F000CC200200000000003A6DEF00CC2002005E
:103100000000000030C0B30030EDB7002E240200F4
:10311000000000003A6DEF0030C0B3003BEDB70097
:10312000A62002000000000006E8A900050020001B
:103130000500780072170200000000000040B30094
:103140004220AF00050037008502E80036EDB700E9
:103150002424020000000000F5FF370028C8BF004B
:1031600036EDB700242402000000000027C8BF008D
:10317000800278000B60EF00060020000500780058
:103180008600780004002000E22B0200000000000E
:1031900000C2B30036EDB700242402000000000096
:1031A00000C2B30036EDB700242402000000000086
:1031B00010C4B3003AEDB70030C0B3003BEDB70028
:1031C000A62002000000000006E8A900050020007B
:1031D0000500780046170200000000000040B30020
:1031E0004220AF00050037008502E80036EDB70049
:1031F0002424020000000000F5FF37009F00370084
:10320000746080004822DE006624E1009B003A00E2
:103210000100200001007800841702000000000077
:103220008100E8003322AF00FEFF3700A0118800C4
:10323000400020000008E600F6FF370000002000F4
:103240004140800052408000BC3502000000000078
:10325000290020007438020000000000A1002000B6
